:020000040800F2
:10C000003013012001600208D17F0208197E020866
:10C01000CF7F020815720208018C020800000000A0
:10C020000000000000000000000000001381020872
:10C03000457302080000000011810208D98302083C
:10C040001B6002081B6002081B6002081B600208DC
:10C050001B6002081B6002081B6002081B600208CC
:10C060001B6002081B6002081B6002086D72020858
:10C070001B600208BDC10008C57202081B600208EF
:10C080001B600208057302081B6002081B6002089F
:10C09000758B02081B600208197202081B600208F7
:10C0A0001B6002081B6002081B6002081B6002087C
:10C0B000618402081B6002081B6002081B60020802
:10C0C0001B6002081B6002081B6002081B6002085C
:10C0D0001B6002088D8A0208018B02081B6002089F
:10C0E0001B6002081B6002081B6002081B6002083C
:10C0F0001B6002081B6002081B6002081B6002082C
:10C100001B6002081B6002081B6002081B6002081B
:10C110001B6002081B6002081B6002081B6002080B
:10C120001B6002081B6002081B6002081B600208FB
:10C130001B6002081B6002081B6002081B600208EB
:10C1400000000000000000000000000000000000EF
:10C150001B6002081B6002081B6002081B600208CB
:10C160001B6002081B6002081B6002081B600208BB
:10C170001B6002081B6002081B6002081B600208AB
:10C180001B600208DFF80CD000F006F800480047FA
:10C19000F32E030830130120064C074D06E0E0683B
:10C1A00040F0010394E8070098471034AC42F6D3FE
:10C1B000FFF7ECFFC49D0108E49D010810B54FF4A2
:10C1C0000074204621F042F9002819D0204621F0C1
:10C1D000ADF80C4813F072FE0B4C802120682AF059
:10C1E0002AF90028F9D1002108482AF01FF9002176
:10C1F000074821F085F8BDE8104001201BF0BCBEC7
:10C2000010BD00002C7B00201433002000300140C2
:10C210003000024002E008C8121F08C1002AFAD10B
:10C2200070477047002001E001C1121F002AFBD1B6
:10C230007047000010B5442107480EF06AFB002249
:10C24000062106480BF0ECFE054CA06000F074FBE4
:10C250000020207010BD0000207D0020EDC90008E6
:10C2600044350020F8B5044617F0ACFE0026374DE3
:10C270000746009634B1E068686020460BF09EFFE8
:10C28000686802E013F020FE686000690BF078FD3A
:10C290006868406908B10BF073FD6868C0690BF00D
:10C2A0006FFD6868006A0BF06BFD6868016991B109
:10C2B0000BF0FEFD0CF010FE0CF05EFC6868B0F8B0
:10C2C0005011D9B30068017CC9071DD0C06840680F
:10C2D000D0B1002413E0A0F85061F8BD011991F825
:10C2E000301151B900F5AC700EF06AFB696801EBD2
:10C2F000C4010A6B0260496B4160641CA4B26868A7
:10C30000B0F85011A142E9D868684FF4807130301C
:10C3100016F0A1FA6868202100F5987016F09BFAD3
:10C320006868A0F85061384617F045FE00906868CC
:10C330000068436A13B12A680099984716F00CF90F
:10C340000DF0BAFFBDE8F84000F002B8C03400209C
:10C3500070B5094E0024C4EBC40556F8250008B199
:10C3600016F06EF906EB85001C2116F074FA641CB9
:10C37000E4B2042CEFD370BD3C7E00207FB50D46A7
:10C38000040003D113F0A0FD04002CD013F010FE24
:10C39000002828D094F82800400724D4002605B3AC
:10C3A000ADF80060ADF80260204613F0A5FD401E18
:10C3B000ADF80400204613F0E5FD401EADF8060080
:10C3C0006A46294602A80DF0C4FD00280BD020685B
:10C3D000017C890708D5DDE90001C4E90C010120D1
:10C3E00029E0A4F850617FBD82690AB102A9904793
:10C3F00000250AE004EBC501002202A830310DF04F
:10C40000D0FD0028EFD16D1CADB2B4F85001A842A8
:10C41000F0D880B2202804D204EBC00002A930304A
:10C4200004E0A4F8506104F13000694605F082F997
:10C43000B4F85001401CA4F8500160680028D2D024
:10C440000BF0CEFE7FBD10B50446006882680AB1CD
:10C450002146904720680068002801D02060F5E759
:10C4600010BD8068002801D0B0F9160070478068C0
:10C47000002801D0807E8009704770B515460646B9
:10C480000C4651EA05001AD0304608F05BFAB06855
:10C4900001232A46018A21440182B068418A294445
:10C4A0004182214630460AF023FB00220B21304610
:10C4B00013F0FCFD012803D130460AF072FA012086
:10C4C00070BD77B581B00E46050017D0622209F025
:10C4D0006CFE040012D0206880B1284631466322E9
:10C4E00009F063FE10F0FF0208D02368204603998C
:10C4F00098470090BDF80000ADF80C00039804B018
:10C5000070BD00002DE9F047054692B0408C1A9CA2
:10C5100040F00800688490462A8499468A46228919
:10C52000284609F042FE0646A5F820902289514689
:10C53000284609F03AFE0746688CBE4220F0080003
:10C54000688403D13104B1EB074F68D0A5F820808F
:10C5500022895146284609F028FE06468046A5F85D
:10C5600020905146284604F08CFC21890068324610
:10C5700017F0FCFA20890B2823D147F6FF794E45A6
:10C5800001D04F451DD1284609F05BFF00EBD0706C
:10C590004610284609F069F800EBD0704010C845F5
:10C5A00006D1711C431C994200DA00E01946884606
:10C5B0004F4506D1711C421C914201DA0F4600E042
:10C5C000174619480EF0ADF906002BD03560C6E9C4
:10C5D00003872089B0806846C6F808A004F0D0FF21
:10C5E0001248FF21CDE900601148029011480390E4
:10C5F00000200890CDE9090120880B9060889DF803
:10C60000421040420C90E0680790002060F3000167
:10C610008DF8421020690690684605F03BF812B08C
:10C62000BDE8F087FEE70000447D0020E5970108A3
:10C63000E999010841990108142101480EF069B9EE
:10C64000447D00202DE9F84F002490468946064697
:10C6500025464FF0040AE3E0F1680AEBC5000858EC
:10C6600082017AD480B230EA090210D0002230EA86
:10C6700008000ED0002082426FD051F835706A4613
:10C680001021384617F072F8002871D103E001221A
:10C69000EDE70120EFE76A461121384617F066F80A
:10C6A000002865D16A461221384617F05FF8002845
:10C6B0005ED16A461321384617F058F8002857D142
:10C6C0006A461521384617F051F8002850D16A46BD
:10C6D0001421384617F04AF8F0BB6A460A2138465A
:10C6E00017F044F8C0BB6A466B21384617F03EF895
:10C6F00090BB6A466C21384617F038F860BB6A4632
:10C700000121384617F032F830BB6A46042138461A
:10C7100017F02CF800BB6A460221384617F026F8BD
:10C72000D0B96A460321384617F020F8A0B96A4606
:10C730000521384617F01AF870B96A4606213846BE
:10C7400017F014F840B96A463221384617F00EF84F
:10C7500010B96A466E2101E00AE060E0384617F041
:10C7600005F828B96A466D21384616F0FFFF10B16A
:10C770000320BDE8F88F6A466921384616F0F6FFB7
:10C78000F0BB6A466A21384616F0F0FFC0BB6A4625
:10C790006E21384616F0EAFF90BB6A466D21384696
:10C7A00016F0E4FF60BB6A463721384616F0DEFF1C
:10C7B00030BB6A463821384616F0D8FF00BB6A46BF
:10C7C0003521384616F0D2FFD0B96A4640213846A6
:10C7D00016F0CCFFA0B96A464521384616F0C6FFD0
:10C7E00070B96A464121384616F0C0FF40B96A4622
:10C7F0004221384616F0BAFF10B96A46432100E0DC
:10C8000009E0384616F0B2FF28B96A464921384691
:10C8100016F0ACFF08B1022401E004B901246D1C3C
:10C82000708CC0F30510A8423FF616AF2046A0E773
:10C830000148406870470000C03400207047000085
:10C8400010B5182103480EF064F803490120087060
:10C8500010BD0000F07C00208C3500202DE9F84F41
:10C860008146407A0D4600F00700022819D0104694
:10C870008046954200DD2A46164603202A4F2B4B60
:10C8800000EB460020F00304B86819681034411A20
:10C890007A6804EB010C944505D2416821F000410F
:10C8A00024E00846E4E7944219D89A464FF0FF3B4B
:10C8B00008197968884210D9002269461C48CDF8C9
:10C8C00000B004F053FB002269461A4804F04EFB06
:10C8D000B968DAF80000091AEAE7B868DDE7204627
:10C8E00015F022FEC0B1416841F0004188EA6502BE
:10C8F000416089EA02010160416801F04041491C40
:10C9000031F0804141608681A0F80E8005D500F1AC
:10C9100010018160BDE8F88FFEE7B96801F11002EF
:10C9200021448260B960F5E7C83400206C350020EE
:10C93000330A0108E90F010810B5084C01202070E6
:10C9400007480DF0C9FF0028A06803D0BDE81040DB
:10C950000BF046BCBDE810400BF030BC4435002065
:10C96000207D002010B5044690F84200A16B82079C
:10C9700009D4B4F840204AB1A2F57F43FF3B1BD055
:10C98000521EA4F84020B4F84020AAB909B1820789
:10C9900012D5214614480EF03AF8FFF7CDFFE168B2
:10C9A00009B120468847216909B1204688472046B9
:10C9B000BDE8104015F044BEE26B524222630029EC
:10C9C00011D0820702D4626B524222634210521C81
:10C9D00062F3410084F84200A26A206A2262A062E7
:10C9E000E06AE162A06310BD207D002070B5304E8A
:10C9F000706817F0E0FA0546707880F001007070FA
:10CA000047E00020307094F842007178C0F3800253
:10CA10008A4242D061F3820084F84200216B4A19B5
:10CA2000030719D4002917DC002A15DBC00709D138
:10CA3000616939B120468847216A01442162A16AAF
:10CA40000844A062A16809B12046884794F84200D2
:10CA500040F0080084F84200206B4019206316D48F
:10CA6000E16A884200DD2163E1692046884701468A
:10CA7000606A884204D0616262680AB120689047A7
:10CA8000D4E90B01814202DB2046FFF76BFF3078CF
:10CA900018B108480DF020FF03E0214605480DF0CD
:10CAA0002DFF0400ADD117F08DFA706070BD00004D
:10CAB00044350020207D00202DE9FF4F8BB01E461D
:10CAC000DDE91801CDE90601002004901F981E9DA4
:10CAD000042809D0052809D006280CD014287CD1B8
:10CAE00001200290022004E00020FAE701200290D9
:10CAF0000320059008E00120029002200590FFF736
:10CB000097FE0068806B04900D98002416FB00F0DF
:10CB10000A900C98401E09900D98401E08902CE138
:10CB20001A980699604301EB20231B9807996043EC
:10CB300001EB202219124FEA222007D40C9FB942A0
:10CB400004DA002802DB0D9FB84201DB002011E16E
:10CB5000DBB2D2B2802B05DAC3F17F034FF0FF378F
:10CB60005B0003E001275B00A3F580739A46802AEF
:10CB700005DAC2F17F024FF0FF33520003E00123D8
:10CB80005200A2F58072914600FB0618DDF814C031
:10CB90000B9A08FB0C2201EB070C5FEA0C0E73D416
:10CBA000DDF82480C6456FDC10EB03086CD4DDF89B
:10CBB00020C0E04568DCDDF814C017FB0C2B13FB2C
:10CBC00006F707FB0C23029FF7B31F9F052F05D025
:10CBD000142F09D0062F47D053E0D2E092F802C0BC
:10CBE00099789BF8020010E0DDE90A7C0CEB47071E
:10CBF000394400FB06FC00FB067708FB06F81CF82E
:10CC000001C017F80E0018F80110614507D011FB9C
:10CC100009F7C9F580711CFB0171C1F3072160455B
:10CC200007D010FB0AF7CAF580701CFB0070C0F338
:10CC3000072008444008285556D01078517800EB5A
:10CC40000120ADF8000000E01FE01878597800EBF3
:10CC50000120ADF80C009BF800109BF8010001EBDF
:10CC60000020ADF804001CE00498118880B28142D5
:10CC70003FF46CAF19888142FAD0BBF800108142B2
:10CC8000F6D0FF210846D4E72FE01088ADF8000069
:10CC9000BBF80000ADF804001888ADF80C00FF20C8
:10CCA0002855BDF80000BDF80C10884203D1BDF82E
:10CCB0000410884212D009F0FF020099039804F092
:10CCC0009DFE0390DDE900100AF0FF0204F096FEDD
:10CCD0007F220190039904F091FE00901D98BDF809
:10CCE000001000EB4400018045E092F800C092F88B
:10CCF00001800CEB082C1FFA8CF8DDF874C02CF8BE
:10CD00001480DDF87CC0BCF1050F06D0BCF1060F25
:10CD100005D0BCF1140F08D109E092780FE0049A15
:10CD200092B2904501D1002209E0FF2207E00B9A60
:10CD300000FB062C0A9A01EB42021CF8022009B9FA
:10CD4000002F05DBDDF824C0614504D1002F02DD92
:10CD5000CAF1FF000BE008B9002B06DB08998842F6
:10CD60007FF4F4AE002B7FF7F1AEC9F1FF0010FBAA
:10CD700002F0000A2855641C24B21C988442FFF675
:10CD8000CFAE0FB0BDE8F08F2DE9F05F00228046F6
:10CD900011460AF043FD0021404609F06EF90446B1
:10CDA0000021404609F0F5F9204407B20021404631
:10CDB00009F0CBF920440FFA80FB404609F006F950
:10CDC000C11901EB0B000FFA80F9274C404608F01F
:10CDD00099FB824600252BE0D8F80800234900681B
:10CDE00050F82560304609F052FB00BB304609F090
:10CDF00031FE60BB0021304609F00CF938B3012840
:10CE000025D0022823D0032821D00021304609F064
:10CE10005FFA60B906F11400064604F0B8FC384425
:10CE2000A04203DB304604F0B2FCC41924B26D1CEE
:10CE30005545D1D341F6FF70C44212D004EB0B002C
:10CE400000B24946484500DC0846BDE8F09FB6F907
:10CE50001A10B8F91600081A411CA142E6DB0C466C
:10CE6000E4E74846F1E7000001E0FFFF01000400AD
:10CE70002DE9F05F0022054611460AF0B9FC0021B9
:10CE8000284609F0FAF804460021284609F075F909
:10CE900020440FFA80F90021284609F062F9204465
:10CEA0000FFA80F8284609F09FF800EB080101EB23
:10CEB00009000FFA80FB4B4C284608F023FB824602
:10CEC0000021284609F0ACF801284FF000062CD0CC
:10CED0006AE0A8684449006850F82670384609F0AE
:10CEE000D6FA08BB384609F0B5FD38BB00213846F4
:10CEF00009F090F810B3032820D006281ED0082887
:10CF00001CD00021384609F0DDF968B907F114009A
:10CF1000074604F05AFC4844A04204DB384604F0BB
:10CF200054FC00EB090424B2761C5645D1D341F6DB
:10CF3000FF70C44241D004EB08003DE0B5F9180091
:10CF4000B7F91410401A411CA142ECDB0C46EAE789
:10CF5000A8682549006850F82670384609F097FA05
:10CF600008BB384609F076FD88BB0021384609F039
:10CF700051F860B301282BD0042829D0072827D0E6
:10CF80000021384609F0A4F968B907F114000746F2
:10CF900004F01BFC4044A04204DB384604F015FCBE
:10CFA00000EB080424B2761C5645D1D341F6FF703D
:10CFB000C44202D004EB090004B241F6FF70C4423F
:10CFC000584602D05C4500DD2046BDE8F09FFFE7F3
:10CFD000B7F91800B5F91410401A411CA142E1DB61
:10CFE0000C46DFE701E0FFFF010004001CB50B88E1
:10CFF00004892344ADF800304B8844892344ADF8BC
:10D0000002308B8804892344ADF80430C9884389F1
:10D010001944ADF806104369694698471CBD2DE9CF
:10D02000F04F8BB05FEA010A054643D0A5F818A07F
:10D03000286808B115F004FB0AEB4A00062101EB51
:10D04000400015F071FA286058B3022202EB4A0141
:10D0500001440422E96002EB8A010144C5E90101AF
:10D0600001210024BAF1010F1CD04FEACA00083098
:10D0700015F088FA064600EB8A074FEA8A0000B2EC
:10D08000ADF80000C0F101022146ADF80240801069
:10D09000A146A346ADF824204C463F1D01910590C2
:10D0A000B3E0FEE7B4220270E8680480E8684180DB
:10D0B000A86804800BB0BDE8F08F4FF00008BDF900
:10D0C0002400002808DCBDF80210032202EB410115
:10D0D0000844ADF824000DE0BDF80220BDF80010B2
:10D0E0000523521A03EB42021044491EADF82400F6
:10D0F000ADF80010BDF80200401CADF80200684613
:10D1000000F0F0F878B1BDF9000005AB821043F8EB
:10D11000282001AA00F0030142F8281008F10108B4
:10D12000B8F1040FCBDBB8F1040F74D1089905985E
:10D13000884212D126F8140027F81490DDE9010185
:10D140000844DDE903121144084469680855696818
:10D1500000010855641C24B255E00699884219D094
:10D1600026F8140027F814906A68019810556A6828
:10D1700000011055641C059A20B2521E26F810209A
:10D1800027F81090DDE902120A440499091D1144A0
:10D190006A6832E0079926F814008842494627F861
:10D1A000149015D0DDE9012010446A6810556A68B2
:10D1B00000011055641C059A20B2521E26F810205A
:10D1C00027F81010DDE90312114408316A6814E0F1
:10D1D000DDE901021044039A10446A6810556A6838
:10D1E00000011055641C059A20B2521E26F810202A
:10D1F00027F8101004996A680C3111546A68090103
:10D200001154401C04B209F10109684600F06AF8A3
:10D2100000287FF452AF40F2D3211AFB01F106EB54
:10D220004402881232F9022C824205D107EB4402F3
:10D2300032F9022C82421AD0A1EB8021B1F5007F95
:10D2400003DC494341F3CF3106E0C1F58061494336
:10D2500041F3CF31C1F10F0126F8140027F8140073
:10D2600068680155686809010155641C24B2A01E54
:10D270000DE037F8101026F8141036F8101027F8C3
:10D28000141069680A5C0A55641C24B2401E002808
:10D29000EFDAEB6800210846A3F800B01CE0EA686A
:10D2A00022F81100AB6836F8102023F811200BE0AB
:10D2B000D5F808C036F910303CF811209A4200DB4E
:10D2C0001A462CF81120401C37F910208A4201D14F
:10D2D000A042EDDB491C09B2A042E0DB304615F06C
:10D2E0009DF9E7E6B0F90210B0F90000814201DCD7
:10D2F000012070470020704717B581B0022ABDF8A1
:10D30000080036D9BDF80410C0F3C403C1F3C40447
:10D3100023441F2B00D31F2363F3C70143079B0E36
:10D3200003EB503301F0070403EBC40303EB513369
:10D33000ADF804103F2B00D33F23DC0864F3020157
:10D3400063F34F31C0F30420C1F304231844ADF854
:10D3500004101F2800D31F2060F30C21ADF8041027
:10D36000FF2A08D0DDE9010104F022FB0090BDF89E
:10D37000000004B010BD88B2FBE717B581B0022AE7
:10D3800003D8BDF8080004B010BDBDF80410BDF806
:10D390000800C1F3C403C0F3C40413FB04F35B0926
:10D3A00063F3C701C1F30423C0F3042413FB04F3A4
:10D3B0005B0963F30C214B079B0E4407A40E03EBA0
:10D3C000513304EB503013FB00F35B0A63F30201AB
:10D3D0004B079B0E03EB513313FB00F0800960F306
:10D3E0004F31ADF80410FF2A07D0DDE9010104F048
:10D3F000DFFA0090BDF80000C5E788B2C3E717B5B3
:10D4000081B0022ABDF8080036D9BDF80410C0F377
:10D41000C403C1F3C4041B1B002B00DC002363F313
:10D42000C70143079B0E03EB503301F0070403EBE6
:10D43000C40303EB5133ADF80410002B00DC0023D0
:10D44000DC0864F3020163F34F31C0F30420C1F33D
:10D450000423C01AADF80410002800DC002060F39B
:10D460000C21ADF80410FF2A08D0DDE9010104F019
:10D470009FFA0090BDF8000004B010BD88B2FBE731
:10D480002DE9FF4F83B00746DDF84080DDE91356F4
:10D490004FEA4800DDF8489000B2049C0190B9F1D1
:10D4A000040F1CD0B9F1060F19D0B9F1050F56D0F1
:10D4B000B9F1140F50D1B7F90010B7F9022008FBE9
:10D4C000021004EB400A384604F073F983463846EC
:10D4D00004F093F981460024400000907EE0384635
:10D4E00012F074F901460090304615F0E1F9B7F9F1
:10D4F0000010B7F9022008FB021004EB400A38467E
:10D5000004F07BF9834640000290A846B7F9024038
:10D510000AE051464046029A15F0CEF80199641C83
:10D520008A4408EB4B0824B2B7F90600A042F0DAAF
:10D53000B9F1060F10D14EF207000021ADF804003A
:10D540000246084605E035F81030934200D13154C8
:10D55000401C009B9842F6D307B0BDE8F08FB7F9A6
:10D560000010B7F9022008FB021000EB4000044451
:10D57000384604F042F9A8EB000000EB40000FFA37
:10D5800080F8384604F015F98146384604F035F93C
:10D59000002215E000210BE0A378735414F8013B3E
:10D5A00014F8027B03EB072325F81130491C09B25C
:10D5B0008142F1DB521C05EB40050644444412B2A3
:10D5C0004A45E7DBC8E751462846009A15F074F84B
:10D5D0000199641C05EB49058A4424B25C45F2DBE1
:10D5E000DDE904014A000699B7F9023002FB0100A7
:10D5F000B7F9002008FB03210D18002408E04A4673
:10D600002946304615F058F8641C4E44454424B26F
:10D610005C45F4DBA0E72DE9F04F0646C87A89B0F7
:10D6200015460F46022803D8012009B0BDE8F08F47
:10D6300018463A69B9680CF003FF041EF5D0207D46
:10D6400000F01F0007F06EF84FF4807808B1062054
:10D6500010E0207D00F01F000E2806D0142809D00D
:10D6600007F050F840B1052004E038884FF00E096B
:10D6700038B903E0814608E00420FBE7788840459C
:10D6800003D000204FF00509A061226A22B129468B
:10D6900030460CF080F8B7E0A069F0B3294602A844
:10D6A00004F051F8B7F9003013B97888404529D013
:10D6B000A88829886A88401A401C01B2E88807F1C6
:10D6C000040C801A401C02B27888CDE9000C02A834
:10D6D0000CF000FEBDF8080029880844ADF80800E9
:10D6E000BDF80A0069880844ADF80A00BDF80C00CE
:10D6F00029880844ADF80C00BDF80E00698808447C
:10D70000ADF80E0002AA04A8B1680CF022FC0028B3
:10D710007AD004A8D6F8088000E00BE0B060CDF81D
:10D7200000902A4639463046A36904F0F3FBC6F858
:10D73000088069E02A4603A8B1680CF00AFCF0B33F
:10D74000BDF81000BDF80C10401A401C0FFA80FA0A
:10D750000AEB4A0014F016FF059003A901A8D6F8B9
:10D7600008B003F0F0FF012101A812F076F8BDF92E
:10D770000C00B5F90010401A0890BDF90E80B5F9FB
:10D780000200A8EB000536E001AA594606A80CF0F5
:10D79000E0FB70B3059800900898534601B22AB296
:10D7A000204613F035FE01280ED0204613F085FDEB
:10D7B000059814F033FF204613F07FFD00E023E0CE
:10D7C0000020C6F808B030E706A8B060CDF8009099
:10D7D00001AA39463046059B04F09CFBBDF80600C3
:10D7E000401CADF80600BDF80A00401CADF80A0068
:10D7F0006D1C08F10108BDF912004045C4DAC6F8F5
:10D8000008B0059814F00AFF204613F056FD0BE708
:10D810001CB50C4814460078002812D088880A8865
:10D820004B88801A401C82B2C888C01A401C83B240
:10D8300050005843CDE900404C880888214619F033
:10D84000B2FD1CBD843400202DE9F74FC87898B094
:10D850000C4602287ED911460AA803F08FFFB4F9BE
:10D860002000012829DD94F82200FD2825D32088F6
:10D8700018B394F82300BDF828104008C0F38002C4
:10D880001144ADF82810BDF82A10C0F34000084438
:10D89000ADF82A0094F82310BDF82C004908C1F314
:10D8A000C001401AADF82C0094F82310BDF82E00EA
:10D8B000C1F34001401AADF82E0018980AA98268F9
:10D8C0000CA80CF046FB00287ED0E07B10F007058A
:10D8D00019D0E088ADF80000BDF8000061898842E9
:10D8E00000D100250AA805F071F807461C2103A8FD
:10D8F00018F0F6FBA0788DF82500BDF80000ADF813
:10D9000014001FB105E060680090E5E7208800B9C9
:10D91000F5B3E078FD2800D3FF2083460AA803F082
:10D9200078FF81460AA803F04AFF06464846B145FB
:10D9300000DB3046B4F90010B1EB600F00DB4110A2
:10D9400088460CA803F065FF82464FF0FF30169022
:10D95000002000E038E00090B8F1000F00DC77B163
:10D96000504614F00FFE0090002342460AA90EA86C
:10D9700005F096FA00210EA804F038FE1690BDF8C6
:10D980003000ADF80400BDF83400ADF8080000E048
:10D9900011E00098069001A803900890FF208DF8F0
:10D9A000240032464946A01D06F02AFE060018D083
:10D9B000022D0CD015E00AA80390E0788DF8240021
:10D9C00003A9189805F02BFD1BB0BDE8F08FBDF939
:10D9D0003010B06800EB4100BDF92810A0EB410009
:10D9E00004907FB3BDF9324027E027B2ADF806704E
:10D9F000ADF80A7052465946009814F0FBFEBDF986
:10DA0000301053463A46009804F0A2FF8DF81C00EF
:10DA1000012802D102208DF81C00012D08D1BDF98A
:10DA20002A10B068611A00EB41000088ADF81400BC
:10DA300003A9189805F0F3FC641CBDF93600A04258
:10DA4000D3DABCE0FFE7002054E0BDF82A1001EB78
:10DA50000900BDF82E1004B2A1EB090007B2BDF910
:10DA60003200A04203DDBDF93600B84240DB524629
:10DA70005946009814F0BEFEBDF9041053462246E4
:10DA8000009804F065FF8DF81C00012802D10220E7
:10DA90008DF81C00BDF93200A04212DCADF8064042
:10DAA000ADF80A40012D08D1BDF92A10B068611AFD
:10DAB00000EB41000088ADF8140003A9189805F0A8
:10DAC000AEFCBDF93600B84212DBADF80670ADF819
:10DAD0000A70012D08D1BDF92A10B068791A00EB3F
:10DAE00041000088ADF8140003A9189805F097FCD0
:10DAF00009F1010081464045A7DBBDF82800ADF8DB
:10DB00005000BDF82C00BDF82A10ADF8540001EB10
:10DB10000800BDF82E10ADF85200A1EB0800ADF8DA
:10DB2000560014A804F052FF074628430DD0BDF953
:10DB30002E100120A1EB0809BDF92A108DF824B0A0
:10DB40008DF81C0001EB080437E0BDF82A108DF8B1
:10DB500024B001EB0800ADF80600BDF82E10A1EBD3
:10DB60000800ADF80A000020069003A9189805F0F7
:10DB700056FC24E06FB152465946009814F03AFE24
:10DB8000BDF93010534622B2009804F0E1FE8DF842
:10DB90001C00ADF80640ADF80A40012D08D1BDF9D2
:10DBA0002A10B068611A00EB41000088ADF814003B
:10DBB00003A9189805F033FC641C4C45DADD009885
:10DBC00008B114F02BFD1698401C05D0169805F0EE
:10DBD00011FA0EA804F0DEFE002E3FF4F5AE30463A
:10DBE00006F007FDF0E62DE9F0410646086990B021
:10DBF00015460C4600287DD0A07E02287AD92946F9
:10DC00000DA8B2680CF0A5F9002873D00DA8D6F8BD
:10DC10000880B060206906F08DFD022806D001A9B9
:10DC2000206913F06BFB012849D0C9E0002741F6B9
:10DC3000FF70CDE900700297D4E904123B460FA8AB
:10DC400016F0AAFB284603F0E4FD01462A88BDF938
:10DC50003C0001EBD17102EB610100EBD072A1EB52
:10DC600062010844401EADF83000ADF82C10284683
:10DC700003F0A5FD01466A88BDF93E0001EBD171B4
:10DC800002EB610100EBD072A1EB62010844401E7F
:10DC9000ADF83200ADF82E1003A804F0F3FB606974
:10DCA0000390208BADF81800A07E8DF82600009719
:10DCB0000BAA03A93046236904F04EF980E004A8BA
:10DCC00004F030F9A0788DF81C00208BADF8180016
:10DCD000E07E8DF81A00A07E8DF81B00207F4FF0AB
:10DCE000FF3740B101996888ADF80A0007EB515140
:10DCF00008445DE066E0284603F08BFD298800EBD0
:10DD0000D07001EB60000199C1F38A21A0EB5100B2
:10DD1000ADF80800284603F052FD698800EBD0708A
:10DD200001EB60010198A1EB9051C0F38A22ADF89C
:10DD30000A10BDF80830521E1A4407EB5050ADF8D7
:10DD40000C200844ADF80E0002AA04A9304623694D
:10DD500004F0B4F834E001992888C1F38A21ADF8C1
:10DD60000800491E084410E002AA04A930462369AD
:10DD700004F0A4F80198BDF80810C0F38A2001440B
:10DD8000ADF80810BDF80C100844ADF80C00BDF952
:10DD90000800B5F904108842E6DDBDF80A100198C4
:10DDA00001EB5051ADF80A10BDF80E1001EB5050C8
:10DDB000ADF80E00BDF90A00B5F906108842CADDBB
:10DDC000C6F8088010B0BDE8F0812DE9F04180462A
:10DDD00091F8220086B00C461646022868D9208C9D
:10DDE000002865D094F8230010F03E0F60D0C007E3
:10DDF0005ED1104603F00DFD0746304603F0DFFC10
:10DE0000B4F90050874200DA3846B5EB600F00DD08
:10DE10004510314604A803F0B1FC94F82300BDF985
:10DE20001020C0F344014807B4F9200001D428446D
:10DE300040421044ADF810000807BDF91420B4F9B1
:10DE4000200001D428444042101AADF8140094F880
:10DE50002300BDF9121040088007B4F9200001D456
:10DE6000284440420844ADF8120094F82300BDF95C
:10DE700016104008C007B4F9200001D128444042E0
:10DE8000081AADF81600208C281A01B2002900DA11
:10DE90000021A27894F82200CDE90202E08BADF8CF
:10DEA000040000912B4604AA3146404600F003F8D6
:10DEB00006B0BDE8F0812DE9FF4FA3B01F46DDE9B4
:10DEC000326ADDF8C08015460C46FF2E00D3FF26CF
:10DED000084604F07BFD8146384350EA08006DD0C7
:10DEE00023982146826803A80CF033F800286CD0F0
:10DEF00003A803F08EFC02901C2108A814F0ABFCD0
:10DF0000029814F03FFB0B904FF0FF300090002F71
:10DF10000ADD00233A46214616A804F0C1FF00217D
:10DF200016A804F063FB00900123424629461CA872
:10DF300004F0B6FF00211CA804F058FB01900FA8C4
:10DF400008900D90BDF8C4008DF83860ADF8280039
:10DF50008DF839A0B4F90000B5F9001038448842B2
:10DF600000DC0846ADF85000B4F90400B5F904101F
:10DF7000C01B884200DB0846ADF85400B4F902002B
:10DF8000B5F902103844884200DC0846ADF852006A
:10DF9000B4F90600B5F90610C01B884200DB08463C
:10DFA000ADF8560014A803F034FC0146B4F90200A1
:10DFB000B5F9022090420BDC01200AE000962A46C7
:10DFC0002146319B239800F0D0F927B0BDE8F08FAF
:10DFD00000208046B4F90600B5F90620904201DB26
:10DFE000012600E00026B9F1000F44D0BDF80C0076
:10DFF000ADF83C00BDF81000ADF84000BDF90E4092
:10E0000022E0B8F1000F03D1BDF95200A0421ADCA2
:10E010001EB9BDF95600A0421ADB25B2ADF8425038
:10E02000ADF83E5002990B9814F042FCBDF90C106B
:10E030002A46029B0B9804F08BFC8DF8300008A94F
:10E04000239805F0ECF9641CBDF91200A042D8DA5F
:10E050001CA804F09FFC019804F0CCFF0098401C21
:10E0600005D016A804F096FC009804F0C3FF0B98A6
:10E0700014F0D4FAA9E7B4F90000B5F900209042F1
:10E0800001DC012000E000208146B4F90400B5F96C
:10E090000420904201DB012000E00020824609EAD2
:10E0A0000A0202EA08024FF0010B324203D0322981
:10E0B00001DA4FF0000B01208DF8300018EA0B0F49
:10E0C00012D0BDF85000ADF83C00BDF85400ADF8DA
:10E0D00040006088ADF83E00688808A9401EADF891
:10E0E0004200239805F09BF916EA0B0F12D0BDF8F9
:10E0F0005000ADF83C00BDF85400ADF84000E88891
:10E1000008A9401CADF83E00E088ADF84200239815
:10E1100005F085F9B9F1000F12D02088ADF83C0068
:10E12000288808A9401EADF84000BDF85200ADF89F
:10E130003E00BDF85600ADF84200239805F06FF997
:10E14000BAF1000F12D0A88808A9401CADF83C0015
:10E15000A088ADF84000BDF85200ADF83E00BDF813
:10E160005600ADF84200239805F059F9BDF80C00AF
:10E17000BBF1000FADF83C0008D0BDF95000BDF96F
:10E180001010421E914248DA084647E0BDF81000E0
:10E19000ADF84000B5F90200B4F90210401AB842D7
:10E1A00000DB07460FFA87F8002533E06088284433
:10E1B00006B2E088401B07B2BDF90E00B04203DD95
:10E1C000BDF91200B84224DB02990B9814F070FBE1
:10E1D000BDF93C103246029B0B9804F0B9FB8DF858
:10E1E0003000BDF90E00B04207DCADF83E60ADF87E
:10E1F000426008A9239805F012F9BDF91200B8424F
:10E2000007DBADF83E70ADF8427008A9239805F021
:10E2100006F96D1C4545C9DBA0E0401EADF8400085
:10E220000FA803F0F6FA051E41DD59EA08001DD0DB
:10E23000BDF90E4016E027B2ADF84270ADF83E7061
:10E2400029460B9814F034FBBDF93C102B463A4696
:10E250000B9804F07DFB8DF8300008A9239805F099
:10E26000DEF8641CBDF95200A042E4DC59EA060065
:10E270001DD0BDF9564015E027B2ADF84270ADF89B
:10E280003E7029460B9814F013FBBDF93C102B4649
:10E290003A460B9804F05CFB8DF8300008A92398EF
:10E2A00005F0BDF8BDF91200641CA042E4DABDF926
:10E2B0005400BDF90C10421C914201DD084600E0FB
:10E2C000401CADF83C00BDF81000ADF840000FA8B0
:10E2D00003F09FFA051E41DD5AEA08001DD0BDF982
:10E2E0000E4016E027B2ADF84270ADF83E702946F8
:10E2F0000B9814F0DDFABDF93C102B463A460B980A
:10E3000004F026FB8DF8300008A9239805F087F863
:10E31000641CBDF95200A042E4DC5AEA06001DD09C
:10E32000BDF9564015E026B2ADF84260ADF83E604A
:10E3300029460B9814F0BCFABDF93C102B46324626
:10E340000B9804F005FB8DF8300008A9239805F020
:10E3500066F8BDF91200641CA042E4DA1CA804F0BF
:10E3600019FB019804F046FE7BE62DE9FF478AB0D1
:10E370000C46824615461C216846169E14F06BFA20
:10E3800007A80090BDF83400ADF808008DF81860BB
:10E39000B4F90200B5F90210884201DC012700E05F
:10E3A0000027B4F90600B5F90610884201DB012602
:10E3B00000E00026B4F90000B5F90010884201DC45
:10E3C000012100E000218846B4F90410B5F90420C9
:10E3D000914201DB012100E00021ADF81C00A08882
:10E3E000ADF820006088ADF81E0068888946401EA0
:10E3F000ADF822001FB16946504605F010F8E888D4
:10E40000401CADF81E00E088ADF822001EB1694640
:10E41000504605F004F82088ADF81C002888401EFE
:10E42000ADF8200017B1B5F9020001E0B4F902001F
:10E43000ADF81E0016B1B5F9060001E0B4F906000A
:10E44000ADF82200B8F1000F03D06946504604F041
:10E45000E6FFA888401CADF81C00A088ADF820009D
:10E46000B9F1000F03D06946504604F0D8FF0EB052
:10E47000BDE8F0872DE9F0412F4F0646786811F08E
:10E4800037FD04463068C56B696B09B1284688477B
:10E49000786800680188408811FB00F0E1688842D4
:10E4A00001D1012000E00020216859B1616849B123
:10E4B00028B107E078680068816A01B1884720695F
:10E4C0000028F7D10121216178680068C06882695D
:10E4D000D20704D08069800701D5616101E0002086
:10E4E0006061606908B1012700E000273068416978
:10E4F00071B1016911F0300F06D0490704D5D5E993
:10E50000001000F01BF803E0D5E90021FEF76EFDD6
:10E51000206800280BD06168002908D03268127C7E
:10E52000BA43D20703D1A268824202D1A160BDE8FA
:10E53000F081A060FBE70000C03400202DE9F34F1C
:10E540000446854887B041680D682869820701D56F
:10E5500042076FD4C0F30110022829D0012801D04E
:10E56000032867D100200090084611F0C1FC8346C3
:10E57000204603F030F90646204603F00EF94FF42A
:10E58000A051B1FBF6F20190824201DAB1FBF6F044
:10E590000390B4F902000290287CC0F30110012816
:10E5A00013D020886080711E0844E0800027C4E0FA
:10E5B00021462846089A00F0DBF8089A09B021465F
:10E5C0002846BDE8F04FFEF711BD68882188401A43
:10E5D000401EE080801B401C6080E7E70399C01B61
:10E5E000884200DD08460FFA80F90120CBF81000C0
:10E5F0000FBB0198B0421EDB287CB146C0F301106E
:10E60000032810D000204946089A00F0E5F8287C3D
:10E61000C0F30110012808D029880298081A401E6A
:10E62000A080801B54E00120EDE702982080029832
:10E63000304463E08DE0009820B94FF4205013F08F
:10E64000A1FF0090287CC0F3011003281AD00020FD
:10E650008646DDF820C000984946069016FB01F07A
:10E66000401E0590701E4843049000208246884258
:10E6700021DA0498BEF1000F504401D0059A101A17
:10E68000002212E00120E3E7069BBEF1000F03EB3E
:10E69000400863460CF1020C1B88A8F8003001D03A
:10E6A000084400E0401A521C12B2B242ECDB0AF1FC
:10E6B000010000B2DAE7287CC0F30110012819D06C
:10E6C00029880298081AC01B401EA080A0EB0900F0
:10E6D000401C208001984F44874212DBDBF8180071
:10E6E000C0070ED0DBF8180080070AD50120CBF850
:10E6F000140009E00298384420804844401EA0805D
:10E70000E8E70021CBF81410009828B10246214612
:10E710002846FEF76BFC05E0089AF8E7A96A09B1FC
:10E7200028468847DBF810000028F7D1089906FB37
:10E7300009F001EB40003FB2089001988742FFF6D4
:10E740004DAF0098002804D009B0BDE8F04F13F099
:10E7500065BF09B0BDE8F08FC034002030B5048833
:10E760000D88058010880880188810801C8030BDB6
:10E77000F8B5054616460C46084603F02CF8074641
:10E78000204603F00AF817FB00F300200CE006EB2C
:10E79000430706EB40013A88ADF80020B1F800C00D
:10E7A000A7F800C00A80401C5B1E8342EFD869882E
:10E7B0006288E088891A491EE1806988081A401E2B
:10E7C000608029882288A088891A491EA18029880A
:10E7D000081A401E2080F8BD2DE9F0470C46164669
:10E7E0008246002701EBD47931E00025601C00EB64
:10E7F000D07827E0E01B401E01B2601B401E00B233
:10E80000BAF1000F0AD015FB041206EB420311FB0C
:10E81000040106EB410210FB047009E010FB0472D6
:10E8200006EB420311FB040006EB400215FB04104B
:10E8300006EB400117FB045006EB4000FFF78EFF8C
:10E840006D1C2DB2B5EB680FD4DB7F1C3FB2B7EB6C
:10E85000690FCADBBDE8F0872DE9FF4F95B0987BC3
:10E860008A7E00F00F04DDF888800D46032C00D16D
:10E870000424012C19D0022C1FD0042C25D0082CE4
:10E880007DD1DFF890924FF0FF0A6101FD2A35D269
:10E89000DFF884C29CF80000904203D1DCF8040049
:10E8A000A04225D000209D4F20E0DFF868924FF075
:10E8B000800AA9F116090221E8E7DFF858924FF023
:10E8C000C00AA9F114090421E0E7DFF848924FF0EB
:10E8D000F00AA9F110091021D8E719F80060FF2EFD
:10E8E0001CD016FB02F6360A3E54401C8842F4D374
:10E8F000DFF828928CF80020CCF804401798DE88C6
:10E900000996B0F900101598B3F808B0664380680E
:10E91000B0F90020914203DB002202E01646E3E753
:10E92000521A0A92099A8B18B0F90420934201DC1A
:10E93000099901E0511A491C0B911799B0F902206D
:10E94000B1F90210914201DB002200E0521A0E924E
:10E95000B0F9060001EB0B02824201DC584601E0EF
:10E96000401A401C0F900E980A99704301FB040056
:10E9700008EBD00700F007061C21684600E0C5E060
:10E9800013F069FFA889ADF80800A87E8DF818007B
:10E99000A87FC0F3C2008DF81900FDF749FF11F000
:10E9A000ABFA099901FB0BF1814200DC084610909B
:10E9B00013F0E8FD834603901798002501880A9814
:10E9C00001441798ADF81C1002880B98401E0244B1
:10E9D000ADF82020179843880E981844531A5B1CF2
:10E9E000ADF81E001BB21193ADF83010ADF8220047
:10E9F0000F99ADF83200ADF834200844ADF8360078
:10EA00000CA803F0E3FF139007A800900590C4F151
:10EA100008001290DDE9091001440B98081A6043C0
:10EA200014900E985BE02B462AFA06F04FF0000C8B
:10EA30000A991AE03A78DDF848800240A8EB060807
:10EA400032FA08F204D019F802800BF8058001E0D0
:10EA50000BF805C0129A964202D22644E04002E02A
:10EA6000002650467F1C491C6D1C0B9A9142E1DB2D
:10EA7000139880B10BEB0300BDF92220BDF91C10E7
:10EA80008046119B03F064FF8DF8100018B94046D2
:10EA9000119913F0E0FEDDE90A10401A41191098AF
:10EAA000814205D2BDF82200401CADF822000EE0E4
:10EAB00002208DF810006946159804F0B0FCBDF8EE
:10EAC0002200401CADF81E00ADF82200002514986D
:10EAD000304407EBD00700F007060998401C0F9957
:10EAE000099088429FDBBDF91E10BDF922008142CA
:10EAF00009D0401EADF8220002208DF810006946B2
:10EB0000159804F08CFC584613F088FD19B0BDE848
:10EB1000F08F00009A9C0108D43400209C7B0020D8
:10EB20002DE9F04F8346B1F902000C46401E41101A
:10EB300000F001004618B2F90000B3F9005089B0A6
:10EB4000A84200DB2846ADF80000B2F90000B3F996
:10EB50000030984200DC1846401EADF80400508892
:10EB6000801BADF8020050880844ADF806006946E5
:10EB70000846DBF808200BF0ECF9002822D0E088EA
:10EB800018B1A08808B1012000E0002080460126CD
:10EB9000684603F01BFF10B9B8F1000F00D0002643
:10EBA0001C2102A813F057FECDF808D02088ADF83C
:10EBB0001000207A6D468DF8200036B102A9584623
:10EBC00004F02DFC09B0BDE8F08FBDF80410BDF9CC
:10EBD0000000BDF906A0091A491C0EB2BDF80210CA
:10EBE000ADF806104FF00009B8F1000F08D0B4F9E5
:10EBF0000610B4F90420114490FBF1F201FB120954
:10EC0000304613F0BFFC079505900746BDF902504A
:10EC10003EE03146384613F04BFEBDF90010334656
:10EC20002AB2384603F094FE8DF81800B8F1000FB0
:10EC30001FD0F0B1002148460B4615E0B4F904207E
:10EC4000824205DB121A1144104409B200B207E0F7
:10EC5000B4F906C06244824201DC002000E07B542B
:10EC6000491C401C09B200B2B142E7DB02208DF81A
:10EC7000180002A9584604F0D2FBBDF80200401C5F
:10EC8000ADF80200BDF80600401CADF806006D1C92
:10EC90005545BEDD384613F0C1FC93E72DE9FF4F23
:10ECA000B2F90250B3F90240BBB0A54208DA1288AB
:10ECB00065F31F4062F30F0064F31F411A8807E0F9
:10ECC0001B8864F31F40128865F31F4163F30F0034
:10ECD00062F30F010FFA81F906B20714A9EB0604DB
:10ECE0004FEA214AAAEB07053791002C01DD2046A7
:10ECF00000E06042002D01DD294600E069428842C3
:10ED000001DD012000E0002000903C98B0F90210E5
:10ED1000009858B1002D01DD284600E0684242010C
:10ED2000002C01DD20460CE060420AE0002C01DDF1
:10ED3000204600E060424201002D01DD284600E04F
:10ED4000684292FBF0F0AB4A105C10FB01F03F30E0
:10ED5000C0114FEA600800F0010202EB080B4946BF
:10ED60004E4500DA3146A1EB0001ADF8601001DD3F
:10ED7000314600E049460144ADF86410514657451C
:10ED800000DA3946A1EB0001ADF8621001DD394629
:10ED900000E051460844ADF866003B9818A9826827
:10EDA00008460BF0D6F800287ED0009800210028F5
:10EDB0007BD0002C16DDAAEB080000B2CDE90001E3
:10EDC000A7EB080002B24B46314602A803F09CFEB6
:10EDD0000AEB0B00012100B2CDE900014B4607EB25
:10EDE0000B0015E00AEB0B0000B2CDE9000107EBC8
:10EDF0000B0002B24B46314602A803F085FEAAEB97
:10EE00000800012100B2CDE900014B46A7EB080044
:10EE100002B231460DA803F077FE002102A803F0EC
:10EE2000E5FB399000210DA803F0E0FB38904FF08E
:10EE3000FF30804600903C98407AC00623D43819B1
:10EE4000032100B2CDE90001701B03B23A463146FE
:10EE500021A803F059FE379902200A14111909B2AA
:10EE6000CDE90010379801B2481B03B22CA803F07B
:10EE70004BFE002121A803F0B9FB009000212CA833
:10EE800003F0B4FB8046BDF86400BDF86010401A82
:10EE9000401C06B2FDF7CCFC11F02EF8044618A871
:10EEA00010F094FCA04201E0A1E028E003D218A8F1
:10EEB00010F08CFC0446A146204613F063FB82460A
:10EEC000BDF966B0BDF86200ADF8660000244946A1
:10EED000504613F0EDFC1C211AA813F0BCFC3C9822
:10EEE00018A91A910088ADF870003C98007ACDF806
:10EEF00074A08DF880001F91BDF9625044E009EBC9
:10EF00000B00CDE900A103B206EB0B0001B23A46BB
:10EF100002A803F0F9FD0121A9EB0800CDE900A149
:10EF200003B2A6EB080001B23A4673E70AEB040706
:10EF3000BDF9601033462AB2384603F009FD8DF85A
:10EF4000780018B93846314613F085FC3444A119CD
:10EF5000494505D2BDF86600401CADF8660012E0D8
:10EF600002208DF878001AA93B9804F058FABDF8F1
:10EF700066000024401CADF86200ADF8660049460A
:10EF8000504613F095FC6D1C5D45CFDDBDF9621058
:10EF9000BDF96600814209D0401EADF8660002202E
:10EFA0008DF878001AA93B9804F039FA504613F00E
:10EFB00035FB02A803F0EEFC0DA803F0EBFC009873
:10EFC000401C02D021A803F0E5FCB8F1FF3F02D0BD
:10EFD0002CA803F0DFFC399804F00CF8389804F002
:10EFE00009F8009804F006F8404604F003F83FB032
:10EFF000BDE8F08F9A9D01082DE9F04F8346B1F9E5
:10F0000002000C46401E411000F00100158889B036
:10F010000844281AADF8000010880844ADF8040030
:10F02000B2F90200B3F90210884200DB0846ADF8DD
:10F030000200B2F90200B3F90210884200DC08466F
:10F04000401EADF8060069460846DBF808200AF0C5
:10F0500080FF00281FD0E08818B1A08808B10127E0
:10F0600000E000270125684603F0B0FC00B907B1B5
:10F0700000251C2102A813F0EEFBCDF808D0208853
:10F08000ADF81000207A6E468DF8200035B102A947
:10F09000584604F0C4F909B0BDE8F08FBDF804008B
:10F0A000BDF80010BDF90690401A401C0FFA80F818
:10F0B000BDF80200ADF80600404613F063FA824640
:10F0C00000250796059057B1B4F90600B4F904106D
:10F0D0000844BDF9021091FBF0F200FB1215BDF9D6
:10F0E00002602EE04146504613F0E2FBBDF90010ED
:10F0F000434632B2504603F02BFC8DF818008FB116
:10F1000070B1B4F90400A84202DA00208DF81800AA
:10F11000B4F90600B4F904100844A84200DC002544
:10F120006D1C2DB202A9584604F079F9BDF8020011
:10F13000401CADF80200BDF80600401CADF806000A
:10F14000761C4E45CEDD504613F068FAA3E770B545
:10F15000054691F82A0088B00C46022858D9E18C5F
:10F16000002955D0114604A802F008FB218DBDF8F6
:10F170001000491E401AADF81000BDF81200401AE8
:10F18000ADF81200BDF814000844ADF81400BDF845
:10F1900016000844ADF8160004A906A802F0EEFA1D
:10F1A000BDF81810E08C091AADF81810BDF81C1045
:10F1B0000844ADF81C00BDF81A00E18C401AADF807
:10F1C0001A00BDF81E00E18C0844ADF81E0004A82A
:10F1D00002F01FFB064604A802F0F1FAB4F9001091
:10F1E000864200DA3046B1EB600F00DD4110E08C62
:10F1F000A278084403B294F82A00CDE90202A08C58
:10F20000ADF80400009104AA06A92846FEF753FEB3
:10F2100008B070BD7CB50446806961896D4686681A
:10F22000A08961B1002865D0814203D12289E38899
:10F230009A427CD302297BD003297AD0AFE010BB5D
:10F24000E088218988421ED2B4F9060014F0D8FF64
:10F25000B4F90410B4F90E20891A4843216849888A
:10F2600001EBE030ADF80200E0885A3000B214F053
:10F27000C7FFA18810FB01F02168098801EBE0308D
:10F28000ADF8040040E020680088ADF80000206878
:10F29000A18840880844ADF80600B4F9060014F0CF
:10F2A000AFFFB4F90410B4F90E20891A484321685D
:10F2B000498801EBE030ADF80200E0885A3000B236
:10F2C00014F09EFFA18810FB01F0216832460988E6
:10F2D00001EBE030ADF80400694608460AF039FE5B
:10F2E00030B1A0698560D4E90520216903F092FE60
:10F2F000A08970BB2068A18800880844ADF804008C
:10F3000020684088ADF80200B4F9080014F078FFD6
:10F31000A18810FB01F02168498801EBE030ADF8CD
:10F32000060020895A3000B214F06AFF02E015E0AE
:10F3300012E00FE0B4F90410B4F90E20891A484322
:10F3400021683246098801EBE030ADF800006946DB
:10F350001AE024E0022801D0012820D1206832469A
:10F360000088ADF8000020684088ADF802002068F1
:10F37000A18800880844ADF804002068A18840886E
:10F380000844ADF80600294608460AF0E2FD30B10F
:10F39000A0698560D4E90520216903F03BFEA069DE
:10F3A00086607CBD7CB50446806961896D4686684F
:10F3B000A08901290CD0012867D0814203D122897C
:10F3C000E3889A427ED300297DD003297CD0B5E022
:10F3D000012822D1E088218988421ED2B4F9060092
:10F3E00014F00EFFA18810FB01F02168498801EBA1
:10F3F000E030ADF80600E0885A3000B214F000FFAB
:10F40000B4F90410B4F90E20891A48432168098818
:10F4100001EBE030ADF8040042E02068A1880088EC
:10F42000401AADF8000020684088ADF80200B4F939
:10F43000060014F0E5FEA18810FB01F02168498860
:10F4400001EBE030ADF80600E0885A3000B214F06D
:10F45000D7FEB4F90410B4F90E20891A4843216884
:10F460003246098801EBE030ADF8040069460846F1
:10F470000AF06FFD30B1A0698560D4E905202169EB
:10F4800003F0C8FDA089012858D120680088401EDB
:10F49000ADF804002068A18840880844ADF8060053
:10F4A000B4F9080014F0ACFEB4F90410B4F90E205D
:10F4B000891A48432168498801EBE030ADF8020021
:10F4C000208902E018E010E014E05A3000B214F095
:10F4D00097FEA18810FB01F021683246098801EBF4
:10F4E000E030ADF8000069461DE0022804D0032892
:10F4F00002D023E0022821D12068A188324600886A
:10F50000401AADF8000020684088ADF8020020687D
:10F510000088401EADF804002068A1884088084497
:10F52000ADF80600294608460AF013FD30B1A0697F
:10F530008560D4E90520216903F06CFDA06986602F
:10F540007CBD7CB50446806961896D468668A0896A
:10F5500002290CD002287ED0814203D12289E3887F
:10F560009A4279D3002978D0012977D0D4E00228B3
:10F570003FD1E088218988423BD25A3000B214F052
:10F580003FFEA18810FB01F02168098801EBE03003
:10F59000ADF80000B4F9060014F032FEB4F904101E
:10F5A000B4F90E20891A48432168498801EBE030FC
:10F5B000ADF80600B4F9080014F022FEA18810FB93
:10F5C00001F02168498801EBE030ADF802002089A4
:10F5D0005A3000B214F014FEB4F90410B4F90E203D
:10F5E000891A48432168098801EBE030ADF804002E
:10F5F00066E020680088401EADF804002068A188FD
:10F600004088401AADF80200E0885A3000B214F089
:10F61000F7FDA18810FB01F02168098801EBE030BB
:10F62000ADF80000B4F9060014F0EAFDB4F90410D6
:10F63000B4F90E20891A484321683246498801EB03
:10F64000E030ADF80600694608460AF082FC58B181
:10F65000A069856003E00AE03BE034E036E0D4E9ED
:10F660000520216903F0D6FCA089022854D1206826
:10F67000A1880088401AADF8000020684088401E2C
:10F68000ADF8060020895A3000B214F0B9FDB4F983
:10F690000410B4F90E20891A48432168098801EB47
:10F6A000E030ADF80400B4F9080014F0A9FDA18819
:10F6B00010FB01F02168498801EBE030ADF8020051
:10F6C000324669461DE0032803D025E0032800D018
:10F6D00010BB2068A18832460088401AADF80000AF
:10F6E0002068A1884088401AADF8020020682946A9
:10F6F0000088401EADF8040020684088401EADF828
:10F70000060008460AF025FC30B1A0698560D4E9FE
:10F710000520216903F07EFCA06986607CBD7CB574
:10F720000446806961896D468668A08903290ED0E8
:10F73000032867D0814203D12289E3889A427ED38D
:10F7400002297DD001297CD002297BD0B1E0032899
:10F750001FD1E088218988421BD25A3000B214F0B0
:10F760004FFDB4F90410B4F90E20891A48432168FA
:10F77000098801EBE030ADF80000B4F9060014F0A0
:10F780003FFDA18810FB01F02168498801EBE030C2
:10F7900040E02068A18800880844ADF80400206893
:10F7A0004088401EADF80600E0885A3000B214F0E0
:10F7B00027FDB4F90410B4F90E20891A48432168D2
:10F7C000098801EBE030ADF80000B4F9060014F050
:10F7D00017FDA18810FB01F021683246498801EB32
:10F7E000E030ADF80200694608460AF0B2FB30B1DD
:10F7F000A0698560D4E90520216903F00BFCA0898C
:10F80000032856D120680088ADF800002068A18840
:10F810004088401AADF8020020895A3000B214F036
:10F82000EFFCA18810FB01F02168098801EBE030B2
:10F83000ADF80400B4F9080014F0E2FC03E016E0AF
:10F8400010E013E00FE0B4F90410B4F90E20891AA7
:10F85000484321683246498801EBE030ADF80600A4
:10F8600069461BE018B1012801D022E008BB2068DE
:10F8700032460088ADF800002068A1884088401A10
:10F88000ADF802002068A18800880844ADF80400A3
:10F89000206829464088401EADF8060008460AF058
:10F8A00058FB30B1A0698560D4E90520216903F0D7
:10F8B000B1FBA06986607CBD70B5A4B00C4605465E
:10F8C00022AA20A906F053F820A80FF07FFF20B944
:10F8D00022A80FF07BFF00283ED012A9284609F08D
:10F8E00081FD012838D12146684605F04DFC1B48B2
:10F8F00001900220029012A804904FF480300D90E5
:10F9000020A80FF063FF80B120A803906A461A2157
:10F91000284610F0CBFB20AA12A9204603F07AFB60
:10F920006A461B21284610F0C1FB22A80FF04EFFAB
:10F93000002811D022AE6A461A212846039610F0FC
:10F94000B5FB22AA12A92046039603F063FB6A4680
:10F950001B21284610F0AAFB24B070BD609C010852
:10F960002DE9F74FB1F92E00A2B014460D4600283C
:10F9700072D095F8361002296ED9012808D1B5F950
:10F980003400002804DC288E10B9688E0028EFD0DF
:10F990002088298EAA8E0844801AADF82000A388FA
:10F9A00019441144ADF8241062886B8E1A44AB8E52
:10F9B000D21AADF82220E3886E8E3344AE8E3344E3
:10F9C000ADF82630B5F92E6006EBD676A0EB6600D2
:10F9D000401EADF82800012000EB66063144ADF86A
:10F9E0002C10B5F92E1001EBD171A2EB6101491E6B
:10F9F000ADF82A10B5F92E1001EBD17100EB6100C2
:10FA00001844ADF82E0095F836000D90FD2801D968
:10FA1000FF200D9022980AA9826820A80AF099FA7E
:10FA20000028A5D0214603A801F0A8FE4FF0FF371B
:10FA300039463A4603A80FF0EFFEB5F9009003A847
:10FA400001F0E7FE044603A801F0B9FE844203A8D2
:10FA500003DA01F0DEFE02E0FEE301F0B0FEB9EBF6
:10FA6000600F01DD4FEA6009B5F9006008A801F0F8
:10FA7000D0FE044608A801F0A2FE844208A802DADB
:10FA800001F0C7FE01E001F09AFEB6EB600F00DD69
:10FA90004610B5F92E00841904FB04F0400012F062
:10FAA00071FD00900146B5F92E20334608A809F0F3
:10FAB000B1FD0AA802F08AFF012620B9E878FF28E4
:10FAC00001D3A87800B100261F9756B901234A46F2
:10FAD00003A912A803F0E4F9002112A802F086FDA0
:10FAE0001F900AA801F095FE12F04CFD83461C21E0
:10FAF00018A812F0B0FE01A81890CDF86CB01D90B7
:10FB0000A88DADF8680095F836008DF87800A878D3
:10FB10008DF879000AA801F07CFEBDF8281000EBF2
:10FB2000D07001EB60000FFA80FA0AA801F047FEDE
:10FB3000BDF82A1000EBD07001EB600007B2BDF8F1
:10FB40002C00ADF80800001B401C00B2621EADF88E
:10FB50000400ADF8061011440C9209B2ADF80A1079
:10FB60005246504500DC1046ADF80400B94200DBB7
:10FB700039462298ADF80A1001A9826805A80AF052
:10FB8000E8F9C0B34A4603A905A80AF00AFA90BBEF
:10FB900005A801F03EFEBDF91610BDF92A200E9011
:10FBA000891A0098BDF92C2001FB0400BDF914103E
:10FBB000121B891A0844401E119046B14A4603A9F7
:10FBC00005A80AF05EFA10B10120079000E0079640
:10FBD0000E98002827DDBDF81400ADF80400CDF81C
:10FBE0006CB0BDF81800ADF8080002208DF8700068
:10FBF000BDF9168013E016E0ADF80A800798ADF85D
:10FC00000680E8B311981B9018A9229803F007FC0E
:10FC100011982044119008F101000FFA80F8BDF905
:10FC20001A104145E8DABDF82C00ADF80800001BB9
:10FC3000401C00B2ADF80400BDF82E20ADF80A203B
:10FC4000111B491C09B2ADF806105246504500DCA4
:10FC50001046ADF80400781C0F90814200DC791C3E
:10FC60002298ADF8061001A9826805A80AF071F97A
:10FC7000D0B34A4603A905A80AF093F9A8B15FE0FA
:10FC8000FFE722465846119912F016FDBDF91410EF
:10FC9000424658460E9B02F05BFE8DF8700001282C
:10FCA000B2D102208DF87000AEE705A801F0B1FDD9
:10FCB000BDF90A10BDF91A200E90891A0098BDF9F5
:10FCC0002C2001FB0400BDF91410121B891A0844F2
:10FCD000401E11904EB14A4603A905A80AF0D1F979
:10FCE00018B10120079001E02AE007960E9800283D
:10FCF00026DDBDF81400ADF80400CDF86CB0BDF8F9
:10FD00001800ADF8080002208DF87000BDF91A80C7
:10FD100012E0ADF80A800798ADF80680B0B31198EC
:10FD20001B9018A9229803F07AFB11982044119097
:10FD3000A8F101000FFA80F8BDF916104145E8DD81
:10FD4000BDF828002044ADF80400BDF82C00001BCD
:10FD5000ADF80800BDF82A000C99ADF8060008447B
:10FD600000B2ADF80A00B84200DB3846ADF80A0030
:10FD7000229801A9826805A80AF0EBF890B34A46D8
:10FD800003A905A80AF00DF9A8B178E0FFE722461B
:10FD90005846119912F090FCBDF91410424658468D
:10FDA0000E9B02F0D5FD8DF870000128B9D102201C
:10FDB0008DF87000B5E705A801F02BFD0E90BDF998
:10FDC0001610BDF906200098891A01FB0400119055
:10FDD0004EB14A4603A905A80AF053F918B101200B
:10FDE000079001E04BE007960E98002847DD079842
:10FDF00060B100201B90BDF81400ADF80400BDF800
:10FE00001800ADF80800BDF9160033E0CDF86CB06D
:10FE1000F1E7ADF80A800798ADF8068060B10D985B
:10FE2000FF281198007804D095F8361010FB01F0E7
:10FE3000000A8DF8780013E011980E9A0178584660
:10FE400012F0D8FCBDF91410424658460E9B02F041
:10FE50007FFD8DF87000012802D102208DF870001E
:10FE600018A9229803F0DBFA11982044119008F1A8
:10FE7000010000B2BDF91A1080464145C9DA95F873
:10FE800036008DF87800BDF828002044ADF8040055
:10FE9000BDF82C00BDF82E10001BADF80800081BA3
:10FEA000401CADF80A1000B20F99ADF80600884268
:10FEB00000DC781CADF80600229801A9826805A82C
:10FEC0000AF047F8F0B34A4603A905A80AF069F812
:10FED000C0BB05A801F09DFC0790BDF90A10BDF953
:10FEE0001A200098891A01FB040011900798002835
:10FEF00055DD2EB14A4603A905A80AF0C2F800B99B
:10FF000066B100201B90BDF81400ADF80400BDF8E8
:10FF10001800ADF80800BDF91A003BE0CDF86CB050
:10FF2000F1E7ADF80680ADF80A802EB14A4603A984
:10FF300005A80AF0A6F800B976B10D98FF28119827
:10FF4000007800E02BE004D095F8361010FB01F0AB
:10FF5000000A8DF8780013E01198079A0178584646
:10FF600012F048FCBDF9141042465846079B02F0B7
:10FF7000EFFC8DF87000012802D102208DF870008E
:10FF800018A9229803F04BFA119820441190A8F177
:10FF9000010000B2BDF9161080464145C1DD95F85B
:10FFA00036008DF87800BDF82C00ADF80800011B74
:10FFB000BDF82A00491C09B22044ADF8041000B273
:10FFC000ADF80600BDF82E200F9B121B12B2ADF843
:10FFD0000A20984200DB781CADF80600BA4200DC2B
:10FFE0003A46ADF80A205046514500DC01462298B9
:10FFF000ADF8041001A9826805A809F0AAFFC8B3EA
:020000040801F1
:100000004A464D4603A905A809F0CBFF90BB05A8B9
:1000100001F0FFFB10900C990098BDF92C2001FB1A
:100020000400BDF91410121B891A0844401E1190D7
:1000300046B12A4603A905A80AF023F810B14FF0EB
:10004000010802E0B6F1000801D0119800E058461E
:100050001B901098002832DDBDF81400ADF80400A4
:10006000BDF81800ADF8080002208DF87000BDF949
:10007000165020E023E0ADF80650ADF80A50B8F174
:10008000000F12D1DDE91021584612F015FBBDF921
:1000900014102A465846109B02F05AFC8DF8700046
:1000A000012802D102208DF8700018A9229803F0CF
:1000B000B6F96D1C2DB2BDF91A00A842DBDA002397
:1000C000009815E000EB040EAEF10101002204EBF4
:1000D000D47C07E0057891F8008000F8018B01F8E6
:1000E0000159521CB2EB6C0FF4DB5B1C70461BB267
:1000F000A342E7DBBDF828000C99ADF804000844E2
:1001000001B2BDF82A000F9B204400B2ADF80600F2
:10011000BDF82E20ADF80810121B12B2ADF80A205F
:10012000984200DB781CADF80600BA4200DC3A4683
:10013000AAF10100ADF80A201090814200DB0146CF
:100140002298ADF8081001A9826805A809F001FFFE
:10015000B8B34A464D4603A905A809F022FF80BB63
:1001600005A801F056FB0E900C990098BDF90420EB
:1001700001FB0400BDF91410891A0844119046B11E
:100180002A4603A905A809F07CFF10B14FF0010829
:1001900002E0B6F1000801D0119800E058461B902B
:1001A0000E98002832DDBDF81400ADF80400BDF84B
:1001B0001800ADF8080002208DF87000BDF9165047
:1001C00020E023E0ADF80650ADF80A50B8F1000F7A
:1001D00012D158460E9A119912F06EFABDF9141008
:1001E0002A4658460E9B02F0B3FB8DF8700001289A
:1001F00002D102208DF8700018A9229803F00FF99F
:100200006D1C2DB2BDF91A00A842DBDABDF828003A
:100210000C99ADF80400084400B2ADF80800BDF830
:100220002A100C9AADF806101144109A09B2ADF8D4
:100230000A10904201DBAAF10100ADF80800B942B2
:1002400000DB39462298ADF80A1001A9826805A89A
:1002500009F07FFEC8B300E044E14A464D4603A9D9
:1002600005A809F09EFE80BB05A801F0D2FABDF9F1
:100270001620BDF906100D90511A0098BDF9042002
:1002800001FB0400BDF91410891A01EB000846B106
:100290002A4603A905A809F0F4FE10B10120079031
:1002A00000E007960D98CDF86CB0002821DDBDF870
:1002B0001400ADF80400BDF81800ADF808000220E5
:1002C0008DF87000BDF916500FE012E0ADF80A503D
:1002D0000798ADF80650D0B3CDF86C8018A92298D5
:1002E00003F09DF86D1CA0442DB2BDF91A00A84280
:1002F000ECDABDF82800ADF804000C99BDF82E200A
:10030000084401B2101BADF80810401CADF80A20DB
:1003100000B20F9AADF80600904200DC781CADF8F0
:1003200006001098814201DBAAF101012298ADF884
:10033000081001A9826805A809F00BFEC0B34A465F
:100340004D4603A905A809F02CFEA8B158E0FFE727
:1003500022464146584612F0AFF9BDF914102A461C
:1003600058460D9B02F0F4FA8DF870000128B5D1C3
:1003700002208DF87000B1E705A801F04AFABDF936
:100380000A10BDF91A208246891A0098BDF9042086
:1003900001FB0400BDF91410891A0F184EB12A464A
:1003A00003A905A809F06DFE18B14FF0010801E09E
:1003B00026E0B046CDF86CB0BAF1000F20DDBDF8F4
:1003C0001400ADF80400BDF81800ADF808000220D4
:1003D0008DF87000BDF91A500EE0ADF80650ADF87A
:1003E0000A50B8F1000F2FD01B9718A9229803F0DC
:1003F00016F86D1E27442DB2BDF91600A842ECDD9B
:10040000BDF8280001A92044ADF80400BDF82C0077
:10041000001BADF80800BDF82A002044ADF8060026
:10042000BDF82E00001BADF80A002298CDF86CB084
:10043000826805A809F08DFDF0B34A4603A905A816
:1004400009F0AFFDA0B140E022463946584612F00F
:1004500033F9BDF9141053462A46584602F078FA8B
:100460008DF870000128C0D102208DF87000BCE723
:1004700005A801F0CEF9051E27DDBDF81400ADF882
:100480000400BDF81800ADF80800BDF9164018E0EA
:10049000ADF80640ADF80A402946584612F008FA71
:1004A000BDF914102B462246584602F051FA8DF839
:1004B000700018A9229800E007E002F0B0FF641C69
:1004C00024B2BDF91A00A042E2DA2EB912A802F055
:1004D00061FA1F9802F08EFD009812F09FF85846BE
:1004E00012F09CF825B0BDE8F08F00002DE9FF4F19
:1004F00083B00446DDE910870E460846139D01F0DF
:1005000076F98346304601F04EF90190012D0FD067
:10051000022D0FD0032D3ED1404E6FB12088ADF893
:10052000000038784FF0000AFD2837D3424638E003
:100530003B4EF2E73B4EF0E72088ADF80800ADF8FF
:100540000000424602990698B047002702901FE03B
:10055000002517E0BDF8000034F8151088420BD0D4
:1005600004EB450042460088ADF80800ADF80000F5
:1005700002990698B047029004EB4500BDF80810B8
:1005800001806D1C5D45E5DB05987F1C04EB400494
:1005900001988742DCDB07B0BDE8F08F00FB08F074
:1005A000020A00990698B0470290002030E000252A
:1005B00025E0785D10B3504505D1BDF8001034F842
:1005C0001520914215D0FD2801D3424602E000FBE0
:1005D00008F0020A04EB45000088ADF80800029913
:1005E0000698B047029017F805A034F81500ADF84A
:1005F000000004EB4500BDF8081001806D1C5D454E
:10060000D7DB059804EB40041298074409F1010078
:10061000019981468842CADBBDE700007BD3000810
:10062000F9D20008FFD300082DE9FF4F85B004463A
:10063000DDE9127593460E46084601F0D8F880466B
:10064000304601F0B0F882466DB1BDF82000FD2FB4
:1006500000EB00497DD3A8F1040001900020009038
:10066000BDF820703AE1FD2F0ED3002507E0424689
:10067000204608990FF033FA04EB4B046D1C5545E6
:10068000F5DB09B0BDE8F08FBDF80010002060F385
:10069000020189B260F3C70189B260F30C2189B20B
:1006A00060F34F31ADF8001088B20090BDF8000043
:1006B000009001463A46089801F07AF93F1D0190F2
:1006C0000899F808C00689B2000EC1F3C40212FBF3
:1006D00000F2ADF808204A07920E02EB513212FBED
:1006E00000F2ADF80A20C1F3042111FB00F1ADF8CE
:1006F0000C10C0F1FF02002556E000204FE0BDF8CD
:10070000001034F81030994243D004EB40010988BE
:10071000ADF80410ADF80010BDF80430BDF80810B5
:10072000C3F3C40616FB021101EBC11606EBC1317F
:10073000BDF81060C1F3C45161F3C7065907890EB3
:10074000BDF80A7001EB533111FB027101EBC117C7
:1007500000E0C9E007EBC137BF0E67F3020601EB0B
:10076000C11707EBC131C1F3C25161F34F36BDF878
:100770000C10C3F3042313FB021101EBC11303EBB1
:10078000C131C1F3C45161F30C26B1B2ADF81060B0
:10079000019104EB4001BDF804300B80401C404542
:1007A000ADDB04EB4B046D1C5545A6DB69E7002669
:1007B00010E02A78FF2A12D02088ADF808000299AC
:1007C000089801F0F5F80290BDF808002080A41CFC
:1007D0006D1C761C464557DAA807EAD154E02780FD
:1007E000F5E72868411C43D0F0B32A78FF2A4FD0A0
:1007F0002088ADF808000299089801F0D9F8029015
:10080000BDF80800208015F8012FA41CFF2A41D054
:100810002088ADF808000299089801F0C9F8029004
:10082000BDF80800208015F8012FA41CFF2A33D042
:100830002088ADF808000299089801F0B9F80290F4
:10084000BDF80800208015F8012FA41CFF2A25D030
:100850002088ADF808000299089801F0A9F80290E4
:10086000BDF80800208000E00BE0A41C6D1C0AE02D
:10087000A00704D02780C4F80290E78001E0C4E913
:10088000009908342D1D361D01988642A9DD18E017
:100890002780B8E72780C6E72780D4E72780E2E7EC
:1008A0002A78FF2A1ED02088ADF8080002990898FF
:1008B00001F07EF80290BDF808002080A41C6D1C99
:1008C000761C4645ECDBABEB080004EB40041498C7
:1008D000A0EB080005440098401C00905045FFF62E
:1008E00066AFCEE62780E9E700212388ADF8043023
:1008F0008946084633E0002627E0287818B3884266
:1009000005D0FF282FD000FB07F2120A914688423B
:1009100003D134F81600834210D0B9F1FF0F24D070
:1009200004EB46004A460088ADF804000199089897
:1009300001F03EF80190297834F8163004EB4600B7
:10094000BDF8042002806D1C761C4645D5DB14984A
:1009500004EB4B04A0EB080005440098401C0090F9
:100960005045C8DB8DE63A46D0E70898E2E72DE926
:10097000FF4F85B00D46DDE912A7FBF759FFBDF823
:10098000209080464FB1284600F031FF0390284662
:1009900000F009FF8346002640E0B5F9026017E049
:1009A000B5F900400FFA86FB0DE0CDF808A0ADF8D0
:1009B0000490CDF800B0D8F8000023B2079AC769B8
:1009C0000599B847641CB5F90400A042EDDA761C1D
:1009D000B5F90600B042E3DA09B0BDE8F08F0024B3
:1009E00016E0385D98B100FB0AF0000A0290ADF8FD
:1009F00004906888079A304400B2009028880599CE
:100A0000204403B2D8F80000D0F81CC0E047641CB2
:100A100003988442E5DB1498761C07445E45DEDBD0
:100A2000DAE700680968884201D101207047002098
:100A3000704740680A6820F04040904200D2086049
:100A40000020704770B50D46C06A20F078F9044662
:100A5000284611F0F5FD0CB10C2070BD002070BDD2
:100A600070B50D46C06A1EF0B4FA0446284611F06F
:100A7000E7FD0CB10C2070BD002070BD70B5C56ADB
:100A80000E46342011F050FD040009D001463246D4
:100A900028461FF06DFA0028204602D011F0D0FD44
:100AA000002070BD2DE9F043C3B00025D0F82C80A4
:100AB000144689468DF808502F2602AF6A464946EB
:100AC00040461FF0A1FC00280CDD9DF80000022824
:100AD00004D03946204615F064FB05E026703946FF
:100AE000601CF8E710D1257008A1204615F03EFBE8
:100AF0000028E3D006A1204615F038FB0028DDD001
:100B0000002043B0BDE8F0830C20FAE72F2E000050
:100B10002F2E2E002DE9F041C56A0E46022A17D06D
:100B2000012A17D0032A17D00024542011F0FCFC0E
:100B3000071E0BD0014623463246284620F0BEFA57
:100B40000028384602D011F07BFD0020BDE8F0817E
:100B50000124EAE70224E8E70324E6E710B5C06AC7
:100B6000029C20F0EEFB002801DA0C2010BD206072
:100B7000002010BD10B5C06A23B1012B02D0022B9A
:100B800000D0002320F094FC002801DA0C2010BDD6
:100B9000002010BD10B51446C06A20F05BFD00288F
:100BA00001DA0C2010BD2060002010BD2DE9F041BD
:100BB000C56A0F46069E284620F056FD040005D45F
:100BC0003946284620F0D7FC002802DA0C20BDE880
:100BD000F08100203460FAE7B0F90C00032101EB4A
:100BE000400020F00300103070472DE9F041054629
:100BF00000206B8C0E460427C3F30514EA680EE050
:100C000007EBC00151585FEAC11C07D521F07F41B5
:100C1000B14203D152F83000BDE8F081401C84425B
:100C2000EED84FF0806000EBB3204FEAB0506884FC
:100C3000C0F30510C100104611F026FDE860C0B3F6
:100C4000688CC0F30514641E16D06FF003025300C5
:100C5000E86802EBC40141585FEAC11C0CD4890169
:100C60000AD400EBC40103EBC40C6044641ED0E959
:100C700000C0C1E900C0EBD1E868082100EBC40066
:100C800011F0E9FD082011F04FFCE96841F834004B
:100C900012F0BEFDEA6807EBC400115841F0807104
:100CA0001150EA6866F317011150E86850F83400F3
:100CB000B2E7FFE7FEE700002DE9FC410068C068ED
:100CC000C068B0FBF1F5954200DD1546134F78681A
:100CD0000068806900B30020ADF80000ADF80400A2
:100CE000ADF802002CB2601E06B2ADF8066078685E
:100CF0006946006882699047684600F04EFDA84248
:100D000002DD341EEFDC01E0002C02DC0020BDE837
:100D1000FC81BDF906506D1C2846F8E7C034002060
:100D20002DE9FF4F83B0064698468B46059809F09B
:100D3000A2FE01218140B6F820A001F0FF096FEA70
:100D40000A0080B2019096F822004FF0FF37C0F3FE
:100D5000C00500241CE0F16801EBC4004268920168
:100D60003BD5A5B9042202EBC402895801F47F01E6
:100D700059450CD10068817911EA090F07D06A46FC
:100D8000059912F0F3FC01282ED0022830D0641C03
:100D9000708CC0F30510A042DDD81EE0F06850F85A
:100DA0003430997911EA090F16D0042101EBC401FE
:100DB000405800F47F0185B259450DD10198054294
:100DC0000AD1BD4208DD18466A46059912F0CEFCEC
:100DD000012810D002280BD0641C708CC0F30510C1
:100DE000A042DBD8002F0FDB00990120C8F80010CB
:100DF00007B0BDE8F08F5545F6D0AF42ECDA009968
:100E00002F46C8F80010E7E70020F1E72DE9F0478A
:100E1000814642F30006C0F15A001D460F465408B1
:100E200000B2761C13F0ECF9A7EB040800FB08F005
:100E3000C711484613F0E4F900FB08F0C011002F79
:100E400006DD7F3F39120A1B32442A80214405E027
:100E50007F3739120A1B21442A80891BA980002868
:100E600006DD7F380012011B31446980204405E013
:100E70007F300012011B20446980801BE880BDE8A0
:100E8000F0872DE9F04104460020678C0D460426CA
:100E9000C7F30513E2680AE006EBC00151585FEAA8
:100EA000811C03D521F07F41A94202D0401C83421E
:100EB000F2D8834203D002EBC000BDE8F0814FF0CE
:100EC000806000EBB7204FEAB0506084C0F305109B
:100ED000C100104611F0D8FBE060608CC0F3051033
:100EE000401E0DD06FF00703E16803EBC00601EB75
:100EF000C0023144401ED1E90061C2E90061F3D172
:100F00000821E06811F0A7FC082011F00DFBE16852
:100F1000086012F07DFCE168486840F000704860AD
:100F2000E16865F317004860E068C6E70146002005
:100F3000A1F13002092A01D8D0B27047612901D34A
:100F40002039C9B241390629F7D2DFE801F003059B
:100F500007090B0D0A2070470B2070470C207047C3
:100F60000D2070470E2070470F2070472DE9F0418B
:100F7000064615460F46002005E039462046B04794
:100F800001280AD0204607F0DDFB040002D060688B
:100F90008000F2D10020BDE8F08105B12C60012075
:100FA000F9E7000010B50C461CF0D4FF0D4998B1CC
:100FB0000122A27306280DD2DFE800F00C0305071A
:100FC000090B0B2006E0092004E00A2002E01120B2
:100FD00000E01220086002E00020A0730868606052
:100FE00010BD0000883400202DE9F041044640681F
:100FF000096820F04040884227D12046FFF7ECFDE9
:10100000DFF84C800546D8F80800021BA0EB05006D
:10101000561BC8F8080015D02746611932463846D5
:1010200011F04AFB06E0A068401BA0602046FFF7D5
:10103000D3FD0444D8F808008442F4D1B8192946F5
:1010400011F009FC0120BDE8F0810020FBE7000061
:10105000C83400202DE9FC41064614468846D807CE
:1010600029D004F108000125002206F114010746E9
:1010700008F097FF58B100208DF800006A46122151
:10108000304601970FF012F89DF8000098B1608982
:10109000218A0844401EE081B4F90E10B4F906001C
:1010A000814200DDE08102B02A4621464046BDE88B
:1010B000F04101F00DBA0025EEE72DE9F0410746B9
:1010C00088B01C46164688460846FBF7CAF905460E
:1010D00002A9404604F0A0FA2A46114602A80EF0E2
:1010E0009BFB022E05D0012E22D0002008B0BDE8C7
:1010F000F081DDE90201CDE9040100231A4604A9CB
:10110000404605F0EBF804AA06A8B96808F021FFEC
:101110000028EBD0DDE90601CDE900010123002222
:101120006946404605F0DAF8694602AA084602E038
:1011300002AA6846B96808F00CFF0028D6D00098CB
:101140002060019860600120D0E7000070B505467E
:1011500004F0D8F90646002406E0A868006850F8B4
:101160002400FFF7F3FF641CB442F6D3688CC10778
:101170001AD020F001006884284605F011FF2846A7
:1011800005F02AFE86B10021284604F096FF58B1EA
:101190000C494968884207D80B49096801EBC0002F
:1011A00050E9022128469047688C810708D520F035
:1011B000020068842846BDE87040002105F052BD59
:1011C00070BD0000B43400205C3500202DE9F047EC
:1011D0008046089D1F46E86900FB01F39B1200282A
:1011E00006DD934206DD95F8280080070DD489E0DE
:1011F0009342F8DBCB1943439B12002808DD93424E
:1012000037DA95F8280080077CD40120BDE8F08704
:101210009342F6DCA869521C504340F39500021239
:10122000C0B2FF23002826D06E6AC0F1FF0404FB81
:1012300006F4A3EB2426A2EB0104A14636D0002C31
:1012400015DBBC4213DAC0F1FF00C6F1FF014843D1
:10125000A3EB6020C1B295F82800800701D5C1F149
:10126000FF0118F8040007F05EFA08F80400641C97
:101270001CE0A869D0E74FF0FF06DCE7002C10DB8C
:10128000BC420EDAA6EB6000C1B295F828008007D8
:1012900001D5C1F1FF0118F8040007F044FA08F87D
:1012A0000400686A641C361ABC4202DA686AB042FA
:1012B000E4DBBC4218DA002C16DBA869704380120C
:1012C0007043C0F34721E869002801DAC1F1FF014A
:1012D00095F82800800701D5C1F1FF0118F8040036
:1012E00007F021FA08F8040095F82800800707D5D0
:1012F0004946B94506DC00290DDB404609E001E01E
:10130000641C01D5002081E7BC4204DC391B08EBDA
:10131000040011F0A0FA022078E72DE9F05F8A4678
:101320000A9F06461D46B96901FB02F4A012002976
:1013300000DD401C97F82830504502DA980707D4A2
:10134000D2E0A0120AEB050C844502DA98077ED49D
:1013500080E044F39500521C4A4342F395044FEA5F
:101360002029221204F0FF08C0B2A9EB0A0491451B
:1013700005D0002903DA10B9FF209146641E91457B
:1013800026D1002C0BDBAC4209DA40444108980717
:1013900001D5C1F1FF01305D07F0C5F9305597F86F
:1013A0002800641C800706D5A9EB0A01A9424EDA81
:1013B0008CE0304609E0AC4200DD2C46002C46D0E3
:1013C00005DDA5EB040106EB040011F044FA88E00A
:1013D0004FF0FF0B002943DAF969494241434FEAD4
:1013E000A128002C0DDBAC420BDA08FB00F1C1F3A5
:1013F0004721980701D5C1F1FF01305D07F093F94E
:101400003055B969A8F1FF0041438812641E11D418
:10141000AC420FDAC8F1FF014143ABEB6120C1B22E
:1014200097F82800800701D5C1F1FF01305D07F072
:101430007AF9305597F82800A41C800708D5A9EB45
:101440000A01491EA9424CDC0029B2DC49E04BE00C
:10145000AC4202DD0120BDE8F09F002CB1DA40E093
:10146000F969C0F1FF0041434FEAA128002C0EDBCF
:10147000AC420CDA00FB08F0ABEB6020C1B298077D
:1014800001D5C1F1FF01305D07F04DF93055B96963
:10149000C8F1FF0041438912641C0ED4AC420CDA3F
:1014A0004843C0F3472197F82800800701D5C1F1D0
:1014B000FF01305D07F037F9305597F82800641CBC
:1014C000800707D5A9EB0A01A9420DDC0029BFF668
:1014D00070AF06E0AC4200DD2C46002C04D03FF794
:1014E00070AF4FF00200B6E74FF00000B3E7000026
:1014F0002DE9F04107460E464FF00008134809F069
:10150000EBF904461CE02146104809F0F7F90546BE
:101510002068B84200D097B96068B04200D076B970
:1015200021460A4809F073FA216909B12046884723
:10153000204611F085F8FBF7FFF94FF001082C4623
:10154000002CE0D14046BDE8F0810000207D002065
:1015500070B505460C46094809F0BEF90BE0016874
:10156000A94204D14168A14207D0002C05D0014610
:10157000024809F0C3F90028F1D170BD207D002098
:1015800010B50446442111F066F94FF4FA70E06298
:10159000002020626420A0620120A4F840000448DA
:1015A000E06194F8420040F0010084F8420010BD70
:1015B0001F16010838B504464FF480650095D4E93C
:1015C0000B200023194610F090FF4FF46E73322267
:1015D000002100950EF094F90146A26A206A121AC1
:1015E0004A4300EBA22038BD38B504464FF480656D
:1015F0000095D4E90B200023194610F076FF40F245
:10160000B6334FF46172002100950EF079F901466E
:10161000A26A206A121A4A4300EBA22038BD38B5EC
:1016200004464FF480600090D4E90B200023194653
:1016300010F05BFF0146A26A206A121A4A4300EBCF
:10164000A22038BD38B504464FF480650095D4E932
:101650000B200023194610F048FF40F214534FF4BA
:101660007A72002100950EF04BF90146A26A206AB9
:10167000121A4A4300EBA22038BD8B1A002B00DC63
:10168000531A4FF47A714B43B3FBF0F0002800D1AA
:101690000120704770B54168054611B12868FFF711
:1016A00027FF194809F0AAF9184E10B112F08AFC68
:1016B0007060154809F035F9040024D04422294609
:1016C00010F0FAFF2868A84200D12460717894F8DD
:1016D000420061F3820084F84200C0070FD06169C4
:1016E00039B120468847216A01442162A16A084431
:1016F000A06262681AB1206808B1216A9047FBF7BE
:101700001BF9204670BDFEE7207D002044350020F7
:101710000A8802804A8842808A888280C988C1807B
:1017200070470A8802804A8842808A888280C988F5
:10173000C18070470A8802804A8842808A888280F5
:10174000C988C18070470A8802804A8842808A8896
:101750008280C988C18070470A8802804A88428096
:101760008A888280C988C18070470A8802804A8836
:1017700042808A888280C988C18070470A88028036
:101780004A8842808A888280C988C1807047C1881F
:101790004088081A401C00B27047C1884088081A67
:1017A000401C00B27047C1884088081A401C00B233
:1017B0007047C1884088081A401C00B27047C18831
:1017C0004088081A401C00B2704781880088081AB7
:1017D000401C00B2704781880088081A401C00B283
:1017E000704781880088081A401C00B270478188C1
:1017F0000088081A401C00B2704781880088081AC7
:10180000401C00B2704781880088081A401C00B252
:10181000704781880088081A401C00B27047F0B5F4
:1018200004464FF4FA66C1F341307710642501286D
:101830000BD121F4C040B04207DCB84201DDC0F555
:101840007A70584390FBF5F001B2C2F341300128A1
:101850000BD122F4C040B04207DCB84201DDC0F534
:101860007A70584390FBF5F002B2944201DA2046B8
:1018700000E01046884201DA0846F0BD944201DAE1
:101880002046F0BD1046F0BDF0B504464FF4FA66B0
:10189000C1F341307710642501280BD121F4C040F9
:1018A000B04207DCB84201DDC0F57A70584390FBC6
:1018B000F5F001B2C2F3413001280BD122F4C0404F
:1018C000B04207DCB84201DDC0F57A70584390FBA6
:1018D000F5F002B2944201DA204600E01046884258
:1018E00001DA0846F0BD944201DA2046F0BD104608
:1018F000F0BD002208B51146104600F027F8009010
:10190000BDF8000008BD002208B51146104600F0E1
:1019100036F80090BDF8000008BD18B54C09BDF8B8
:101920000030D20864F30203ADF80030C308BDF8FC
:101930000000890863F3C70080B262F30C2080B214
:1019400061F34F30ADF8000080B218BD18B54C09F6
:10195000BDF80030D20864F30203ADF80030C308CC
:10196000BDF80000890863F3C70080B262F30C2061
:1019700080B261F34F30ADF8000080B218BD18B5E9
:101980004C09BDF80030D20864F30203ADF8003012
:10199000C308BDF80000890863F3C70080B262F392
:1019A0000C2080B261F34F30ADF8000080B218BD5A
:1019B00018B580B2030243EA102083B288B2010254
:1019C00041EA1020121D0C4980B2D40840EA0040C0
:1019D00043EA034208400A40121A624300EB5210E5
:1019E000084040EA104080B2010241EA1020ADF800
:1019F000000080B218BD00001FF8E00718B580B2E3
:101A0000030243EA102083B288B2010241EA1020A7
:101A1000121D0C4980B2D40840EA004043EA034258
:101A200008400A40121A624300EB5210084040EA94
:101A3000104080B2010241EA1020ADF8000080B2EF
:101A400018BD00001FF8E00781B2C1F3C402C2EB69
:101A5000C20000EB0220C01D4209184662F3174085
:101A60004A07920E02EB513202EB420303EB0222D1
:101A7000D21C920962F30F20C1F30421C1EBC10211
:101A800002EB0121C91D490961F30700FF2161F340
:101A90001F607047FF2208B511461046FFF76FFF21
:101AA0000090BDF8000008BD7CB50E7BDDE9065452
:101AB000022E08D94E88002E05D0A54203D0CDE9CC
:101AC00000544469A0477CBD38B50446102110F08D
:101AD000C2FE01206080FF202073BDF800100020AE
:101AE00060F3020189B260F3C70189B260F30C218F
:101AF00089B260F34F31ADF8001088B20090BDF8A4
:101B000000000090BDF80000208038BD2DE9F04FA6
:101B100085B0824610B294468B460FFA82F9AAEB42
:101B2000000EDDF838800FFA8EF2049203F5B471DE
:101B3000ABEB00021E4613B203920AEB0002119CAB
:101B40005844029212B207B2019088457DD04FF4FA
:101B5000B4718E4202D9A6F5B476B6B2884503D9DF
:101B6000A8F5B4701FFA80F80F99ACEB010000B231
:101B70000090109818B101EBD1704010401C05B2D4
:101B80005A21B6FBF1F0B8FBF1F1C0B2C9B204289A
:101B900000D10320042900D1032188427ED146458B
:101BA0007CD868B3012854D0022878D003287ED18D
:101BB00006F15A0000B212F023FB009910FB01F16C
:101BC0000AEBE130401B208030B212F019FB10FB11
:101BD00009F10BEBE130401B608008F15A0000B2C4
:101BE00012F00EFB10FB09F10AEBE1302844A08053
:101BF0000FFA88F012F004FB009910FB01F15AE192
:101C000030B212F0FDFA009910FB01F10BEBE1305C
:101C1000401B60805A3630B212F0F2FA10FB09F124
:101C20000AEBE1302844A0800FFA88F012F0E8FABD
:101C300010FB09F10BEBE1302844E08008F15A0079
:101C400000B212F0DDFA009900E0E6E010FB01F1CD
:101C500029E030B212F0D4FA10FB09F10BEBE130BD
:101C60002844E0805A3630B212F0CAFA009910FBCC
:101C700001F10AEBE1302844A0800FFA88F012F05D
:101C8000BFFA009910FB01F10BEBE130401B6080C3
:101C900008F15A0000B212F0B3FA02E036E009E0AF
:101CA00005E010FB09F10AEBE130401B208005B094
:101CB000BDE8F08F06F15A0000B212F0A1FA10FB55
:101CC00009F10AEBE130401B208030B212F098FAA3
:101CD000009910FB01F10BEBE1302844E0800FFA92
:101CE00088F012F08DFA10FB09F10BEBE130401B8C
:101CF000608008F15A0000B212F082FA009910FBDD
:101D000001F10AEBE1302844A080D0E730B101288E
:101D100037D0022861D003287ED099E001297CD1F8
:101D200008F15A0000B212F06BFA10FB09F10AEB4D
:101D3000E130401B20800FFA88F0029012F060FA28
:101D4000074630B2804612F05BFA874201DA029809
:101D500000E0404612F054FA009910FB01F10BEB41
:101D6000E130401B60805A3630B212F049FA10FB65
:101D700009F10AEBE1302844A08001982844E08072
:101D800095E7022964D1AEEB050020800FFA88F0B8
:101D900012F036FA10FB09F10BEBE130401B6080CA
:101DA00006F15A0000B2019012F02AFA074608F133
:101DB0005A0000B2804612F023FA874201DD0198F2
:101DC00000E0404612F01CFA009910FB01F10AEB0A
:101DD000E1302844A08030B269E0032938D106F10F
:101DE0005A0000B212F00CFA10FB09F10AEBE130D4
:101DF000401B20800398401B608008F15A0000B20D
:101E000012F0FEF910FB09F10AEBE1302844A08042
:101E10000FFA88F0804601E019E019E012F0F0F9BD
:101E2000009910FB01F730B2064612F0E9F900996B
:101E300010FB01F0874201DD404600E0304612F021
:101E4000DFF9009910FB01F00BEBE03096E729B1C8
:101E5000049820806380A280E78028E708F15A0078
:101E600000B2039012F0CCF9074606F15A0000B216
:101E7000019012F0C5F9874201DA039800E0019859
:101E800012F0BEF9009910FB01F10AEBE130401BA2
:101E9000208030B212F0B4F910FB09F10BEBE13005
:101EA000401B608002982844A0800FFA88F012F04E
:101EB000A7F910FB09F10BEBE1305FE72DE9F041E9
:101EC0001D0017460E4604461AD0F07A02281AD989
:101ED000D4F81CC0BCF1000F03D02046E047012815
:101EE00011D02B463A4631462046FBF794FB012899
:101EF00009D006A239462046BDE8F04107F04BBCA8
:101F000002A23946F8E7BDE8F08100004E6F0A648E
:101F10006174610038B58469049D002C01D000957E
:101F2000A04738BD38B50446182110F094FC0022B3
:101F300011461046FFF7F1FC0090BDF8000000903C
:101F4000BDF800002081FF20E072401C608001206D
:101F5000207538BD704700002DE9FF4FADB0887E79
:101F60003A9E98460C4602287ED9206800287BD0ED
:101F70002D98006A002877D0202216A814F089F83E
:101F800020681590B8F1000F6ED098F80000002876
:101F90006AD02D982F9982682BA807F0DAFF0028C5
:101FA00062D0207FB0F1000A01D14FF0010A607FBA
:101FB000810703D42F98FFF714FC0FE0B4F9121037
:101FC000009141F6FF72CDE90120B4F91430414689
:101FD0001FA8226812F0E0F9BDF97C001599B4F948
:101FE00012200025B1F908906F1E02EB09011F9124
:101FF0002F990988ADF80C102F994A88ADF80E205A
:10200000B4F916102891B4F918100A44ADF80E204E
:10201000EEB1E1B92F99B1F90210002917DAB368CE
:102020005A1A002A00DCCA1A1F994FF480634942E9
:1020300003EB41018A4200DD37603168002906DB8D
:102040000D46BDF80E10B2881144ADF80E10627F37
:102050000021CDE90012B4F9142008EB050703466E
:1020600025903846159900E09FE008F043FD471998
:102070002BE0617F0020CDE90001B4F9142008EBCA
:102080000700259B159908F035FD3D464719BDF819
:102090000E101F98084400B2ADF80E008EB110F576
:1020A000806F0EDB306800280BDA35602F98BDF9A1
:1020B0000E10B0F90200081A70602F98B0F90200F3
:1020C000B06018F8050000286FD02D98BDF90E10EB
:1020D00080684944B0F902008142CADB5046CDF81D
:1020E00088A0BAF1020F02D0032816D029E0607F41
:1020F0000090B4F91430791B08EB0500159A12F022
:10210000ACF906462F98FFF76CFB801BBDF80C104E
:1021100000EBD07001EB600011E0607F0090B4F93B
:102120001430791B08EB0500159A12F096F9064653
:102130002F98FFF756FBBDF80C10801B0844ADF834
:102140000C00D4E901A9CA4502D95046CA468146C5
:10215000A07F800717D012A800F025FAA089ADF85B
:102160004800159890F90E0000B90120ADF84A001A
:10217000A07E8DF85000A07FC1089DF8510061F34A
:1021800001008DF8510000202090FFF7B2FB239052
:10219000FFF7AFFB029004A800F050FF208AADF8D3
:1021A0001400BDF90C00279062E166E1BDF80C1047
:1021B000289800260844ADF80C0008EB050026908E
:1021C000781B1E962990B6E0AAF57F424FF0000BCF
:1021D000FF3A09D0A9F57F42FF3A05D0A84A29184D
:1021E00040461268904783461EAB2AAA21A926982A
:1021F00008F068FC607FC00710D02198232802D027
:10220000012E12D00AE026B1012E06D0022E0AD0ED
:1022100004E01E98012620908DE00026E0680290E0
:10222000022E45D046E0002685E020283FD11E99A9
:102230002098081A072801D0A08936E0209A26980D
:1022400069461044062210F8013B01F8013B521E7A
:10225000F9D100208DF806009DF80100FEF766FE1A
:1022600006469DF80000FEF761FE06EB0010239085
:102270009DF80300FEF75AFE06469DF80200FEF7A1
:1022800055FE06EB001B9DF80500FEF74FFE0646C7
:102290009DF80400FEF74AFE06EB0010C2B2239838
:1022A0000BF0FF01C0B2FFF751FB0226239042E082
:1022B000239802902A9A219915980EF00CF82490F0
:1022C0004FF6FF70824521D081451FD0D3451DD3E5
:1022D000CB451BD2BDF80C00ADF80000BDF80E10C8
:1022E000ADF80210A28A02442498401E1044ADF8B2
:1022F00004001F986A46401E0844ADF8060004A971
:102300002D9800F087FEE089ADF80800BDF80800C0
:10231000ADF8640003AA16A9219B2D9800F031F9AD
:102320002498002807DDBDF80C00A18A01442498F8
:102330000844ADF80C0029991E9881423FF644AF3D
:10234000A07F800723D52798ADF800002068BDF94D
:102350004A1001ABB0F9080001EBD17100EBD0706D
:10236000401000EB6100BDF80E106A460844BDF84D
:102370000C10ADF80410ADF80200ADF80600BDF881
:102380000800ADF8480012A92D9800F0FFF8A07FD2
:10239000C0071FD02798ADF800002068BDF80E10C8
:1023A00001AB028940891144091A15986A4690F9CF
:1023B0000D00081ABDF80C10ADF80410ADF80200BD
:1023C000ADF80600BDF80800ADF8480012A92D9838
:1023D00000F0DCF8617F0020CDE9000108EB070682
:1023E000B4F914203046259B159908F083FB3D462F
:1023F00047192F980088ADF80C002298022802D0C7
:10240000032815D027E0607F0090B4F91430791BC1
:102410003046159A12F021F806462F98FFF7E1F999
:10242000801BBDF80C1000EBD07001EB600010E0D9
:10243000607F0090B4F91430791B3046159A12F081
:102440000CF806462F98FFF7CCF9BDF80C10801B4E
:102450000844ADF80C00BDF80E101F9808442D99E3
:1024600000B2ADF80E008968B1F90610884204DCAC
:1024700018F8050000287FF499AE31B0BDE8F08F60
:10248000B035002038B50446202110F0E4F9FF20D3
:10249000A076FFF72EFA0090BDF80000A0810B484F
:1024A00020604FF6FF706060A060FFF722FA009096
:1024B000BDF80000E081052010F0ECFB0090BDF8B5
:1024C000000020820020E07638BD000034DC0408E3
:1024D000036C002B00D018477047436C002B00D0D2
:1024E000184770472DE9F0410546C06B17460E4668
:1024F000002826D0E86C10F017F804001CD0E96C16
:1025000010F0A9F9FAF794F9296821626968E16184
:10251000A968A16100683A462146007CC0F380109A
:1025200084F824003068206070686060EB6B284697
:102530009847050001D003E0FEE7204610F080F840
:102540002846BDE8F08170B50C46054601F07DFFD8
:10255000206A2860E0696860A069A860FAF768F9F5
:10256000006894F82420016962F386110161AA6C65
:1025700012B12146284690472046BDE8704010F031
:102580005FB830B4046AA44630BC604730B44C88AD
:10259000002C06D00C7A022C03D9446AA44630BC25
:1025A000604730BC704738B504460A2110F053F933
:1025B00001206080FF202072BDF80010002060F331
:1025C000020189B260F3C70189B260F30C2189B2BC
:1025D00060F34F31ADF8001088B20090BDF80000F4
:1025E0000090BDF80000208038BD000010B5044602
:1025F0000A4A002052F8303023B1401CC0B21028E3
:10260000F8D301E0102802D34FF0FF3010BD42F89C
:10261000304002EBC002516010BD0000AC7E0020D3
:102620002DE9FF4F81B08B460E9C15461E46B4F92E
:102630000A10B4F90C00571AB4F9082004F1100A72
:10264000ABEB020204F13C09B4286DDAB4F90E30A8
:10265000B42B7DDA00287BD0002BFCD0984277DDAC
:10266000A94276DC616D79434FEAA12CA16A7F1CF7
:1026700079438912A0F20F14582C01D8002909DBE4
:10268000441E592C01D8002904DB5B38B32802D240
:10269000002900DD0021A3F20F10582801D80029DD
:1026A00009DB581E592801D8002904DB5B3BB32BFA
:1026B00002D2002900DD0021ACEB010001EB60003B
:1026C0000124871AB74200DD3746002F0DDD3BB2EB
:1026D0002A465946CDF800A0019800F09FF9040061
:1026E00003D13946019810F0B6F8B74200DD3746FD
:1026F000002F00DA00270BEB070001B2F61B019850
:1027000033B20744CDF800902A46384600F086F9E7
:10271000050003D13146384610F09DF8AC4277D120
:10272000204605B0BDE8F08F68DDB4F90E30B42B5B
:1027300064DD984262DDA9420BDB616DA46A7943D6
:102740007F1C7C438912A412A0F20F17582F01E0BE
:1027500054E0A5E001D8002C09DB471E592F01D811
:10276000002C04DB5B38B32802D2002C00DD0024EF
:10277000A3F20F10582801D8002C09DB581E592845
:1027800001D8002C04DB5B3BB32B02D2002C00DD14
:102790000024081B04EB60000127841AB44200DD0A
:1027A0003446002C0DDD23B22A465946CDF8009060
:1027B000019800F033F9070003D12146019810F089
:1027C0004AF8B44200DD3446002C00DA00240BEB5A
:1027D000040001B2361B019833B20444CDF800A0C6
:1027E0002A46204600F01AF9050003D1314620465A
:1027F00010F031F8AF4251D1384692E74FF001085E
:102800004746B42805D040B10ADAA94203DC09E002
:1028100044E0A9420FDC03200CE0A942FBDC0AE003
:10282000A942F8DD33462A465946CDF800A0019862
:1028300000F0F4F88046B4F90E00B42806D050B188
:10284000B4F90A000CDAA8420CDC0DE0B4F90A0075
:10285000A84207DC11E0B4F90A00A8420DDC01E04F
:10286000A84201DC032708E033462A465946CDF842
:102870000090019800F0D2F80746B8F1000F09D097
:1028800047B1B8F1030F03D0B8F1010F04D005E050
:10289000032F03D1002044E7012F01D0022040E79D
:1028A00001203EE72DE9F8430546884640F26710CF
:1028B000411C089C1746002B01DA002302E08B42E2
:1028C00000DB0346002C01DA002402E08C4200DB2E
:1028D00004469C4203DAC3F5B470204403E0E01AD6
:1028E000002800DC181BA5F86800AB81EC81A5F876
:1028F00008806F8115482860012028718B4200D91B
:10290000FEE7B42B01D2002000E00120002C01DB07
:102910008B4200DDFEE7B42C05D3A4F1B401B42949
:1029200001D2002600E0012600903A46414605F11A
:10293000100000F0C6F823463A46414605F13C0037
:10294000009600F0BEF8BDE8F883000021260108DB
:102950002DE9F8431E4617468846814600250C4C53
:102960000DE00090D0F800C033463A464146484654
:10297000E047002808D0022800D10125083420684B
:102980000028EED115B10220BDE8F8830120FBE755
:10299000AC7E002010B50179022906D0052913D19B
:1029A0008068BDE810400FF04BBE04464069002827
:1029B0000AD00169002904DA40680FF041FE60691D
:1029C000EFE74169491E416110BD000070B5124D2D
:1029D000060007D0002455F83410B9B10879022850
:1029E00005D002E02868002800D0012070BD887C56
:1029F000B1F91020C007304601F1080102D007F0FC
:102A000040FB01E007F0CDFA0028EED0641CE4B2F0
:102A1000102CE0D3002070BDAC7E0020F8B5069CE1
:102A2000A58A266A521B658A12B2491B94F828505F
:102A300009B24FEAC57526B100948DB3FEF7C6FB07
:102A4000F8BD85B1207C810728D000F00301012961
:102A500024D0022901D1511C20D4C043800719D1B0
:102A6000002A1BDC16E0227C02F00304022C15D0A5
:102A7000D543AD0712D0012C01D100290EDC9207FD
:102A800001EB030208D0002A04DB494200D50021F3
:102A900099420DDB0020F8BD002A02DA0120F8BDC2
:102AA0000CE04A42F6D49A4206DA991A104401E040
:102AB000002901DB0FF0CFFE0220F0E7FEF72DFC2E
:102AC000EDE72DE9FC471C46DDF8288016460F4649
:102AD0008146B42B01DDB43C24B204F15A0000B2AB
:102AE00011F08EFB07EB6015204611F089FB06EB19
:102AF000601000B2CDE900082BB232463946484694
:102B000000F002F8BDE8FC872DE9F0470F46DDE94B
:102B100008699846154604462C210FF09CFEB542E4
:102B200006D1B9F1030F03D16D1E761E2DB236B258
:102B3000B54205DD4046B846074630462E460546B6
:102B400027816581A4F80C80E68184F81090678263
:102B5000A8EB07004B46A582002801DD024601E0F4
:102B6000A7EB0802711B002901DD0D4600E0AD1B3B
:102B7000AA4294F8282002DD42F0010201E022F08E
:102B8000010284F828200025E561244E2660A56115
:102B90002571D6074FF480150DD020B195FBF0F6C6
:102BA0004E43B612E66121B195FBF1F14143881223
:102BB000A061E0690CE021B195FBF1F64643B61245
:102BC000A66120B195FBF0F048438012E061A06956
:102BD0002062980709D003F00300012808D00228DA
:102BE00013D0D843800714D006E022F0020001E0A1
:102BF00042F0020084F82800206A811061620028F7
:102C000001DA48426062BDE8F087206A0028EFDC04
:102C1000EBE7206A0028EBDDE7E700001D2A01084A
:102C20002DE9FE4F0546DDF830900F461C4699F819
:102C300012009046C0F3000BB9F91060684609F124
:102C40000801FEF789FDBDF90210BBF1000F2FD07E
:102C500041454FDCBDF9061041454BDBBDF9000095
:102C60008119B94205DCBDF904203919921B914242
:102C700009DDBDF902108B1943453FDCBDF9062083
:102C8000931B43453ADBBBF1000F18D0C01B00D5A6
:102C90000020A04230DCBDF90410C91B091A491CF0
:102CA0004218A24200DD211A002925DB2844F4E065
:102CB000414513DCBDF9061041450FDBCEE7C61BCD
:102CC000A6420BDC002E03DB314628460FF0C3FD85
:102CD000BDF90400C71B7F1C002F02DC0020BDE8EB
:102CE000FE8FA74203DAE11BE8190FF0B4FD1EB90D
:102CF000A74201D10120F2E70220F0E7BDF804303D
:102D0000C21B181A401C0FFA80FCBDF80600401ABE
:102D1000401C03B2A8EB010000B2B04202DA301A44
:102D2000401E01E0991B401AD9F8141000B202238A
:102D3000CF6803EB4003FB5A37F81080A3EB08037E
:102D4000ADF808308B68496833F8103037F8100058
:102D500000EB010A02EB0C00801B18440FFA80F90B
:102D60009019C01A401E07B2BBF1000F4FF00006C9
:102D700021D06DE0811B01EB0A0010F801BC09EBCA
:102D800006005FEA000808D4A04506DA15F8081026
:102D9000584605F0C8FC05F80800B7EB060808D44B
:102DA000A04506DA15F80810584605F0BCFC05F8F1
:102DB0000800761C36B2BDF908008642DADB09EB62
:102DC0000600A04201DA014600E02146002901DAAE
:102DD000002002E0A04200DB204600B2211A284475
:102DE0000FF039FDBDF90800381A411CA14201DA83
:102DF0000A4600E02246002A01DA002402E0A1424D
:102E000000DA0C4621B2284647E0811B01EB0A009C
:102E100010F8010CC0F1FF0B09EB06005FEA000897
:102E200008D4A04506DA15F80810584605F07BFCD2
:102E300005F80800B7EB060808D4A04506DA15F82F
:102E40000810584605F06FFC05F80800761C36B2ED
:102E5000BDF908008642D8DB791CA14201DA781C52
:102E600000E02046002801DA002704E0A14201DA50
:102E70007F1C00E027463AB2A9EB0200A11A884263
:102E800001DA034600E00B46002B01DA002002E0E5
:102E9000884200DB084601B2A8180FF0DCFC2BE7E3
:102EA0002DE9F0411546064688880A881C46801A96
:102EB000401C02B2C8884B88C01A401C00B2824233
:102EC00000DA1046B5EB600F00DD4510002D00DA8A
:102ED000002506F10800FEF73FFC3582B474374840
:102EE0003060022030710023BDB1354A00204FF41C
:102EF0007A77C0EBC00102EB8101B1F91810A94249
:102F00001BD1C0EBC00002EB80004169491C41614C
:102F10000269102D04DA012103E07361BDE8F0813C
:102F200029111144B94205DA102D01DA012100E01E
:102F30002911571807617061F0E7401C0428D8D3A5
:102F400000242046C0EBC00102EB8101D1F814C07F
:102F5000BCF1000F07D12CB1D1F810C0D4F810E0AB
:102F6000F44500DA0C46401C0428EBD33CB1606900
:102F7000401CC4E90430102D0EDA01200DE01C20A5
:102F80000FF0D2FA040006D01C210FF064FC4FF0C1
:102F9000FF3020610BE0FEE728111844B84205DA43
:102FA000102D01DA012000E028111F1827612046AA
:102FB00029467461BDE8F041FAF731B8212C0108C7
:102FC0003C7E0020F0B50026094D0746344605EB4F
:102FD000C4004068B84204D155F83460204600F07F
:102FE00009F8641CE4B2102CF1D33046F0BD0000A7
:102FF000AC7E00200021421C08D0054A002352F874
:10300000301042F8303002EBC00043600846704791
:10301000AC7E002030B4D38854881B1B5B1C1BB2D1
:10302000012B09DB938814881B1B5B1C1BB2012B33
:1030300002DB036930BC184730BC704738B5044622
:1030400038210FF008FCFEF725FD0090BDF80000C8
:1030500024F8040FFEF71EFD0090BDF8000060800C
:10306000FEF751FC0090BDF80000E080FF252572BE
:103070000220A072FEF747FC0090BDF800006083BC
:10308000FEF741FC0090BDF8000020850748206154
:1030900004F8015CA57584F82650A57784F83250B1
:1030A000E07F20F03E001E30E07738BD34DC0408BD
:1030B0002DE9F04FC7B08346DDE95065087B98469F
:1030C00014460F4602287DD9B7F90200002879D0AE
:1030D000AE4277D01AB281469246404500DD914615
:1030E00001A8FFF7ABFF787B00F003008DF8060026
:1030F000B86840B100208DF80700B8680590387BAB
:103100008DF81E0005E0387B8DF807003888ADF893
:1031100008002188A8F10102A1EB0803ADF8F830FE
:103120006188A1EB0800ADF8FA0021881144ADF8E0
:10313000FC10B4F802C0ADF800316244ADF80411DF
:10314000ADF8FE20ADF80201ADF80621B7F802C0D7
:103150006344ADF80031B7F802C060440FFA80FC58
:10316000ADF802C17888081AADF804017988C01A50
:10317000511A4FF0FF3231920022401C09B200B2C6
:10318000ADF806114292002813DDA1EB0C00401CA3
:1031900000B200280DDD012347F6FF7240A932A8D6
:1031A000FFF77EFE01204290002132A8FFF71EFAB1
:1031B0003190002347F6FF723EA938A8FFF770FE52
:1031C000002100E028E038A8FFF710FA439006F548
:1031D000B470A84205D005F5B4714FF4B4708E42B6
:1031E00020D147F6FF70ADF804003EAA01A9584669
:1031F000FFF710FF4398FFF7FDFE3198401C02D007
:103200003198FFF7F7FE38A8FFF7C4FB4298002873
:1032100002D032A8FFF7BEFB47B0BDE8F08FA6F59D
:10322000B476B6B28642FAD202E0A5F5B475ADB274
:103230008542FAD228B245900090B4F90220B4F940
:10324000001033B20FA84493FFF72CFB00210FA806
:10325000FFF7CCF94690B54203D9A81BC0F5B4706E
:1032600000E0701BDBF8081000913C282ADDB8F163
:103270000A0F27D95A20B6FBF0F1B5FBF0F000F0A9
:103280000300ADF8B40001A8ADF8ACA0ADF8B050A3
:1032900001F003012E902A94ADF8AE60ADF8B210A3
:1032A000ADF8B6903EA8CDE92F0B2AA8FBF7B2FFE8
:1032B0002AA8FCF777F82AA8FCF743F92AA8FCF714
:1032C0002EFA04E03EAA01A95846FFF7A3FE0FA874
:1032D000FFF760FB38A8FFF75DFB429810B132A8FA
:1032E000FFF758FB4698FFF785FE4398FFF782FEED
:1032F0003198401C02D03198FFF77CFE787B400764
:103300008AD509F0FF022AAB51464498FDF77EFDAD
:10331000BDF8A80021882AAA0844ADF8A800BDF885
:10332000AC0021880844ADF8AC00BDF8AA00618863
:103330000844ADF8AA00BDF8AE0061880844ADF8B5
:10334000AE0042A8009906F004FE42ADC0B10023D1
:1033500047F6FF722AA92CA8FFF7A2FD00212CA88E
:10336000FFF744F9064658463EAA01A9CBF8085093
:10337000FFF750FE3046FFF73DFE2CA8FFF70AFB93
:1033800009F0FF022AAB51464598FDF73FFDBDF815
:10339000A80021882AAA0844ADF8A800BDF8AC000E
:1033A00021880844ADF8AC00BDF8AA006188084443
:1033B000ADF8AA00BDF8AE0061880844ADF8AE00D3
:1033C00042A8009906F0C5FDC0B1002347F6FF7280
:1033D0002AA92CA8FFF764FD00212CA8FFF706F905
:1033E00004463EAA01A95846CBF80850FFF712FE42
:1033F0002046FFF7FFFD2CA8FFF7CCFA0098CBF88A
:10340000080009E770B514460D460646FAF71CFA9F
:10341000224629463046BDE87040FAF7E4BB7CB549
:103420000446087E0D4602280ED9A268684629681F
:1034300006F08FFD002807D0626B0AB12046904746
:10344000626D2946204690477CBD2DE9F04FCD683E
:1034500089B00C46804615B1207C00286ED0207CB7
:10346000012800D10025D8F80400FEF7C0F9079024
:10347000D8F8082005A8216806F06BFD00285DD06B
:10348000F9F7D6F983460068D8F80090C16951BBB6
:10349000007C400611D4D8F80400BDF91410B0F92E
:1034A0000020B0F90200891ABDF91620121A0798F7
:1034B00000FB021109EB410014E0D8F80410BDF93B
:1034C0001630B1F90200B1F90010181A079B5843E1
:1034D00000EB400000EB0902BDF91400401A00EBBC
:1034E000400010448146D4F804A05FEA0A0013D0DB
:1034F0002068FEF77CF906462068BDF91410B0F983
:103500000020B0F90200891ABDF91620121A06FB34
:1035100002110AEB410A00E0002645B3DBF8000087
:10352000007C000710D460690CF050F902460021BD
:1035300008E0685C802802D9FF2001E035E0002027
:103540006854491C9142F4DB6069FEF750F9074664
:103550006069BDF91410B0F90020B0F90200891AB1
:10356000BDF916202944121A07FB021500E00027B6
:10357000D8F804004188008849420AB2404201B2AA
:1035800005A80CF056F9DBF80000C069C8B1606806
:103590000028207E0CD001A9009681E8A1005346A6
:1035A00005A94846079A05F059F809B0BDE8F08F1B
:1035B0008DE8A100A36805A94846079AFDF7D7F949
:1035C000F3E7607E78B161680029217E23D0009600
:1035D000CDE90370CDE90115534605A94846079A80
:1035E00004F00EFEE1E760680028207E0AD001A901
:1035F000009681E8A100534605A94846079A04F0C1
:10360000B9FED2E78DE8A100A36805A94846079A4C
:10361000FDF70AF8C9E7CDE90270CDE90015A36806
:1036200005A94846079AFCF761FFBEE72DE9F04778
:103630001D469046DDE90829B5F9024014FB08F063
:1036400001EB4001B5F900000A9B01EB4006B3F91C
:10365000021001FB09F102EB4101B3F9002001EB7B
:103660004207A988081A401C00B24FEA400A0AE043
:103670005246394630460FF01FF8641C06EB4806E8
:1036800007EB490724B2B5F90600A042F0DABDE81D
:10369000F0872DE9FF4F9BB00C461B981546DDF8CF
:1036A000A0A0816817A8FEF760F817A8FFF78EF9A9
:1036B0001390208818B96088B0F5807F01D0012070
:1036C00000E0002014901C2106A80FF0C4F8E07A56
:1036D0008DF83000207B0DF1380B00F00F008DF8D5
:1036E0003100CDF818B0DDE9131001434FF00006AA
:1036F0004FF002082BD1BAF1040F06D0BAF10E0F29
:103700000AD0BAF1140F20D021E0A07AF8B91E989F
:1037100006A9CDE9065012E01B9829468268684642
:1037200006F017FC00280DD01E9807960B950990FF
:103730002089ADF820008DF8288006956AE01B9856
:10374000FFF76DFE1FB0BDE8F08FA07AE8B31B98BD
:1037500080680188ADF838108088ADF83C001B986F
:1037600080684088ADF83A001B988068C088ADF842
:103770003E002846FEF741F815902846FEF719F856
:1037800012900EA8FEF715F807460EA8FEF735F8BA
:103790000D90F9F74DF80CF0AFFB06460EA80CF0B3
:1037A00015F801460D98B14201D9B6FBF0F7784300
:1037B000169040000EF0E6FE814616980EF0E2FEEE
:1037C0000646CDF82CB0099000E011E002208DF8FB
:1037D00028007F1EBDF83A00BDF93EB03844199765
:1037E000CDF81C90ADF83E00BAF1040F1AD113E0E9
:1037F0002846FEF702F804462846FDF7DAFF1E9930
:1038000007910A46610001FB002006950B9509907F
:103810008DF8288006A992E7208818B96088B0F54D
:10382000807F01D0022000E001208DF82800C2E056
:103830000EA910A8FDF799FF6888404202B22888B7
:10384000404201B210A80BF0F4FF149870B1CDE91A
:10385000024ACDE9049615991298CDE9000110A904
:10386000159B1E9A1B9800F0D5FD0BE0CDE9014A8F
:10387000CDE9039615980090024610A8129B1E9958
:10388000F9F7FEFDA07A022863D9218989B2C1F334
:10389000C40212FB00F2ADF808204A07920E02EBB8
:1038A000513212FB00F2ADF80A20C1F3042111FBE2
:1038B00000F1C0F1FF02ADF80C10002046E009EB6A
:1038C000400CBCF80010ADF80410BDF80430BDF891
:1038D0000810C3F3C40717FB021101EBC11707EB74
:1038E000C131BDF80070C1F3C45161F3C707590776
:1038F000890EBDF80A8001EB533111FB028101EB07
:10390000C11808EBC1384FEA986868F3020701EB69
:10391000C11808EBC131C1F3C25161F34F37BDF893
:103920000C10C3F3042313FB021101EBC11303EBCF
:10393000C131C1F3C45161F30C27ADF80070B9B2C5
:103940000091BDF80010ACF80010401C1699884298
:10395000B5D31398E8B1B046BDF93A7015E0BDF99A
:1039600038103A4640460D9BFEF7F2FF10B1022890
:1039700004D006E040460D990EF06DFF02208DF850
:1039800028000D997F1C88443FB2BDF93E00B84223
:10399000E5DA06A91B98FFF742FDBDF83E0019992C
:1039A000401CADF83A00084400B2ADF83E0058455E
:1039B00001DDADF83EB0BDF93A1059457FF738AF9B
:1039C00030460EF02BFE48460EF028FEBAE6000008
:1039D00010B50C46582120460EF03DFF104860619E
:1039E0001048206110482063104820621048A061F0
:1039F000104860621048A0621048E062104860639E
:103A00001048A0631048E0631048206410486064C8
:103A10001048A064104860652C20E06410BD0000D0
:103A2000B13001085941010805340108253C01085D
:103A3000933601083B3D0108DD3E01089141010834
:103A4000134401082D360108293B01085D3A01089D
:103A5000A93A01081F3C01084B3401082DE9F04147
:103A600017460C460646F8F7E3FE0546F807A06A37
:103A700020F000410BD060690EF0EDFEA06A40F02E
:103A80000041A1622868016941F0400104E0A1629F
:103A90002868016921F04001016160690834C6E9C4
:103AA0000004B460BDE8F081FEB5054600680290F0
:103AB0000098164620F0E00000900C466868FDF77C
:103AC000A2FE009960F3942100916868C188408843
:103AD000081A0099401C60F35F510091A06A002809
:103AE00001DA052000E0042060F304010091206A5F
:103AF0002860E0696860A069A860F8F799FE00682E
:103B000094F824206B46016962F38611016104F187
:103B1000080231462846FEF7D1F9284600F095FC08
:103B200068460DF077F8FEBD70B5064615460C46A2
:103B3000D00701D0002070BDA80743D5A06A00F0CF
:103B4000004000F5C040A06220460BF03FFEA16A95
:103B5000400021F00042824202D960F31E01A162BE
:103B6000A06A20F000400EF0DFFC2146606168B9D9
:103B7000A06A00F0004000F54060A06220F0004024
:103B80000EF0D2FC214660610028D4D00846D0E96E
:103B900000128160E2606188E181A1892089081AB0
:103BA000401CA16A00B221F0004100EB400291FBF1
:103BB000F2F12182A16A21F0004191FBF0F0411065
:103BC00061822AE00846D0E900128160E2600BF0D1
:103BD000FDFD4100A06A61F31E00A06220F00040DC
:103BE0000EF0A2FC6061A16A21F000410EF033FEEC
:103BF000A06A05F0010565F3DF70A0626069002826
:103C000099D0306004F108007060B060F8F710FEE1
:103C10000068016965F386110161204670BD48693D
:103C20000EF00EBDF0B51D46074697B014460E4681
:103C3000086800232A460FA90CF0A7FAF0B3BDF8D4
:103C40004420002A3FD0BDF842C0BCF1000F3AD05A
:103C50002088BDF84610084401B2ADF84C10306819
:103C600003894089181A638801EB0C041844BDF8D5
:103C70004830801AC01A03B2ADF84E30B868B0F9B7
:103C800000C064451FDBB0F90440A1421BDC991859
:103C9000B0F90220914216DBB0F90600834212DC33
:103CA00029460F980CF06DFA00280CD00F99097B6B
:103CB000890708D10FAB13AA314600E005E0009058
:103CC0003846FAF7C9FD17B0F0BD202DFBD3A5F596
:103CD0007840FF38F7D0A5F500500C38F3D0208895
:103CE000BDF84610BDF84820084401B26088104471
:103CF00002B2BDF84400104400B20090BDF842008A
:103D0000084403B214A80BF0A1FD01A8FFF796F92F
:103D100002208DF807008DF82E008DF83A008DF8FE
:103D20001E00B089ADF822000120ADF824003B69E7
:103D300014AA01A938469847C5E72DE9F04715466A
:103D4000B1F9022092B01C460E468146002A7ED070
:103D5000307A02287BD9B5F90010B4F9000081420D
:103D600005D1B5F90230B4F90270BB426FD081427F
:103D700000DA084602EBD271A0EB6100ADF840001A
:103D8000B5F90000B4F90010B6F90220884200DC51
:103D9000084602EBD27100EB6100ADF84400B5F9C2
:103DA0000200B4F90210B6F90220884200DB08468E
:103DB00002EBD271A0EB6100ADF84200B5F9021040
:103DC000B4F90200B6F90220814200DD084602EB98
:103DD000D27100EB6100ADF8460010A90846D9F891
:103DE000082006F0B6F8002875D010A9D9F808A068
:103DF000C9F80810B5F90200B4F90210884206D1DA
:103E000023462A4631464846FAF78AFE0EE0B5F9BF
:103E10000000B4F90010234688422A46314648463D
:103E200002D1FBF7E9F801E0FAF738FF707A0107F1
:103E300001D440074DD56846FFF700F93088ADF84A
:103E4000040047F6FF70ADF80000307A00E042E071
:103E50008DF80300B6F90200471040F3000000F1AE
:103E60000108707A400718D528880EAAC01BADF843
:103E700038006888C01BADF83A002888C119A1EB4A
:103E80000800ADF83C006888C119A1EB0800ADF846
:103E90003E0069464846FFF7BDF8707A000718D51E
:103EA00020880EAAC01BADF838006088C01BADF892
:103EB0003A002088C119A1EB0800ADF83C006088E9
:103EC000C119A1EB0800ADF83E0069464846FFF76E
:103ED000A1F8C9F808A012B0BDE8F0872DE9FF4F9E
:103EE0008BB01F461646032B7ED3002E7CD0B80025
:103EF0000EF048FB04007BD0002530682060284687
:103F00007A1E15E006EB800136F92030B1F904C0C5
:103F1000634505D1B1F90230B1F906C0634505D05A
:103F200004EB850309686D1C1960ADB2401C80B2BA
:103F30009042E7DB06EB8700B6F9001030F9042C5D
:103F4000914205D1B6F9021030F9022C914206D007
:103F500004EB850150F8040C6D1C0860ADB2032D14
:103F600043D37C48D0E90010CDE90210002027E0BF
:103F7000BDF9081034F92020914200DB1146ADF85C
:103F8000081004EB8003BDF90A10B3F90220914236
:103F900000DB1146ADF80A10BDF90C1034F92020F1
:103FA000914200DC1146ADF80C10BDF90E10B3F9CA
:103FB0000220914200DC1146401CADF80E1080B288
:103FC000A842D5D30B9802A9826805A805F0C1FFC5
:103FD00058B10B9805A90026806809900B9881605C
:103FE000B4F90220012010E002E020460EF016FB9A
:103FF0000FB0BDE8F08F04EB8001B1F902109142DF
:1040000001DA0A4606B2401C80B2A842F3D32C2142
:1040100005FB01F00EF0B6FA8346B2460490D14695
:104020004FF00008701E00D528446A1E09F10101F6
:104030000792914200DD002134F8203034F8262028
:1040400034F821709B1A04EB8000BA1A478804EBFD
:10405000860004EB8101408849883E1A081A002135
:10406000089116FB02F110FB03F0814267DA012090
:10407000089001E00898E8B307980AF10106864223
:1040800000DD0026B9F1010700D52F4404EB8600BE
:1040900004EB8A01B0F90200B1F90220904216DB6C
:1040A00012D034F9263034F92A108B420CD04FF05C
:1040B000010CCDE9000C5846FEF726FD5846049940
:1040C000FEF794FA0BF12C0B08F10108B246A84553
:1040D00023D004EB870004EB8901B0F90200B1F9A9
:1040E0000220904217DB13D034F9273034F929101D
:1040F0008B4200E023E00BD00026CDE900065846B5
:10410000FEF702FD58460499FEF770FA0BF12C0BEE
:1041100008F10108B946A845ACD3DDE90B0102AAB4
:10412000FEF778FF0498FEF74DFF04980EF076FA3C
:1041300020460EF073FA0B990998886058E7BAF197
:10414000010600D52E44079809F1010787429DDD3D
:1041500000279BE7BC9D010870B514460D46064636
:10416000FBF7FEFB224629463046F9F76DFB224657
:1041700029463046F9F737FD224629463046F9F7F9
:1041800024FE224629463046BDE87040FAF7DFBFDC
:104190002DE9FF4F99B00F4628984FF480314FF02A
:1041A0000A0BB0F90000DDE92A6540420F9028981B
:1041B0004088B1FBF0F00F990E9091FBFBF428982A
:1041C00004F1010A40681290604200EB800001EBAC
:1041D000400920B210F014F801900FFA8AF010F0A4
:1041E0000FF85A34009020B210F00AF880460AF115
:1041F0005A0000B210F004F8019AC9F10A0101FB5B
:1042000002F4009B01FB08F100FB091103FB0943C9
:1042100091FBFBF093FBFBF20D9050110C900D986D
:1042200040110D90BDF9480000021090BDF94A0000
:1042300000021190B8883988401A401C04B2F888EE
:104240007988401A401C00B21790002049E014A859
:104250000090B7F9021013AB01EB0A02B7F9001096
:1042600008A805F0B4FC16A80090B7F9021015AB29
:1042700001EB0A02B7F9041008A805F0A8FCDDF864
:104280004CC01598149AA0EB0C0816980021831ABC
:104290000846012C07DD601E4FEA082191FBF0F172
:1042A0001B0293FBF0F0289B80320CF1800C1B7DED
:1042B000DB07299B1CD00DF10C08CDF800C088E865
:1042C0005100CDE90121CDE90653DDE91B01DDE90E
:1042D0002623F8F7F1FB0AF1010006EB440625441A
:1042E00000B2179982468842B1DB1DB0BDE8F08F5D
:1042F000042B4BD0052B10D0062B47D0142BEAD122
:10430000DDE91B38CDF81080DDE926EBCDE90010A2
:10431000CDE902C2B146002078E0DDE91BE3CDE93A
:1043200000100393269B0293B146E346DDF89C8080
:10433000002028E0009941430BEB212301994143E0
:1043400002EB21211B124FEA212C08D403998B4246
:1043500005DABCF1000F02DB02998C4502DB00217B
:1043600029540EE00CFB083303EB430303EB0E016F
:104370000B7891F801C003EB0C2329F810308B78EF
:104380002B54401C00B2A042D4DBA4E70DF10C0872
:10439000CDF800C088E85100CDE90121CDE90653F0
:1043A000DDE91B01DDE9262304F073FE93E70099A4
:1043B000029A414302EB21220199DDF80CC04143EE
:1043C0000CEB212112124FEA212107D4DDF810C095
:1043D000624503DA002901DB714502DB0021295423
:1043E00012E001FB0B2C03EB4C0C09EB4008BCF872
:1043F00000C0A8F800C00BFB0EFC03EB4C0C6244A1
:1044000001FB0B210A782A54401C00B2A042CEDBEB
:1044100061E770472DE9F04387B08946DDE9125125
:10442000DDE91076DDE90E8C70B1C46A002C08D08D
:10443000CDF80080CDE904510396CDE901C7494686
:10444000A04707B0BDE8F083FEE7416B002900D02C
:104450000847704710B5174917481DF046FF38B197
:10446000144915481DF05BF9124913481DF03DFF32
:1044700012480BF05BFF1148432101704FF40071AB
:1044800041800F4981600F49C1600F4901610F49A7
:1044900041610F4981610F49C1610F4901620F49B3
:1044A00081620F4941620449C162BDE810400BF0CE
:1044B00041BF0000540C0408544000209C7C0020A4
:1044C000150B0108450A01085D0B0108AD0B010839
:1044D000750B0108950B01087D0A0108610A0108A6
:1044E000A50A01082DE9FC418646807815460C4650
:1044F00010FB04F00012824203DCBEF80000BDE8AD
:10450000FC819EF808C00EEB8C0212F8023C13FBF3
:1045100004F31B129D4202DB32F8040CEFE7002289
:10452000012324E00EEB8307BF7817FB04F73F124B
:10453000BD421ADC0EEB830737F8040DADF804001A
:104540000198FDF781FA0646B888ADF80400019895
:10455000FDF77AFA0146B87810FB04F0BA79001238
:1045600012FB04F2C0EB222203E05B1CDBB29C4591
:10457000D8D8E2B3281A00B2C0EB002090FBF2F0CA
:10458000C0B2C0F1FF02C1F3072313FB00F3C6F36F
:10459000072414FB023303EBC31404EBC334BDF84C
:1045A0000050230F63F30205C1F3074313FB00F32D
:1045B000C6F3074717FB023303EBC31707EBC333FD
:1045C0009B0E63F3C705C9B211FB00F0F1B211FBFA
:1045D000020000EBC01101EBC030800E60F30C252F
:1045E000600E60F34F35ADF80050A8B287E7FFE7E3
:1045F000FEE74168002901DA0EF022B8704700009A
:10460000FEB50546407A16460C4640072ED0224F8E
:10461000387820B9002000F043F801203870687A1B
:1046200000F00700022817D0304680EA6400684096
:104630000190002000906A4601A91848FCF796FCFA
:1046400001280BD0324621462846F8F707F900909A
:1046500000280BD0002418E02046E6E7009804224A
:10466000416802EBB1714FEAB1014160FEBD2246E3
:104670002846FFF737FF02900098BDF808108068C1
:1046800000EB4400641C018024B20098B0F90E10C5
:10469000A142ECDCFEBD0000C8340020230A010862
:1046A00070B5094C054620680DF0CAFF28460DF08C
:1046B0003BFF2060054CA06020B129460EF0CBF8EE
:1046C000656070BDFEE700006C350020C834002036
:1046D000014600200F290AD2DFE801F00909090983
:1046E000080A080C0E10120C0E1012001020704751
:1046F000182070470120704702207047042070473F
:104700000820704701460020891E0D2909D2DFE8E4
:1047100001F007080807080707070707070707004A
:104720000120704701460020032901D0062900D14D
:1047300001207047032130B10078A0F120015F29EA
:1047400003D80120704708467047802801D3022013
:10475000704700207047000038B5174C20780028BB
:1047600029D10DF083FFF8F76BF805F0A7FDF7F7F7
:1047700061FD05F0A9FDFDF7EDFBF7F75DFF4FF4D7
:10478000B4710E4806F0C5F85C210D4806F0C1F87A
:10479000F8F754F805F07EFE0A4800909DF80000F6
:1047A000112802D0002010B1FEE70120FBE70BF03A
:1047B000A8FC0120207038BDAC340020FC7C002017
:1047C000087D0020443322112DE9F0410A4C0746B0
:1047D0000A4D60680E46401CC100606028680DF0FC
:1047E00053FF286038B1616800EBC10040E90276F0
:1047F0000846BDE8F081FEE7B43400205C350020B7
:104800002DE9FF410C46074602F024F90646E00771
:1048100002D0384602F0C5F8F8692043F861E00795
:1048200011D00221384601F037FE60B1384600F061
:1048300017FF050007D00BF08FFF28460CF00CF88F
:1048400008B102F0AEF8384602F004F9B04202D1E5
:1048500014F0C07F07D0384600F042FF02F033F971
:10486000384602F030F9E0060CD502AA694638460F
:1048700001F07DF86946384602F0B6F802A93846DC
:1048800002F0B2F8BDE8FF81028C11438A4201D0E8
:1048900003F05CB870472DE9F047174688464FF69D
:1048A000FF79054600234A46394605F0BDF8698C74
:1048B00000240426C1F30513EA6808E006EBC400EF
:1048C00010585FEA801C01D4C00102D5641CA342C9
:1048D000F4D84FF0806000EBB1204FEAB05068840C
:1048E000C0F30510C10010460DF0CEFEE860688CE4
:1048F0006FF00703C0F3051009E0E96803EBC00C93
:1049000001EBC0026144D1E900C1C2E900C1401E0F
:10491000A042F2D8E868082100EBC4000DF09BFF2C
:10492000E96841F83480E86806EBC401425867F34F
:10493000170242504A4639462846BDE8F04702F081
:10494000C5BC000010B504468068002813D10B4890
:104950004168491C41601C200DF0E6FDA06058B183
:104960001C210DF078FFA1680F204876A068017E19
:1049700041F00301017610BDFEE70000AC340020D9
:104980002DE9FC410D460746012101F079FD002883
:1049900050D1384600F0A8FE044600F043FE06461B
:1049A0000BF0DAFAA0420ED030460BF0DDFAA0424E
:1049B00009D030460BF0BEFAA04204D030460BF0CE
:1049C000B1FAA04236D14FF400263146384601F004
:1049D0005EFD18BB3846F7F744FD044607F11401A5
:1049E0006846FCF79EFEBDF800002946001BADF8A6
:1049F0000000BDF802006A46001BADF80200BDF8D9
:104A000004002044ADF80400BDF806002044ADF8D1
:104A10000600084605F09DFA00280CD0002301226C
:104A20002946384601F05AFC38461DE0012101F0C4
:104A300027FD10B10020BDE8FC813146204601F081
:104A400026FD80B9D4E90501CDE90001002301224A
:104A50006946204601F042FC29466A46084605F0B0
:104A600078FA0028E7D0204600F03AFE0400DDD1B5
:104A70000120E0E72DE9F0410E460746002401F051
:104A8000F9FB050035D03146384601F0E7FB022836
:104A90002FD905EBD570012101EB60053146384671
:104AA00001F0E2FB28440FFA80F83146384601F065
:104AB000C9FB05463146384601F0CAFB002D01DD31
:104AC000294600E06942002801DD024600E042423A
:104AD000914205DD002D01DD284604E0684202E038
:104AE000002800DC4042404400B2002800DA2046A2
:104AF00004463146384601F022FB05000ED031460F
:104B0000384601F010FB022808D93146384601F03A
:104B100010FB2844A04200DB044624B2384631464C
:104B2000692201F042FB05B2384631466A2201F0A3
:104B30003CFB00B2854200DD2846002801DD204410
:104B400004B22046BDE8F08170B50D4606465B22F2
:104B500001F02BFBC4B230462946162201F025FB9A
:104B600004B90124204670BD002803D000688842A3
:104B700001D1012070470020704700002DE9F0416D
:104B80000D4606460027364900E00068B8B1826944
:104B90000A42FAD08069C0F30F1080460DF0C4FCC1
:104BA000041E31D041460DF056FEC4E900654FF0B9
:104BB00001086FF0030625B1A86878B332E03846E3
:104BC000EBE70BF081F905001AD0EA68F2B1686AE8
:104BD000401C8100686210460DF056FDE860696A6D
:104BE00006EB81014450A782E78200200BF084F994
:104BF000401E208300200BF0C5F9401E608323E097
:104C000020460DF01DFD0020BDE8F08104200DF0D0
:104C10008BFCE8600460C5F82480E4E7FFE72846E1
:104C2000FFF790FEA868016881B14168491C4160A6
:104C3000A868890000680DF027FDA9680860A968C8
:104C4000496806EB810144502046DDE704200DF061
:104C50006BFCA96808600460A968C1F80480F3E7E8
:104C6000F0FF0F0070B5054601F02DFF002000F0A9
:104C700093FA28460FF01EF9284600F06FF801203D
:104C800000F08AFA4FF6FF724FF47021284602F0C6
:104C90001DFB284602F002FB0BF0D2FD030007D0FB
:104CA000284601F0C8FE18B1294618460BF000FD51
:104CB000284600F015FD04000DD02A4622210BF0F5
:104CC000F5F92A46232120460BF0F0F92846BDE8E5
:104CD000704001F066BE70BD7FB50C46064601F01F
:104CE000B9FE0546E0060CD502AA6946304600F03A
:104CF0003EFE6946304601F077FE02A9304601F0DB
:104D000073FEF069A043F061E0070ED0304601F079
:104D100048FE304601F09EFE38B1304600F0E0FC1F
:104D200001F0D1FE304601F0CEFE304601F092FE99
:104D3000A84202D114F0C07F07D0304600F0D0FC6A
:104D400004B0BDE8704001F0BEBE7FBD028C22EA17
:104D500001018A4201D002F0F9BD704770B50568C3
:104D60000446286818B120602046FFF7F7FF256049
:104D70006A682846002A03D02146BDE870401047E3
:104D800070BD2DE9F0414D680C46EDB1284600F0AC
:104D90000DFD0646284600F0D5FD074628460021B1
:104DA000102201F002FAE98A12220844C01BE082B4
:104DB000401E60832846002101F0F7F9A98A0844C3
:104DC000801BA082401E208341F20200E061002D82
:104DD00005D043F20200E06143F20230E06140F0AE
:104DE000740040F40060E06102D040F40040E061F3
:104DF000BDE8F08110B501460348FFF7BFFE044649
:104E0000FFF730FF204610BD609C01082DE9F041FE
:104E1000074601F0C6FD384600F062FC4FF0000482
:104E20000500264608D1384600F0FCFB040018D0E7
:104E30002069B84200D10126384603F09BFC65B1D9
:104E4000284602F001FD0022222128460BF02EF90F
:104E50000022242128460BF029F9002E01D0002041
:104E60002061BDE8F081000070B50C46084605F0F1
:104E70000FFA002000F090F92046144A002102F0B9
:104E8000FBFA012000F088F900212046FCF730FBF6
:104E9000204600F0E5FB10B120460BF020FDA06895
:104EA000002811D00068002518B10DF0C9FBA068DA
:104EB0000560A068C06818B10DF0C2FBA068C560AD
:104EC000A0680DF0BDFBA56070BD0000FFFF0F00E6
:104ED0002DE9F047A2B080460BF0A5F80446404605
:104EE0000BF0DFF8012700260546122C72D0DFF800
:104EF0009492152C6CD0182C7AD140460BF099F86E
:104F0000824601462846FAF7D7FC0021284601F0E0
:104F1000C0F850B105F59070FEF754F8040004D0C5
:104F2000FDF738FD20460DF079FB0021284601F001
:104F30009CF800285CD06846FEF780F88DF8036086
:104F40008DF81A608DF82A608DF836606A46002167
:104F5000284601F0C9FB0021284601F0A7F9804648
:104F60000021284601F09CF9044605F1140120A80F
:104F7000FCF7CEFBBDF88010A1EB0800BDF8841053
:104F8000ADF8800001EB0800ADF88400BDF88200A8
:104F90005146001BADF88200BDF886002044ADF8F4
:104FA00086000EA800F0F0F820A81B96CDE910703E
:104FB000CDF83C90CDF848D00EAA1A2128460BF027
:104FC00075F820AA69465046FEF724F8D4E001E0BF
:104FD00055E00DE040460BF062F8044600780228E8
:104FE00006D00021284601F054F820B1022020709C
:104FF00022B0BDE8F0870021284601F01DF9824665
:105000000021284601F052F981460021284601F08E
:1050100047F9804605F114016846FCF779FBBDF8B5
:1050200000105246A1EB0900BDF80410ADF80000D5
:1050300001EB0900BDF80210ADF80400A1EB080077
:10504000BDF80610ADF8020001EB0800ADF806004F
:105050006946606804F0A5FF68B10021284600F0A9
:10506000F8FFFD2807D328460021602201F09DF8B3
:10507000C0B2FD2801D22770BAE72670B8E74046D3
:105080000AF0D7FF80466846FDF7D8FF0021284682
:1050900000F0EBFF28B19DF8230040F001008DF8EF
:1050A00023006A460021284601F01EFB0021284605
:1050B00001F0FCF807460021284601F0F1F804460B
:1050C00005F114018A4620A8FCF722FBBDF88000F8
:1050D0004146C01BADF88000BDF884003844ADF8EF
:1050E0008400BDF88200001BADF88200BDF8860088
:1050F0002044ADF886000EA800F046F820A8CDE9BF
:105100001060CDF83C90CDF848D00EAA1A21284660
:105110001B960AF0CBFF0021284600F0BAFF20B111
:10512000BDF8000008B1012700E00027049C07B18A
:10513000049620AA69464046FDF76CFFE7B11820A7
:105140000DF020FA0746BDF9002000235146FDF777
:10515000A7FE05F590713846FDF748FA64B18DF861
:1051600003608DF822608DF82A608DF8366020AAE1
:1051700069464046049427E70EAA1B2128460AF0F8
:1051800095FF35E7609C010870B50C46054648213F
:105190000DF061FB2C6070BD014908707047000084
:1051A000BC3400202DE9FF41884608460AF03BFF49
:1051B000044640460AF03BFF0546012C23D0082C4C
:1051C00023D0032C3ED02A2C3ED00D2C4CD00E2CBC
:1051D0007DD0092C7CD00A2C7BD00F2C7AD0292CA6
:1051E00079D0222C78D0242C77D0132C76D0152C83
:1051F00003D0182C01D0122C34D104B04046BDE8A5
:10520000F041FFF765BE2021FAE02021FFF79EFD67
:1052100040460AF01FFF0CF052FB002822D1082163
:10522000284601F02DF900281CD095F820004FF0F9
:105230000101C007284602D0FFF788FD30E0FFF7E4
:1052400023FB2DE02021F8E000F05CF90646002465
:1052500006E0A868006850F8240001F034FC641CE3
:10526000B442F6D3BDE8FF81082101F009F9F8B195
:1052700040460AF014FF0478132C06D0112C04D0F9
:10528000142C07D0122C05D008E001212846FFF786
:10529000FBFA03E001212846FFF758FD0A2CE1D074
:1052A00004B02846BDE8F04100221C210AF0FEBEF1
:1052B0004FF40161284601F0E3F80028D2D02846D7
:1052C00001F0ACFB0028CDD10027284607E06DE0B7
:1052D00095E09AE0B0E0B5E0D1E0F2E0F6E000F071
:1052E00065FA0646284600F0C1FA044640460AF030
:1052F000D6FE007812281BD011280CD013282BD0F2
:105300001428AFD1284600F049FA800703D0002EB8
:1053100038DC002C36DC284600F0A7F90446284685
:1053200000F01EFBE11704EB9171A0EBA1000BE074
:10533000284600F09AF90446284600F011FBE117D0
:1053400004EB917100EBA10001B204B03A4628468B
:10535000BDE8F04102F062BA284600F01FFA80076B
:10536000E6D0002E01DC002CE2DD284601F069F8D1
:105370000446284600F0EDFAE11704EB917100EBCA
:10538000A1000BE0284601F05CF80446284600F036
:10539000E0FAE11704EB9171A0EBA10001B204B0B7
:1053A0003A462846BDE8F04102F022BA4FF4806147
:1053B00001F066F818B10121284602F0FCF92846F0
:1053C00000F04EF90BF042FA064602240CF042FAC5
:1053D00010B940460AF03EFE0CF07DFA022801D0DA
:1053E000042800D106241EB144F00801284607E035
:1053F00021462846FFF748FA082128461DE04021AB
:1054000004B0BDE8F041FFF73FBA4021FFF79EFC32
:10541000284600F0D2FD02287FF424AF02AA694694
:10542000284600F0A4FA6946284601F0DDFA02A9F0
:10543000284601F0D9FA15E70E2104B0BDE8F04185
:10544000FFF784BC002100F0DFFD04460021284660
:1054500000F02DFE204302D0284601F034FB284600
:1054600000F050F80646002406E0A868006850F8EE
:10547000240001F028FB641CB442F6D3F2E60021BC
:10548000012200F092FE06B228460021042200F01C
:105490008CFE04B20021284600F0B6FD074600212C
:1054A000284600F004FE384305D142F2D17086420E
:1054B00001D08442BFD104B02846BDE8F04101F0DC
:1054C00002BB688C40F002006884F4E70021FFF71B
:1054D000D1FA014604B04046BDE8F0410AF006BEEC
:1054E0008068002809D0002902DA4268511803D4E4
:1054F00043680A468B4201D800207047006850F884
:10550000220070478068002800D04068704770B55E
:105510000C46054600F114012046FCF702F9A86884
:10552000002812D02188808A081A2080A968A088C3
:10553000898A0844A080A9686088898A401A6080A6
:10554000A968E088898A0844E08070BD70B50C467F
:105550000546002100F091FD06462146284600F050
:105560005BF8704202B2114620460AF055F900215C
:10557000284600F0F6FD21880844208000212846B6
:1055800000F0FBFDA188081AA0800021284600F049
:1055900000FE6188084460800021284600F0D5FDA7
:1055A000E188081AE08070BD2DE9F041064600212F
:1055B00000F0EFFD05460021304600F0C6FD044630
:1055C0000021304600F059FD0746304600F04DF806
:1055D000401B001B794200EB410000B2BDE8F081A6
:1055E0002DE9F0410646002100F0BBFD05460021F3
:1055F000304600F0C2FD04460021304600F03DFD7B
:105600000746304600F01DFF401B001B794200EBAF
:10561000410000B2BDE8F0810A4600F114011046D5
:10562000FCF77FB810B5416809B100F05DF8044699
:105630000A4805F051F90EE00022416A05E0C3680E
:1056400053F82230A34208D0521C9142F7D80146A9
:10565000024805F053F90028EED110BDFC7C002073
:105660008068002800D0806870471430FCF78FB83D
:1056700070B5064600F034F8051E08D0002408E096
:1056800021462846FFF72CFFB04201D1204670BDCD
:10569000641C2846FFF736FFA042F1D84FF0FF30D8
:1056A00070BDF0B4458C00240426C5F3051712E044
:1056B000C56806EBC40C55F80C505FEAC51C09D54B
:1056C00025F07F459D4205D1C06850F83400F0BCFC
:1056D0000EF04CB8641CA742EAD8F0BC002070471A
:1056E000002800D04068704700B50146FFF7F8FF7A
:1056F0000028FAD1084600BD2DE9F047DFF8949064
:1057000080464C46FFF7FEFE06460025DFF888A0DF
:105710000FE0D8F808005146006850F82570384668
:1057200000F0B5FE20B9B7F91A00A04200DB04462C
:105730006D1CB542EDD30021404600F030FD82469D
:105740000021404600F007FD06460021404600F0DB
:105750009AFC05464C4505D0B8F81A00801B401B42
:10576000201A04B2404600F031FC07464046FFF7DD
:105770007CFFA0EB0A00801B694200EB4100391A54
:10578000404600F0EDF8081A00B2844200DD2046E1
:10579000BDE8F08701E0FFFF01000400806818B158
:1057A000407E00F00F0070470F2070472DE9F84F42
:1057B0000646002100F03AFC012807D0B068002816
:1057C00002D0008A404200B2BDE8F88F0021304686
:1057D00000F0D9FC00900021304600F0C8FC814662
:1057E0000021304600F04FFC824641F6FF7B5C46CC
:1057F0003046FFF787FE804600250EE0B068194965
:10580000006850F82570384600F041FE20B9B7F91D
:105810001400A04200DC04466D1C4545EED35C45F7
:1058200006D0B28A09EB0A001044001B04B200E063
:105830000D4C304600F0D8FB0546304600F001FE26
:105840000099411AA1EB0901CAF1000001EB4000E7
:10585000291A304600F07DF8084400B28442B3DDD6
:105860002046B1E70100040001E0FFFF2DE9F04709
:105870000646002100F0DAFB01280AD0DFF8A090EC
:1058800030464C46FFF73EFE80460025DFF894A0E8
:1058900015E0B068002801D0B0F91000BDE8F0872D
:1058A000B0685146006850F82570384600F0EFFDAA
:1058B00020B9B7F91800A04200DB04466D1C45452D
:1058C000EED30021304600F05EFC07460021304652
:1058D00000F04DFC82460021304600F0D4FB054626
:1058E0004C4504D0308BC01B401B201A04B23046FC
:1058F00000F07AFB8046304600F0A3FDC11BA1EB0F
:105900000A00694200EB4101A8EB0101304600F0BA
:1059100020F8081A00B28442C0DD2046BEE700002D
:1059200001E0FFFF010004008068002802D0007E33
:10593000C0F3810070478068002802D0007EC0F369
:10594000011070478068002802D0408A404200B2AF
:1059500070478068002802D0008A404200B2704739
:105960008068002802D0408A404200B270472DE98A
:10597000F04F8DB016460C464FF0FF37054600221B
:105980003B4611462046009709F060FF00223B4647
:1059900011463046009709F059FF1021284600F0C3
:1059A0006FFD002816D0284600F007FB070011D035
:1059B00000200BF055FF8046022F08D010E00BF0BE
:1059C0007EFFA84209D040460BF04AFF8046B8F15E
:1059D000000FF4D10DB0BDE8F08FB8F1000FF9D091
:1059E0002846FFF7AFFF09902846FFF785FE0C9089
:1059F0002846FFF7DBFE07902846FFF737FF0B909E
:105A00002846FFF7CBFE8146002019F00C0F0390CB
:105A100014D0012F10D0032F02D0022F07D00DE099
:105A20000998002808DC0C98002805DC06E04046B0
:105A30000BF036FF0C2801D10120039000200290CA
:105A40005FEA897014D0012F10D0032F02D0022FEB
:105A500007D00DE00798002808DC0B98002805DC2B
:105A600006E040460BF01CFF032801D10120029004
:105A7000DDE902010843ADD04FF4803739462846AE
:105A800000F0D4FA012800D000200A9039462846B8
:105A900000F085FB01903946284600F05CFB089039
:105AA0003946284600F063FB80463946284600F018
:105AB0006AFB814628460122394600F076FB0FFA40
:105AC00080FB2846FFF7D1FD0090284600F0B9FC86
:105AD0000690039800B158468246029800B1584695
:105AE000059028463946212200F05FFBC0B202280B
:105AF00008D228463946312200F057FBC0B20228AE
:105B0000FFF468AF09990098A02701440C98084455
:105B100000B204900398002870D004980028FBD0AD
:105B2000E88A7080688BF0800A9840B1A98A01EBFE
:105B300008003080ABF101010844B08007E0298BF8
:105B4000A1EB0900B080A0EB0B00401C3080DDE928
:105B50000001411A0898091A0598081A0099099035
:105B60004843049990FBF1F000B2039000200AF042
:105B7000B1F900EB8001502000EB4100B0F5A07FAF
:105B80000ADB00200AF0A6F900EB8001502000EBB0
:105B9000410090FBF7F000E001200399884201DA10
:105BA000084616E000200AF095F900EB800150202D
:105BB00000EB4100B0F5A07F0ADB00200AF08AF973
:105BC00000EB8001502000EB410090FBF7F000E07B
:105BD0000120099900B2091A0AB2009B0499C91A56
:105BE00009B200290BDCE98A019808447080698BAE
:105BF0000898091A0598081A401EF08090E00C9B3E
:105C000012FB03F393FBF1F1511A019AEB8A114451
:105C1000194409B2401E71800844F080B5F916207D
:105C200001981044814238DA708000200AF052F95D
:105C300000EB8001502000EB4100B0F5A07F0ADBB3
:105C400000200AF047F900EB8001502000EB4100F2
:105C500090FBF7F000E00120B6F902100844B6F915
:105C60000610884219DD00200AF034F900EB8001AB
:105C7000502000EB4100B0F5A07F0ADB00200AF0C5
:105C800029F900EB8001502000EB410090FBF7F078
:105C900000E0012071880844F080B5F91A200598C9
:105CA000B6F90610121A0898101A814238DDF080F1
:105CB00000200AF00FF900EB8001502000EB4100BA
:105CC000B0F5A07F0ADB00200AF004F900EB8001A8
:105CD000502000EB410090FBF7F000E00120B6F906
:105CE0000610081AB6F90210884219DA00200AF0E4
:105CF000F1F800EB8001502000EB4100B0F5A07FEF
:105D00000ADB00200AF0E6F800EB8001502000EBEF
:105D1000410090FBF7F000E00120F188081A708044
:105D2000DDE9060101440B98084400B20590029891
:105D300000283FF44FAE05980028FAD0698B0898E8
:105D4000081AE080A0EB0B00401C6080A88A20802D
:105D5000288BA0800698A0EB0801A1EB0901A1EB1C
:105D60000A00019006994843059990FBF1F000B2B2
:105D7000009000200AF0AEF800EB8000502606EB01
:105D800040004FF4A07B584509DB00200AF0A2F840
:105D900000EB800006EB400090FBF7F000E00120F4
:105DA0000099884201DA084613E000200AF092F8D0
:105DB00000EB800006EB4000584509DB00200AF0AC
:105DC00089F800EB800006EB400090FBF7F000E064
:105DD0000120019900B2091A0AB2DDE90513C91AB6
:105DE00009B2002916DCA98A0A9840B14144AAF1F7
:105DF000010008442080298BA1EB090008E001EB99
:105E000008002080298BA1EB0901A1EB0A00401EAC
:105E1000A080DFE50B9B12FB03F393FBF1F1511A1A
:105E20000A9A09B2EAB3AA8A401E531808EB0A027A
:105E3000991809B221800844A080B5F914001044D3
:105E4000884233DD208000200AF044F800EB800017
:105E500006EB4000584509DB00200AF03BF800EB58
:105E6000800006EB400090FBF7F000E00120B4F961
:105E700000100844B4F90410884217DD00200AF02D
:105E800029F800EB800006EB400058450ADB0020B3
:105E90000AF020F800EB800006EB400090FBF7F0E2
:105EA00001E039E0012021880844A080B4F9041001
:105EB000B5F9182077E0A08000200AF00BF800EB7D
:105EC000800006EB40005D46A84272DB00200AF02D
:105ED00001F800EB800006EB400090FBF7F0B4F90E
:105EE0000410081AB4F90010884292DA002009F070
:105EF000F1FF00EB800006EB4000A8425BDB0020D6
:105F000009F0E8FF00EB800006EB400090FBF7F0A3
:105F1000A188081A20805DE5AB8A4144194409B282
:105F2000401E21800844A080B5F9142002EB08002F
:105F3000814232DA2080002009F0CCFF00EB8000A3
:105F400006EB4000584509DB002009F0C3FF00EBD9
:105F5000800006EB400090FBF7F000E00120B4F970
:105F600000100844B4F90410884216DD002009F03E
:105F7000B1FF00EB800006EB4000584509DB002034
:105F800009F0A8FF00EB800006EB400090FBF7F063
:105F900000E0012021880844A080B5F91820B4F958
:105FA0000410A2EB0A02A2EB0900814283DC11E596
:105FB000FFE7012093E70120AAE7806818B1007E7F
:105FC00000F00300704703207047000008B5054942
:105FD0006A46496800912C210AF068F8BDF9020070
:105FE00008BD00007C9C010808B505496A4609689F
:105FF00000912C210AF05AF8BDF9000008BD0000FC
:106000007C9C0108008C704710B5092200F0CDF887
:10601000C0B210BD10B5092200F0C7F8C0B210BD63
:1060200010B5162200F0C1F8C0B210BD10B516228E
:1060300000F0BBF8C0B210BD70B50C46054620227A
:1060400000F0B3F8024621462846BDE87040F6F756
:1060500038BA10B5212200F0A8F8C0B210BD10B5B2
:10606000682200F0A2F8C0B210BD10B5342200F0D2
:106070009CF8002800D0012010BD10B5322200F09D
:1060800094F800B210BD10B5322200F08EF800B2C4
:1060900010BD10B5172200F088F8002800D00120AC
:1060A00010BD10B5042200F080F800B210BD10B58C
:1060B0000A2200F07AF880B210BD10B50A2200F072
:1060C00074F880B210BD10B5602200F06EF8C0B256
:1060D00010BD70B50E460546FFF7F5FF02281AD928
:1060E000FF24FD2802D2C0EB0020040A0EB10026D6
:1060F00003E02846FFF7F4FA054655B13146284635
:10610000FFF7E1FF022806D9FD28F2D24443240A12
:10611000EFE7022C01D8002070BDFD2C01D3FF2039
:1061200070BD204670BD10B5372200F03EF8C0B2F9
:1061300010BD10B5382200F038F800B210BD10B50F
:10614000352200F032F800B210BD10B5112200F077
:106150002CF800B210BD10B5112200F026F800B2E4
:1061600010BD10B5122200F020F800B210BD10B51D
:10617000122200F01AF800B210BD10B5132200F080
:1061800014F800B210BD10B5132200F00EF800B2E2
:1061900010BD10B5102200F008F800B210BD10B507
:1061A000102200F002F800B210BD2DE9F8430E46AF
:1061B000074615460121104601F02AFF80460024BB
:1061C00014E06B462A4631463846FAF7A9FD0446E4
:1061D000012824D0B8F1000F0CD0022C02D00EB14F
:1061E000002603E03846FFF77BFA0746002FE8D188
:1061F000012C14D01EB9012D05D0042D03D0284642
:106200000DF010FB0AE038680FE0012D0AD0C18ABA
:1062100051B160B1012D0CD0B0F91600009000987A
:10622000BDE8F883818AF3E700680028EDD10020FB
:10623000F4E7B0F91400F1E710B50B22FFF7B5FF52
:1062400000B210BD10B54122FFF7AFFF00B210BD84
:1062500010B54222FFF7A9FF00B210BD10B54522CC
:10626000FFF7A3FFC0B210BD10B54322FFF79DFF9B
:1062700000B210BD10B54022FFF797FF00B210BD6D
:1062800070B50C4605465522FFF78FFF02462146A2
:106290002846BDE87040F6F714B95722FFF785BFCE
:1062A00010B56A22FFF781FF00B210BD10B5692258
:1062B000FFF77BFF00B210BD10B50122FFF775FF9D
:1062C00000B210BD10B50722FFF76FFF00B210BD7E
:1062D00010B50822FFF769FF00B210BD2DE9FF419C
:1062E00007460888ADF800004888ADF80200088825
:1062F000ADF80400C888ADF806008888ADF808003D
:1063000048880C46ADF80A00A088ADF80C00E0887B
:10631000ADF80E001D4616466946384601F001FDEF
:106320002B463246384601A901F0FBFC2B4632468B
:10633000384602A901F0F5FC2B463246384603A93F
:1063400001F0EFFCBDF90000BDF90430984201DA1C
:10635000054600E01D46BDF90820BDF90C108A4233
:1063600001DA164600E00E46B54203DA984206DB33
:10637000184604E08A4201DA104600E00846208010
:10638000BDF90030BDF904108B4201DD1D4600E06F
:106390000D46BDF90820BDF90C00824201DD16460C
:1063A00000E00646B54205DD8B4201DD184604E0FB
:1063B000084602E0824200DD1046A080BDF90230AE
:1063C000BDF90600834201DA1D4600E00546BDF92D
:1063D0000A10BDF90E20914201DA0E4600E0164681
:1063E000B54203DA834206DA184604E0914201DA44
:1063F000084600E010466080BDF90210BDF9063085
:10640000994201DD0D4600E01D46BDF90A00BDF9C7
:106410000E20904201DD064600E01646B54205DD3D
:10642000994201DD084604E0184602E0904200DC93
:106430001046E08005221146204609F0EDF9BDE83E
:10644000FF811430FBF7C1B970B50546FFF748F975
:10645000040012D0E88AE18A451A2046FFF780FA44
:10646000054400212046FFF794FE2D1A0021204606
:10647000FFF703FE281A00B270BDB5F9160070BD13
:10648000C069814301D00020704701207047C06976
:10649000084000D001207047008C084000D0012047
:1064A00070477FB50D4606460221FFF7E9FF002839
:1064B00020D080213046FFF7EFFFE8B902A930462F
:1064C000FFF725F80022294602A803F02AFE04005F
:1064D00012D04FF480313046FFF7D2FF70B1012067
:1064E0008DF8040000956A461121304609F0DEFD62
:1064F0009DF8040004B070BD0020FBE72046F9E7DA
:10650000F8B514460D4606465022FFF74EFE00B27F
:106510006080002810D0304629465322FFF745FE00
:10652000C0B22073022807D929463046FFF7D1FDB3
:10653000022802D800202073F8BDFD2804D2217B58
:1065400011FB00F0000A2073207B0228F4D95222AC
:1065500029463046FFF729FE024629463046F5F720
:10656000B0FF0090BDF8000020803046294654223C
:10657000FFF71BFEA060304629465122FFF715FEAB
:1065800000B10120617B002D60F382016173D3D0E3
:1065900029463046FFF763FD617B60F301016173BB
:1065A000F8BDF8B514460E4605464622FFF7FDFD38
:1065B000C0B2E072022807D931462846FFF789FDAC
:1065C0000021022801D8E172F8BDFD2804D2E27A48
:1065D00012FB00F0000AE072E07A0228F4D9218070
:1065E0004FF480706080288BA98A4822401A401C92
:1065F00000B200EBD0704010A080688BE98A401A8E
:10660000401C00B200EBD0704010E08028463146BC
:10661000FFF7CBFD10F0FF00A0720DD047223146EE
:106620002846FFF7C2FD024631462846F5F749FFE6
:106630000090BDF800002081002EC5D031462846CC
:10664000FFF70DFD2073F8BDF8B514460D4606465C
:106650005622FFF7AAFDC0B2A076022807D9294624
:106660003046FFF736FD022802D80020A076F8BD9C
:10667000FD2804D2A17E11FB00F0000AA076A07EC6
:106680000228F4D929463046FFF7FAFD0090BDF8FC
:106690000000A081304629465822FFF786FDA082DF
:1066A000304629465922FFF780FD60823046294650
:1066B0005A22FFF77AFDA17F60F30201A1773DB175
:1066C00029463046FFF7CBFCA17F60F3C501A177D7
:1066D00029463046FFF7E1FD2060304629465B221F
:1066E000FFF763FD2077F8BDF8B514460D46064662
:1066F000FFF7EFFC074685B1022F09D80020E070B4
:10670000A07684F8220084F82A0084F83600F8BDC8
:1067100029463046FFF7A3FCA070304629460B22DD
:10672000FFF743FD2080E078002856D03046294608
:106730002122FFF73AFDC0B2E07002284DD9294668
:106740003046FFF779FC0090BDF80000A08030468D
:1067500029462622FFF729FD010007D0487A400785
:1067600004D00A22A01D0BF0A7FF36E030462946D0
:106770002322FFF71AFD0146E07B61F30200E0737C
:10678000400721D029463046FFF756FC0090BDF85F
:106790000000E080222229463046FFF706FD02462F
:1067A00029463046F5F78DFE0090BDF80000608167
:1067B000304629462422FFF7F8FC2072304629464D
:1067C0002522FFF7F2FC2073304629462722FFF7E7
:1067D000ECFCE17B60F3C501E173304629463222CF
:1067E000FFF7E3FC00B2208428B394F8220010B332
:1067F000304629463122FFF7D8FCC0B284F8220087
:10680000022818D9304629463322FFF7CEFC94F8E7
:106810002310302260F3450184F8231029463046C6
:10682000FFF7C3FC024629463046F5F74AFE0090C2
:10683000BDF80000E08329463046FFF780FCE08485
:10684000E8B194F82A00D0B129463046FFF76BFC36
:1068500084F82A00022812D929463046FFF769FC3D
:106860002085362229463046FFF79FFC02462946FE
:106870003046F5F726FE0090BDF80000A084A07E0B
:1068800080B3304629462822FFF78FFC206148B3A9
:10689000304629462922FFF788FCC0B2A07602289C
:1068A00020D92069FDF746FF02286CD02A2229460C
:1068B0003046FFF77AFC024629463046F5F701FEDE
:1068C0000090BDF800002083304629462B22FFF7B8
:1068D0006CFCE076304629462C22FFF766FC00B1BE
:1068E0000120207794F8360070B329463046FFF730
:1068F000C1FCE08540B394F83600022824D929462B
:106900003046FFF7ABFC84F8360002281CD9294634
:106910003046FFF797FC208629463046FFF798FC63
:10692000608629463046FFF79FFCA0864422294610
:106930003046FFF73AFC024629463046F5F7C1FDDE
:106940000090BDF80000A085FD2FBFF4E0AE14F864
:10695000030F10FB07F0000A04F8140BE07810FB9B
:1069600007F0000AE070E07A10FB07F0000AE0721E
:10697000E07C10FB07F0000AE074E07F10FB07F0FA
:10698000000AE077F8BD29463046FFF786FC6061D3
:1069900029463046FFF774FC0090BDF800002083C4
:1069A000A0E77CB50546F5F75CFD044605F114014A
:1069B0006846FAF7B6FEBDF800006946001BADF860
:1069C0000000BDF80200001BADF80200BDF8040095
:1069D0002044ADF80400BDF806002044ADF80600E0
:1069E000284600F001F87CBD7CB50C460546FEF754
:1069F00019FE09F0DDFA00280FD021466846FAF7A3
:106A000090FE69462846FDF7BBFF002805D02846C2
:106A1000FEF708FE6946F5F7B1FC7CBD006800286A
:106A200008D0017E8907F9D0007E00F0030001281C
:106A300000D0002070470068002809D0017E11F0C6
:106A40000C0FF8D0007EC0F38100012800D0002098
:106A50007047000010B504460849FFF718FD08B15B
:106A6000002010BD2046FEF73BFE0028F9D0002193
:106A7000FFF723FB0028F4D0012010BD0100060021
:106A80007CB50546F5F7EDFC044605F114016846B2
:106A9000FAF747FEBDF800006946001BADF800009C
:106AA000BDF80200001BADF80200BDF80400204450
:106AB000ADF80400BDF806002044ADF806002846F5
:106AC000FDF75EFF7CBD10B5418C41F001014184B2
:106AD000FEF70AFE418C41F004014184FEF7A2FD5D
:106AE0004068002803D0BDE8104001F079BB10BD1C
:106AF0002DE9F047994616460F468246FEF702FDFD
:106B00008046002520E0DAF80800B9F1000F00689F
:106B100050F8254005D04FF480212046FFF7B0FC07
:106B200088B9A08A00233844A082E08A32463044E3
:106B3000E082208B394638442083608B3044608368
:106B40002046FFF7D5FF6D1C4545DCD3BDE8F08737
:106B50002DE9FF47456816460F4604469DB30021C0
:106B60002846FFF7FEFA804600212846FFF711FB72
:106B700081464FF480212046FFF782FC48B1A98A64
:106B800007EB0800084407B2E98A06EB090008444D
:106B900010E02846FEF7DDFEAA8A02EB0801081A7B
:106BA000384407B22846FEF7DBFEEA8A02EB090109
:106BB000081A304406B200212846FFF75EFA391859
:106BC00030440FB206B2A08A381A07B2E08A301AEF
:106BD00006B20FB9002E43D02046FFF7E2FE02A90D
:106BE0002046FEF719FD4FF0000875B169462846AA
:106BF000FEF7ACFC0022694602A803F0D2F95FEA76
:106C0000000802D1284600F01FFEA08A3246384410
:106C1000A082E08A39463044E082208B0023384449
:106C20002083608B304460832046FFF761FF25B1ED
:106C300022462221284609F039FA2046FFF7B1FE04
:106C4000002D0DD00022694604F1140003F0A9F9CB
:106C5000B8F1000F01D1002802D0284600F0F4FD61
:106C6000BDE8FF872DE9F0410E460746FEF763FEBB
:106C7000A0B93846FEF766FE04463846FEF73CFDEE
:106C800000280BDA002C09DD4042844200DB044678
:106C900022B233460021384600F088FC3846FEF721
:106CA00043FE002825D13846FEF780FD04463846CD
:106CB000FEF7DCFD054600213846FFF7B7F901284D
:106CC0000BD0002D15DA002C13DD6842844200DB66
:106CD000044621B23346002206E0002C09DA002DDA
:106CE00007DD3346002221463846BDE8F04100F07A
:106CF0005DBCBDE8F0812DE9F0470E4686B0054643
:106D0000876802A93046FEF787FC3046F5F7A9FBF5
:106D10000146024602A808F07FFD02AA394604A8EF
:106D200003F017F94FF4002420B921463046FFF74D
:106D3000A7FB00B101205FEA00090DF1100A10D095
:106D40002A4614213046C5F808A009F0AFF92A46B2
:106D50001521304609F0AAF92A461621304609F0D5
:106D6000A5F921463046FFF78BFB20B1386800902B
:106D70007868019006E006F114023946684603F08F
:106D8000E8F888B1C5F808D03046FEF7BBFB80466E
:106D9000002407E0B068006850F82410284601F08D
:106DA00047FF641C4445F5D3B9F1000F10D02A46C3
:106DB00017213046C5F808A009F078F92A461821AD
:106DC000304609F073F92A461921304609F06EF968
:106DD000AF6006B0BDE8F0872DE9F14F82B00298B0
:106DE000FFF738FE00287CD10298FEF779FC00906E
:106DF00000210298FFF766FA834600210298FFF708
:106E000067FA0546009858B1FEF7EAFB81460098FC
:106E1000FEF7CAFB0746CBF34130012803D013E04D
:106E20002A4659469AE02BF4C040B0F5FA6F0BDCC5
:106E3000B0F57A7F01DDC0F57A7000FB09F06421BE
:106E400090FBF1F00FFA80FBC5F3413001280ED121
:106E500025F4C040B0F5FA6F09DCB0F57A7F01DDAA
:106E6000C0F57A707843642190FBF1F005B20021FF
:106E70006B220298FFF799F904B200216C22029864
:106E8000FFF793F90FFA80FA0298FFF7DAFA8046D3
:106E90000298FEF7EAFB0646C4F3413001280FD101
:106EA00024F4C040B0F5FA6F0ADCB0F57A7F01DD5A
:106EB000C0F57A7000FB08F0642190FBF1F004B299
:106EC000CAF34130012811D12AF4C040B0F5FA6F5D
:106ED0000CDCB0F57A7F01DDC0F57A707043642177
:106EE00000E05BE090FBF1F00FFA80FA0BEB04009E
:106EF00004B205EB0A0005B200210298FFF78AF8F8
:106F000050B1012828D0801E082825D2DFE800F0E3
:106F10000C14212C3419393C00210098FFF780F81B
:106F2000012819D10320EEE709EBD970401008EBD6
:106F3000D871A0EB610001E0A9EB0800204404B285
:106F40000AE007EBD770401006EBD671A0EB6100AA
:106F500000E0B81B284405B22A462146029803B037
:106F6000BDE8F04FFFF7F4BD09EBD970401008EB16
:106F7000D871A0EB610001E0A9EB0800204404B245
:106F8000E7E7A9EB080006E009EBD970401008EB31
:106F9000D871A0EB6100204404B2D2E7BDE8FE8FB7
:106FA0002DE9F04F0446408C87B0010501D540051E
:106FB0007ED42046FEF794FB5FEA000878D0204696
:106FC000FEF7F4FB0590608C002600054FF4FA6B89
:106FD00042F2D17A03D52046FFF733FA5DE0002173
:106FE0002046FFF769F90546504501D1012600E02A
:106FF0000026C5F34130012805D125F4C04058458D
:1070000001DC012000E0002081464046FEF7E8FA5E
:10701000074626B12046F5F72BFF05462BE0B9F1D0
:10702000000F28D0B8F82200000518D400214046EF
:10703000FFF742F9504512D100212046FFF71DF815
:10704000054600212046FFF78CF800EB05090021DA
:107050002046FFF792F8411901EB09000AE025F4F8
:10706000C040B0F57A7F01DDC0F57A7078436421C5
:1070700090FBF1F005B2204600210222FFF795F8BF
:107080000FFA80F9204600210322FFF78EF802B2A2
:107090003B4649462846FAF7F7FB07462046FEF7E7
:1070A00051FC0490608C4FF00009400505D500E0CC
:1070B0006BE02046FEF7D9FA53E000212046FEF7A8
:1070C000F0FFA0F51C510546D13906D000208146BD
:1070D000C5F34130012802D007E00120F7E725F48D
:1070E000C040584501DC012000E0002083464046B6
:1070F000FEF75AFA8246B9F1000F04D02046F5F7A0
:1071000043FE05461BE0BBF1000F18D0B8F8220083
:10711000400507D400214046FEF7C3FFA0F51C51EF
:10712000D13936D025F4C040B0F57A7F01DDC0F505
:107130007A7000FB0AF0642190FBF1F005B2204662
:1071400000210522FFF731F80FFA80FB20460021CD
:107150000622FFF72AF802B2534659462846FAF7A4
:107160005EFB054656EA090605D0DDE90421002349
:10717000204600F012FB2046FFF763F9B8421BD10E
:107180002046FEF772FAA84216D1002007B0BDE8EB
:10719000F08F00212046FEF770FF054600212046B3
:1071A000FEF7F7FF00EB050B00212046FEF7CDFFB1
:1071B000411901EB0B00C1E72046FFF7F2FB6946DE
:1071C0002046FEF729FA02A94046FEF7BFF9002241
:1071D00002A9684602F0E5FE060002D1404600F032
:1071E00033FBE08A6D1E2844608300212046FEF7B1
:1071F00017FF01281CD0A08A7F1E384420836A46CE
:107200002921204608F052FF22462221404608F05C
:107210004DFF2046FFF7C5FB608C002240F00200C6
:10722000608402A904F1140002F0BBFE36B904E048
:10723000208BC01B401CA082E1E710B1404600F04B
:1072400003FB204600F002F801209FE738B5054611
:10725000F5F707F904460020ADF800006A4613214F
:10726000284608F023FFBDF90000A04202D02846BE
:10727000FFF797FBBDF80000A96831B930B1284687
:10728000FDF760FBBDF80000A968C882BDF90000E9
:10729000A04202D02846FFF784FB38BD70B50546F2
:1072A0000021FFF709F8044600212846FEF7F9FE01
:1072B00042F2D1718C4203D0884201D0002070BDCF
:1072C0002846FFF700FC012070BD00002DE9F84FB3
:1072D0000646514890460C460078002870D030464B
:1072E000FFF75FFB04F47F040421404600F090FEAA
:1072F00007460221404600F08BFE814601214046B0
:1073000000F086FE00901021404600F081FE054608
:107310004FF6FF7BEFB1B4F5702F12D08CB1304631
:1073200000210422FEF741FF00B242F2D17A50451B
:1073300007D0304600210122FEF737FF00B250454A
:107340004DD100222A21304608F0B0FE3046FFF72A
:10735000BAFB4FF4702A544500D084BBD84500D006
:107360002FB13046FEF7BCF908B1FFF7ACFB54452E
:1073700000D024BB1DB3304600216E22FEF715FF5E
:1073800000B240B9304600216D22FEF70EFF00B278
:10739000B0F5807F01D0022514E030460021612243
:1073A000FEF703FFC0B2FF2807D130460021682254
:1073B000FEF7FBFE10F0FF0F03D0012502E00EE008
:1073C00028E00025B06820B1817E65F387118176C1
:1073D00005E025B13046FDF7B5FAB068F4E75D4643
:1073E000A84502D0B9F1000F02D03046FFF72EFFBA
:1073F0003046FFF7D6FAA84504D0009949EA0700BD
:10740000084207D0B4F5803F04D03046BDE8F84FBD
:1074100001F0F4BDBDE8F88FBC3400202DE9F04147
:1074200004460E46408C154600210423C0F3051285
:107430000AE0E06803EBC107C059C70103D520F09B
:107440007F40A84202D0491C8A42F2D88A4202D127
:107450000020BDE8F081E06850F8310031460CF0C2
:107460007BFA28B1324629462046FFF72FFF01E07C
:107470000028EED00120ECE72DE9F05F0E00044675
:107480001FFA82F802F47F074FF6FF7B03D0F079F2
:1074900008B94FF0000B00252B4658E0E0680421A6
:1074A00001EBC50A814650F80A004FF6FF7281B21F
:1074B00000F47F0C904501D0414509D1B7F5702FFC
:1074C00001D0BC4504D12EB159F83510B14201D0DC
:1074D0006D1C3CE0800104D500233946204602F0B3
:1074E000A3FAE06850F80A10CA0101D489010CD54A
:1074F00050F835000CF090FAE06850F835000BF0C9
:107500009FF8E168002041F83500284608230AE08A
:10751000E16803EBC00C01EBC0026144401CD1E9FF
:1075200000C1C2E900C1618CC1F30511491E81424D
:10753000EED8608C0109491E61F309106084C0F324
:107540000510C100E0680BF09FF80123E060608C3B
:10755000C0F30510A842A1D8002B09D0BBF1000050
:1075600006D0024639462046BDE8F05FFFF7AEBEC2
:10757000BDE8F09F70B506460B480078002812D091
:1075800000200CE0002406E0E86850F824103046A3
:1075900001F053FD641C686AA042F5D8284608F043
:1075A000D1FC0500EED170BDBC340020F0B515460D
:1075B000064691B00C4651EA050072D0012B1DD051
:1075C00039493046F9F794FF38493046F9F790FFCA
:1075D00000220921304608F069FD012861D12A46C0
:1075E00021463046F4F749FF01285AD111B0304600
:1075F000BDE8F04000220A2108F058BD3046FEF7F1
:1076000011F807466846F9F7BBFF29480096039032
:1076100014B3384608F070FC401022460021FAF7F7
:107620002CF8642801D04FF064000B903046FEF730
:1076300090F94142201A0891CDE909101B480190A8
:107640001C4807906A460921304608F02FFD0128A2
:1076500027D16846FAF71EF8002D22D0384608F0E8
:1076600091FC40102A460021FAF707F8642801D05F
:107670004FF064000B903046FEF772F94142281A31
:107680000891CDE90910084801900A4807906A4618
:107690000921304608F00AFD012802D16846F9F7B1
:1076A000F9FF11B0F0BD0000CD930108B5930108BA
:1076B0001F910108E91501082DE9F047154682469A
:1076C00099460C4651EA050065D0504600F058FB3B
:1076D0005046FEF73EF940420FFA80F808EB0400EE
:1076E00004B200215046FEF7A1FC012813D0002C63
:1076F00013DC25DA5046FEF759F806465046FEF7E9
:10770000B5F8304400B2002800DA0020404284423C
:1077100016DA04B214E0002C02DA4FF000040FE095
:107720000EDD5046FEF742F806465046FEF79EF83C
:10773000304400B2002800DA0020844200DD044614
:107740005046FEF70DF9404206B2701905B2002D01
:1077500002DD4FF0000510E00FDA5046FEF7F2F8B8
:1077600007465046FDF7C8FF384400B2002800DA4B
:1077700000204042854200DA05B2A4EB080001B2C5
:10778000A81B02B251EA020005D04B465046BDE8A4
:10779000F047FFF70BBFBDE8F08770B516461D46F2
:1077A00004461A4600F024F82A4631462046BDE831
:1077B000704000F033B8F8B50F46054600F0E0FA27
:1077C000002000902846FDF78BFF044605F11406C3
:1077D0000AE03B466A462946304601F0A5FC2546AC
:1077E0002846FDF77DFF0446002CF2D1F8BD0000CD
:1077F00070B50E46144605460749F9F779FE284646
:10780000FEF7A7F8801B01B223462846BDE870406A
:107810000022FFF751BF0000B593010870B50E4676
:10782000144605460749F9F763FE2846FEF798F81F
:10783000801B02B223462846BDE870400021FFF7B6
:107840003BBF0000CD9301081FB5044602AA69465C
:10785000FEF78DF8684607F0B9FF20B902A807F0D7
:10786000B5FF002810D0684607F0B0FF18B1694690
:107870002046FFF7B9F802A807F0A8FF002803D0B8
:1078800002A92046FFF7B0F81FBD002200F02BB977
:1078900070B50C460546FDF755F8A868848270BDA2
:1078A00038B50C46054600236A460421FDF7F9FE6B
:1078B000012807D0002804D100222146284600F0E4
:1078C00063F938BD0098A042F6D138BD2DE9F041EA
:1078D0000C4615461F4606461946F9F786F92A460C
:1078E00021460CF043F9224639463046BDE8F041C6
:1078F000FFF7ECBC70B51546044600F0E1F92946E7
:107900002046BDE8704000F0F1B970B50C46054660
:10791000FDF718F8A868417E01F00F01A14200D0E0
:10792000447670BD70B50C460546FDF70BF8AB68A4
:107930001A7E02F00300A04207D064F301021A7617
:107940002846BDE87040FFF72CB870BD2DE9F34F15
:1079500089B08346008C0A9988427DD00390ABF8A9
:10796000201058460A9A0399F4F76CFE02900028FA
:1079700072D04FF4207420460AF004FE804621465F
:107980000AF069FF002420466BE0DBF80C000422BB
:1079900002EBC90500EBC90A405920F07F4000F016
:1079A000BEF90190DBF80C00405920F07F4000F058
:1079B000B3F907900A990198884350D1DAF8040086
:1079C00080014CD405AA6721DAF8000000F0D0FA53
:1079D000012844D10027059D39E000261BE006EB75
:1079E000860108EB810106914868049000F097F940
:1079F0000090049800F090F9296831F81720069952
:107A000009898A4206D10799884203D1DDE900013C
:107A1000884202D2761CA642E1D3A64216D104EBDC
:107A20008400A98928F8201008EB8000298A418069
:107A3000A968C1602968641C31F817100181696860
:107A40000161DAF8041021F07F4141607F1C286851
:107A500030F8170018B100E042E0202CBDD309F146
:107A600001008146BBF82200C0F30511494501D948
:107A7000202C8AD300250EE005EB850108EB81065A
:107A8000706800F049F90146009658460A9B039A2F
:107A9000F4F738FD6D1CA542EED340460AF0BEFD5A
:107AA000029801280CD0032810D0022818D158467B
:107AB000FEF777FF0BB05846BDE8F04FFFF7C6BBA7
:107AC0000BB05846BDE8F04FFEF76BBF0BB0584601
:107AD000BDE8F04F4FF6FF724FF47021FFF7F6BB91
:107AE0000BB0BDE8F08F13460A460921FFF7EEBE42
:107AF00013460A466621FFF7E9BE13460A4665218A
:107B0000FFF7E4BE07B481B01346BDF80810ADF826
:107B10000010009A522104B0FFF7D8BE13460A465F
:107B20005321FFF7D3BE13460A465121FFF7CEBEBD
:107B300013460A465021FFF7C9BE07B481B0134669
:107B4000BDF80810ADF80010009A202104B0FFF72E
:107B5000BDBE13460A462121FFF7B8BE07B481B067
:107B60001346BDF80810ADF80010009A302104B09B
:107B7000FFF7ACBE13460A463121FFF7A7BE1346F6
:107B80000A463221FFF7A2BE13460A460421FFF738
:107B90009DBE13460A460A21FFF798BE13460A46C1
:107BA0006021FFF793BE07B481B01346BDF80810FB
:107BB000ADF80010009A362104B0FFF787BE1346D7
:107BC0000A463721FFF782BE13460A463821FFF7DF
:107BD0007DBE13460A463521FFF778BE13460A4696
:107BE0001121FFF773BE13460A461521FFF76EBE3B
:107BF00013460A461221FFF769BE13460A461321AF
:107C0000FFF764BE13460A461421FFF75FBE134612
:107C10000A461021FFF75ABE13460A460B21FFF70A
:107C200055BE13460A464321FFF750BE13460A4687
:107C30004021FFF74BBE13460A465B21FFF746BEC5
:107C400007B481B01346BDF80810ADF80010009AD3
:107C5000552104B0FFF73ABE13460A465721FFF7F5
:107C600035BE13460A465621FFF730BE13460A4674
:107C70006E21FFF72BBE13460A460121FFF726BEF1
:107C800013460A460721FFF721BE13460A4608217C
:107C9000FFF71CBE38B50C46054600236A46012195
:107CA000FDF7FFFC012807D0002804D1002221465F
:107CB0002846FFF7E0FF38BD0098A042F6D138BD56
:107CC00038B50C46054600236A460721FDF7E9FC56
:107CD000012807D0002804D1002221462846FFF7BA
:107CE000CFFF38BD0098A042F6D138BD38B50C465C
:107CF000054600236A460821FDF7D3FC012807D07A
:107D0000002804D1002221462846FFF7BEFF38BDD7
:107D10000098A042F6D138BD00F47F00704780B2D1
:107D200070472DE9F0411E4615468846070025D0CC
:107D3000F4F79DFB022813D000249EB13DB13846D4
:107D4000FDF7CEFC33462A464146FFF7EAFF002CFA
:107D500014D0324641463846BDE8F04101F0B8BE85
:107D60000124EAE724B132464146384601F0B0FE2C
:107D7000002D03D03846FDF7B3FCD7E7BDE8F0810E
:107D800070B50B4D2978002910D101212970FDF71C
:107D9000ABFC044605E021F0040060842046F9F7BE
:107DA000D5F9618C4807F6D40020287070BD00001A
:107DB000B434002010B51BF021FB0D4A4FF448638A
:107DC000A2F5C851A1F11C0007F08DFF094807F08A
:107DD00099FF08484FF4A0710180AA21418006490B
:107DE00041610649C160BDE8104007F0B5BF000021
:107DF0002C6200202C7B002011D8000810490020A4
:107E000010B50A4809F0EEFC084802210170084943
:107E1000416009F0FBFC074C606008F083FC014600
:107E2000A0606068BDE8104009F05BBE7C7B00206C
:107E3000A50F0108883400202DE9FC410E460025DD
:107E400007462A46143102F0ACF8002826D001215A
:107E50003046FEF715FB00BB3046F4F708FBE0B9EF
:107E600000208DF800006A4612213046019708F084
:107E70001DF99DF8000002280FD03046FDF742FBA7
:107E8000401E04000ED4B068006850F82410384634
:107E9000FFF7D2FF050009D102E00020BDE8FC8118
:107EA000641EF0D59DF8000000B935462846F5E778
:107EB0002DE9FC410025DFF8B4804FE0284490F81C
:107EC0003001E8BB002441E0011991F83011C1BB39
:107ED000A5423AD000EBC40100EBC5003030303190
:107EE00002F0B3F868B37068B04600EBC40200EB70
:107EF000C50168463031303202F0A7F9684607F014
:107F000065FC0646D8F8040000EBC500303007F0E9
:107F10005DFC0746D8F8040000EBC400303007F0E1
:107F200055FC3844864210D2D8F80400464600EB8F
:107F3000C50069463030F9F7FDFB0120716801E0AA
:107F40000BE002E0214481F83001641CD8F8040001
:107F50004646B0F85011A142B6D86D1CD8F80400BE
:107F6000B0F85021AA42A9D8BDE8FC81C034002055
:107F700070B515468288C479A2F57F43FF3B07D0D0
:107F80008CB3012C34D90668002306EB84022CE064
:107F9000002313E0026802EBC302168826F4404671
:107FA0008E420AD11088010428D4400401D53046FD
:107FB00013E050682860012070BD5B1C9C42E9D82A
:107FC00024E032F8130020F4404088420CD132F80B
:107FD00013100A0412D4490402D50BF023FCE9E77C
:107FE00006EB830010E011E05B1C9C42E9D80DE039
:107FF00022F440438B4209D1110401D5022070BD07
:10800000510401D51846E8E70068D3E7002070BDA9
:1080100010B50C4602F036FD204000D0012010BD06
:108020002DE9F041074615460E460B4802F079FC53
:10803000040010D0A7604FF0FF30266020610020C0
:1080400060610BF0BFFFE5600449606001200871CA
:108050002046BDE8F081FEE7F07C00208C35002052
:1080600010B504460146054802F0D1FC044B01223C
:108070002046DA70BDE810400AF0E2BAF07C002039
:108080008C3500202DE9F047494CA07810B1012033
:10809000BDE8F0870120A0702078002528B10BF002
:1080A00091FF5FEA000A02D007E0A570EFE72069C0
:1080B000401C2061642800D925613E4FA946A04696
:1080C0003D4888F8039088F8049002F005FC386079
:1080D00033E0394802F012FC3C680646207DC007B8
:1080E0002AD10025204600F07EF868B92569002DC8
:1080F00001DD681E20610BF065FF6060A16811B1B1
:108100000DB120468847012598F8030020B9206961
:1081100010B92046FFF7A4FF75B198F8041098F83D
:108120000300014308D038680028C9D14FF0FF355B
:10813000214802F0D1FB11E03E6039680029C8D126
:10814000F4E7207DC00705D1204600F04CF8A84296
:1081500000D205462146184802F0D0FB0400F0D1B9
:1081600050460BF028FFD8F80C1044460844C8F8D5
:108170000C00D8F808000BF01EFFB0F5FA7F13D3FF
:10818000E16864225143B1FBF0F0C0B26070642832
:1081900001D9002001E0C0F1640060702646C4F8F7
:1081A0000C900BF00FFFB06084F8029028466FE748
:1081B0008C35002060350020F07C002001214161D9
:1081C000704710B504460BF0FDFE2168401A401EB2
:1081D000606010BD10B504460BF0F4FE606010BD89
:1081E00000214161704710B5044640680BF0E3FE82
:1081F0002168814201D8002010BD081A10BD00007E
:108200002DE9FF4F85B00546DDE913981E460F4660
:108210000846169CF9F7EBFA03903846F9F7C3FACB
:108220000290012C13D0022C13D0032C4CD14E4FB2
:108230002888ADF800003088B8F1000FADF80400D0
:1082400009D098F80000FD2841D3484642E0474F46
:10825000EEE7474FECE7DDE900104A46B8470490E7
:1082600000202DE0002420E0BDF8040036F81410B2
:10827000884205D1BDF8000035F8141088420ED0B0
:1082800005EB44004A460088ADF8000006EB4400C8
:108290000088ADF80400DDE90010B847049005EB54
:1082A0004400BDF810100180641C03988442DBDB9D
:1082B000079805EB4005129806EB400608F101000F
:1082C000029980468842CDDB09B0BDE8F08F00FB03
:1082D00009F0000A82460246DDE90010B847049022
:1082E00000203CE000242DE018F8040048B3FD28ED
:1082F00001D3484602E000FB09F0000ABDF8041073
:1083000036F81420914207D1BDF8001035F814203A
:10831000914201D182450FD005EB44018246098884
:10832000ADF8001006EB440102460988ADF80410D0
:10833000DDE90010B847049005EB4400BDF81010CB
:108340000180641C03988442CEDB0798159905EBE5
:1083500040051298884406EB40060BF10100029993
:1083600083468842BEDBAFE77BD30008F9D2000822
:10837000FFD300082DE9FF4F85B00646DDE91379EC
:108380001D460C460846F9F732FA80462046F9F7B2
:108390000AFA8346B9F1000F06D0FD2F7ED9A8F165
:1083A0000400049000201DE1FD2F14D300244FEAA7
:1083B00048070BE03A46294630460AF07DF907980F
:1083C000641C06EB4006129805EB40055C45F1DBAA
:1083D00009B0BDE8F08F002021E0002415E006EB95
:1083E000440A3A46BAF80000ADF8000005EB440034
:1083F0000088ADF80400DDE90010F9F7D9FA009023
:10840000BDF80010AAF80010641C4445E7DB07988B
:1084100006EB4006129805EB400509F10100814684
:108420005845DADBD4E74F46002419E03A78AAB180
:10843000FF2A06EB440018D082460088ADF8000001
:1084400005EB44000088ADF80400DDE90010F9F701
:10845000AFFA0090BDF80010AAF80010641C7F1C51
:10846000444575DAB807E1D172E005EB44010988AB
:108470000180F3E73868E8B3401C6DD03A78BAB1B0
:10848000FF2A06EB440075D082460088ADF8000054
:1084900005EB44000088ADF8040000E0ACE0DDE945
:1084A0000010F9F785FA0090BDF80010AAF8001046
:1084B0007A7807F1010AAAB1FF2A06EB44005ED0E0
:1084C00000904088ADF8040005EB44004088ADF80A
:1084D0000800DDE90110F9F76BFA0190BDF804100E
:1084E000009841801AF8012FBAB1FF2A06EB440028
:1084F00049D000E02AE000908088ADF8040005EB48
:1085000044008088ADF80800DDE90110F9F750FA61
:108510000190BDF80410009881809AF80120AAB15A
:10852000FF2A06EB440032D08246C088ADF8000036
:1085300005EB4400C088ADF80400DDE90010F9F750
:1085400037FA0090BDF80010AAF80610241D3F1D50
:10855000049884428EDB39E005EB440006EB4401CD
:1085600002880A8042884A8082888A80C088C880BF
:10857000ECE7FFE705EB44010988018098E705EB8C
:1085800044014988ADE705EB44018988C4E705EB60
:108590004401C988C180D9E73A78AAB1FF2A06EB1D
:1085A000440024D082460088ADF8000005EB44006A
:1085B0000088ADF80400DDE90010F9F7F9F9009042
:1085C000BDF80010AAF80010641C7F1C4445E3DBD2
:1085D000079806EB4006129805EB40051598814474
:1085E0000398401C03905845FFF61DAFF0E605EBDD
:1085F000440109880180E7E700202BE000241DE00A
:1086000019F80400C8B1FD2801D33A4601E07843C7
:10861000020A06EB440000900088ADF8040005EB68
:1086200044000088ADF80800DDE90110F9F7C0F951
:1086300001900098BDF804100180641C4445DFDB04
:108640000798159906EB40061298894405EB4005FA
:108650000AF1010082465845D0DBB9E62DE9FF4F0B
:1086600085B01D46DDE913B80E46F4F7E1F8824601
:108670003046F9F7BCF881463046F9F794F8039094
:10868000B8F1000F4FF000071ED048E0002415E0BD
:1086900005EB4400CDF808B00088ADF80400708800
:1086A000079A384400B2009030880599204403B2FC
:1086B000DAF80000D0F81CC0E047641C4C45E7DB4A
:1086C00012987F1C05EB400503988742DEDB09B05A
:1086D000BDE8F08F00241AE018F80400B0B100FBE8
:1086E0000BF0000A029005EB4400079A0088ADF8F1
:1086F00004007088384400B2009030880599204406
:1087000003B2DAF80000D0F81CC0E047641C4C4506
:10871000E2DB15991298884405EB40057F1C03980D
:108720008742D7DBD3E7FD2902D2022901D80020F6
:10873000704710FB01F000EBC01101EBC030C0F33B
:10874000C750704770B5094D04466868002808D0C6
:1087500044B12046F8F740FAA9682044884200D383
:10876000002070BD0248006870BD0000C8340020C1
:108770006C3500202DE9F04104460022212107F04C
:1087800095FC00287ED0608C40F48050608401E02D
:10879000FFF7F0FF00212046FCF7A2FE0028F7D1EA
:1087A0002046FCF75DFF0646002009F059F8054613
:1087B00000271CE0A86AA04202D0E86AA04203D1C8
:1087C0002146284609F0F4F8686BA04200D16F6397
:1087D000686DB04207D109F04DF8A04203D121469F
:1087E000284609F0E5F8284609F03AF80546002D34
:1087F000E0D12046F3F727FE6068042600282046D3
:1088000002D0FCF735FF29E0FCF70CFF0546416A72
:108810000022C06804E050F82230A3420AD0521C63
:108820009142F8D806E0E86806EB8201415840F82A
:108830002210521C686A401E9042F4D8686A401E9A
:1088400081006862E86809F01FFFE8601EE00968BF
:1088500006EB80028A5841F82020401C6168896834
:108860004A68521E8242F2D8606880684068401EA2
:1088700048606168800089680A680146104609F00E
:1088800003FF00E007E06168896808602046BDE8F2
:10889000F04109F0D5BEBDE8F08100002DE9F04FB0
:1088A000524F064685B078680168CC6BC968896804
:1088B0002160016809698A0701D4C90723D007F03C
:1088C00061FB401E05B2786807F016FB401E03B23C
:1088D0000022114603A8009506F0B8FF03A96160C5
:1088E00078680068027CC068920705D5826942F00A
:1088F00002028261A16073E08169826961F34102D1
:108900008261A6606CE03046F8F765FF814630462C
:10891000F8F743FF8046786807F034FB0146B6F964
:108920000600814203DC786807F02CFB401E05B28C
:1089300042464946BA467868F8F7BEF981460027AC
:10894000B6F902000DF1040B28E03288ADF80420DE
:10895000B288ADF80820ADF80600ADF80A10C4F8EA
:1089600004B0C4F808B0DAF804000168C96889687E
:108970002160BDF90A10A94201DDADF80A50BDF928
:108980000A70BD4205D10068C068816941F00201EA
:108990008161204600F02CF80FFA88F000EB0908FE
:1089A000A8F10101A942D0DDBD421CD03188ADF84B
:1089B0000410B188ADF80810ADF80600ADF80A5003
:1089C000C4F804B0C4F808B0DAF804000168C96853
:1089D000896821600068C068816941F00201816195
:1089E000204600F005F805B0BDE8F08FC034002047
:1089F0002DE9F0415F4F064690B0786807F078FAAD
:108A0000F168044609B130468847786800680188F3
:108A1000408811FB00F0E168884201D1012000E0AC
:108A20000020216859B1616831B128B907E0786840
:108A30000068816A01B1884720690028F7D10024C5
:108A4000786807F089FA01467068FFF7F5F905467E
:108A50007868416919B17068FFF7EEF9044655EA84
:108A6000040051D1786807F08DFA401E0FFA80F8A3
:108A7000786807F041FA401E03B2002211460EA8A2
:108A8000CDF8008006F0E2FE306BB0B16846FAF730
:108A9000D5FA78680EAAC16A049190F829108DF869
:108AA0001A10418DADF8041090F829008DF80300DC
:108AB000336B69463046984726E07868C06A98B1BB
:108AC00006A908F01BFC01281ED16846F9F72AFA0E
:108AD00078680EAA90F829108DF80B10C36A6946C1
:108AE0003046F9F7EBF90FE06846FAF7A7FA78682D
:108AF000418DADF8041090F829008DF80300694607
:108B000030467268FAF786FA786890F82810C90734
:108B10000CD005B905693046294600F09FF9786800
:108B2000406990B104B9044621460BE0406928B180
:108B300004B904462146304600F090F90DB9786832
:108B400005692946304600F089F9786807F0F2F99E
:108B50000146304600F082F9786807F0E3F90146F3
:108B6000304600F07BF9786810B0BDE8F041F5F7C9
:108B700081BC0000C03400202DE9F0412B4F0020C3
:108B800038607868B0F85051002D4DD0002603E0D1
:108B9000411991F83011D1B16D1EF9D50068416BC2
:108BA00001B1884778680168C9688A6922F00102C2
:108BB0008A610168C9688A6922F002028A6190F8B4
:108BC0002810002441F0040180F8281022E02E46ED
:108BD000E4E7011991F83011D9B9B44205D101681F
:108BE000C9688A6942F001028A610168C9688A69B4
:108BF00022F002028A6100EBC4003030FFF74EFE23
:108C0000786800EBC400303006F0E0FD39680844B5
:108C10003860641C7868B0F85011A142D9DC10F8B3
:108C2000281F21F004010170BDE8F081C03400204C
:108C30002DE9F04F0D4680468BB001212846FDF707
:108C40001FFC00287ED12846F3F711FC040028D031
:108C5000284600216122FDF7A8FA00F0FF0BBBF1C6
:108C6000020F6FD306AB224629464046F8F725FA95
:108C7000012867D105F114010127002206A80A91F5
:108C800001F08FF9A8B100208DF8200006A8099006
:108C900008AA1221284607F009FA9DF8200038B1E9
:108CA00007E00BB029464046BDE8F04FFEF723B879
:108CB0000027012C01D147F002073A4606A9404699
:108CC000F9F710FC04003DD0284600216F22FDF783
:108CD0006CFA00B260F30F0681462846002170222C
:108CE000FDF763FA00B260F31F468246C9F34130D4
:108CF000012818D129F4C049B9F5FA6F13DC0A9894
:108D0000F8F769FD014630B220F4C040B0F57A7F33
:108D100002DDC9F57A7000E048464143642091FBCA
:108D2000F0F060F30F06CAF3413001281AD12AF49B
:108D3000C049B9F5FA6F15DC0A98F8F72EFD01461F
:108D4000301400E084E020F4C040B0F57A7F02DD0A
:108D5000C9F57A7000E048464143642091FBF0F089
:108D600060F31F466846F9F7DDF88DF80BB028462A
:108D700000216E22FDF719FA00B2ADF80000B0F53F
:108D8000616F02DDA0F5616003E0002803DA00F501
:108D90006160ADF80000284600216D22FDF705FA5C
:108DA000ADF80200284600216822FDF7FEF98DF893
:108DB0000C00294840680068007CC0F3C0008DF8B2
:108DC0001400B8073AD5D4E90001C4E9020160896A
:108DD000618A0844401E00B2E081B4F9061088425E
:108DE0002CDDE1812AE0B80705D53B462246414605
:108DF0002846F8F72FF929464046FDF77CFFA88A58
:108E00006A468119D8F804000088081AADF80400F1
:108E1000E88A00EB2641D8F804004088081AADF82B
:108E2000060021464046F9F758FBB8070CD5E08903
:108E3000401C6081618A0844401EE081B4F90A0048
:108E4000BDF91E108842CEDD21464046F9F77BFB76
:108E50000BB0BDE8F08F0000C03400202DE9F047D2
:108E60000F00814605D11B48406807F075F80700E0
:108E70002AD039464846FFF7DBFE20E00026FCF703
:108E800041FB8046002408E0A868006850F82410E0
:108E9000E6B14846FFF7CCFE641C4445F4D34A468D
:108EA0001721284607F002F94A461821284607F0FC
:108EB000FDF84A461921284607F0F8F82F463846AB
:108EC000FCF70EFC0500D9D1BDE8F087B942E3D12B
:108ED0000126E1E7C03400202DE9F04F464C8DB06B
:108EE000606801680A7CD2077ED0C9684968002999
:108EF0007FD000F5AC7001F081FD002879D1606869
:108F00000168C9688B680C930A68934200D14A686B
:108F1000924606F0F1FF0B90202103A80DF0E0F837
:108F20000025A0463CE0411991F83011B9BB00F58D
:108F3000AC7001F0D1FC0746A0462EE0D8F8040042
:108F40003946444600F5AC7001F0D8FC83466068B1
:108F5000394600EBC50203A8303200F061FF064637
:108F6000401C19D000240DF10C0909E001F0F7FCB8
:108F700009EBC401641C0A6802604968416064B27C
:108F8000D8F80400B442394600F5AC70EEDB01F0CD
:108F90003EFD384609F054FB5F46002FCED16D1CD4
:108FA000D8F804004446B0F85011A942BBD8264670
:108FB00000F5AC7001F090FC12E00B98CDF800A029
:108FC000CDE901047068DDE90B2100682346C06B20
:108FD000856BA8477068214600F5AC7001F08EFCE7
:108FE0000400EAD1706800E003E000F5AC7001F025
:108FF0005DFC0DB0BDE8F08FC03400202DE9F041DC
:109000000746FCF77FFA0646002412E0B8680068BD
:1090100050F824502846FDF7C4FC00222A21284697
:1090200007F044F82846FDF7BCFC2846FFF7E6FFAA
:10903000641CB442EAD3BDE8F0812DE9F041064654
:10904000488C0D460022C0F305100EE026B1E968F9
:1090500051F83210B14207D14FF6FF724FF4702130
:109060002846FEF733F902E0521C9042EED828461B
:10907000FCF748FA0746002407E0A868006850F8A3
:1090800024103046FFF7D9FF641CBC42F5D3BDE87D
:10909000F0812DE9FF5F9846DDE91354DDE90E7696
:1090A0008246DDF848B0F3F7C3FB00685946D0F8B4
:1090B0003890204609F0FCFB002084462BE01099F4
:1090C000414307EB21221199414306EB2121121262
:1090D0004FEA212107D4019B9A4204DA002902DBDE
:1090E000029B994202DB04F800C007E001FB082163
:1090F0000AEB410105EB4002098811801599062908
:1091000007D135F810201FFA89F18A4201D104F8FD
:1091100000C0401C00B25845D1DBBDE8FF9F0022D3
:1091200000680A2106F0C2BF2DE9FF4F85B09046C6
:109130000C460846FCF7D4FA06461021FDF7A0F9C4
:1091400000286FD03046FCF729FB834600253046C7
:10915000FCF7F1FB1434CDE9024000B9059C002175
:109160003046FCF790FF824600213046FDF717F8A5
:10917000504407B200213046FCF7EDFF504401B2E5
:109180000191F08A61883844411AB8F80200728B64
:10919000091A0FFA81F90199511AE288891A401ABD
:1091A00000B200903046FCF760FA0199C01B401AEB
:1091B00000B20490B9F100010DDB0098002815DA27
:1091C0000846B9F1000F06DD05463046FCF7BAFB4C
:1091D000401B0AD40AE00098002807DD404205B28F
:1091E0003046FCF789FAE84200D5002503980128AB
:1091F00004D0022806D003280CD114E0F08A61883C
:10920000384403E0718B0198081AE1882944401A18
:10921000284405B200243046FCF786FB0090A8B134
:10922000029F14E0BEE00498F18A00EBD07007EBD7
:1092300060000A18E0886188401A401C00B200EB08
:10924000D07005EB60000844101AE1E7059F00218B
:109250003046FCF78CFF50440FFA80F9002130466D
:10926000FCF791FF5044B18A0FFA80FA01EB090034
:109270003988338B421AB8F80010501AA3EB0A024F
:10928000BB8800B2D21A891A09B200280ADB002969
:1092900012DA002806DD04463046FCF787FA001B88
:1092A00009D409E0002907DD484204B23046FCF742
:1092B000DDFAE04200D500243046FDF7C2F8A0EB0D
:1092C0000901A1EB0A0001B20098012804D002288C
:1092D00007D003280DD122E0B18A01EB09003988BB
:1092E00003E0318BA1EB0A00B9882144401A2044E5
:1092F00004B22E493046F8F7FBF807462C493046B1
:10930000F8F7F6F8074306D000220A21304606F0A7
:10931000CDFE012846D15FEACB7012D014E001EBFC
:10932000D171B28A09EB61000244B8883988401AC9
:10933000401C00B200EBD07004EB60000844101A2F
:10934000D5E7002C00DA00245FEA8B7002D4002CF1
:1093500000DD00245FEA4B7002D4002D00DA002506
:109360005FEA0B7002D4002D00DD00250898B8F9E3
:109370000010002800D020460844A8F80000B8F9E2
:10938000021002D14FF0000000E028460844A8F87F
:109390000200089B09B02A4621463046BDE8F04F3E
:1093A000FEF704B909B0BDE8F08F0000CD930108C5
:1093B000B593010810B50346FCF7CBFA084401B297
:1093C000BDE8104000221846F3F757B810B5034621
:1093D000FCF7C6FA084402B2BDE810400021184666
:1093E000F3F74BB8F8B505460C460846F9F726FEE4
:1093F0004FF4803631462846FCF72BFEE0700228F9
:1094000008D9284631462022FCF7CFFE0090BDF84F
:109410000000A080284631463122FCF7C6FEC0B2CB
:10942000002784F82200022814D928463146322227
:10943000FCF7BBFE00B22084002809DD2846314637
:109440003022FCF7B2FE0090BDF80000E08301E09E
:1094500084F82270284631464522FCF7A6FEC0B2A9
:1094600084F8360002281AD9284631464022FCF7F3
:109470009CFE00B2E08500280FDD284643223146DD
:10948000FCF793FEA086284644223146FCF78DFE69
:109490000090BDF80000A08501E084F836703146E8
:1094A0002846FCF716FEFD280AD2E17811FB00F1F0
:1094B000090AE1704143080A84F8220084F8360062
:1094C000E07830B994F8220018B994F836000028F2
:1094D00005D031462846FCF7AFFE20800120F8BDBC
:1094E0002DE9F84F044615460E464FEA61084FEA4B
:1094F000610AC80701D1A8F101086000009009F0D5
:1095000041F807462B46002025E003EB440B3BF8CF
:10951000021C7143601E16D4002200EB0A0C27F8CF
:109520001010A44501DA33F81C208A1AA0EB0801B8
:10953000012901D5198803E003EB410131F8021C30
:10954000401E1144E8D539461846009A09F0B4F88F
:109550005B4609F101008146A042D6DB4FF47F5201
:10956000B2FBF6F100201FFA81FC14FB04F30CE0BF
:1095700035F8101041B1914202D125F810C003E036
:1095800091FBF6F125F81010401C8342F0D8002121
:1095900039E005EB410399461A887243002024E024
:1095A000002A02DA4FF0000C01E04FEAA21C27F873
:1095B00010C0A0EB0A0CBCF1000F02DCB3F800C035
:1095C00003E00CFB041C35F81CC0A2EB0C0C00EBF8
:1095D0000802521CA24200DB621E02FB041203EBD3
:1095E000440335F81220401C6244A042D8DB4A46AE
:1095F000002005E037F81030138002EB4402401CD5
:10960000A042F7DB491CA142C3DB3846BDE8F84F56
:1096100009F004B82DE9F0470E468AB01D46804691
:10962000014617469246541907A8F8F7A7F807EB22
:10963000D77005EB600147F30002891A891EADF867
:109640002010012101EB6000ADF81E004046F8F744
:10965000E0F8BDF82010081AADF81C004046F8F7F5
:10966000AEF8BDF81E1000230844ADF822002A46CB
:1096700007A901A8F9F714FC5746BAF1010F01D068
:109680004FEA6A07204608F07DFF804635460020F5
:1096900034E02146404609F00BF901A80090DDF8BE
:1096A00004C023B20FFA89F200214046E04738B1E6
:1096B00098F80000800190FBF7F02880012017E067
:1096C0006100284609F0C7F814E008EB000218F81A
:1096D000001012F8012C914204D105EB400131F841
:1096E000021C02E0890191FBF7F125F81010401CE3
:1096F000A042EADB05EB440509F101008146A042E6
:10970000C7DB404608F08AFF01A8F9F743F9012FAB
:1097100014D020B2324639460546FFF7E1FE0AF082
:109720000100384401B2012927DD4FF47F5090FB3E
:10973000F1F2002097B204FB04F318E00020314658
:10974000644304E036F8102092090A54401C844215
:10975000F8DC0AB0BDE8F08736F8102032B1FF2AF5
:109760000FD0920192FBF1F226F81020401C8342A8
:10977000F2D832462846FFF7B3FE00203146644354
:1097800006E026F81070F1E716F810200A54401C85
:109790008442F9DCDDE7F0B597B0074615460E4682
:1097A00001A8F9F74BFCFF2211461046F8F7B5F86F
:1097B0000090BDF800000090BDF80000ADF8080072
:1097C0000024324601A93846F9F724FC0FA8F8F71F
:1097D00059FE2B4632460FA938460094F8F7BCFBD9
:1097E00017B0F0BDFEB5066804460A46708C002529
:1097F0000421C0F305130BE0F06801EBC507C05965
:10980000870104D5A76820F07F40B84203D06D1CC3
:10981000AB42F1D8FEBDA18844295CD00EDC3329CF
:109820004CD006DC202956D0222954D0302913D11F
:1098300051E0342942D036290ED14CE0622940D083
:1098400006DC472947D0552945D0572904D135E0B2
:10985000672933D0682931D062B3FF2A2CD0D4E9EC
:1098600003031B1A534300EB23200090F0680127E9
:1098700001AA50F8350009F079FF60B1DDE9000177
:10988000884208D1BDF80020BDF804309A4202D1C8
:10989000884200D10027F068A188009A50F835006E
:1098A0000AF064F9002FB5D0A288A1682068FDF7FE
:1098B0000DFDFEBDE068D8E72069D6E7FF2AFBDA98
:1098C000F8E7E0680028F7D02369002BCDD0802A84
:1098D000CBDB0093CAE7002A01DCA0892AE0FF2A3B
:1098E00001DB208A26E0208AD3B280B2020242EA5B
:1098F0001020A78982B2B8B2070247EA10201B1DC8
:10990000DF080E4B80B240EA004042EA02421840B3
:109910001A40121A7A4300EB5210184040EA1040E5
:1099200080B2020242EA1020ADF8080080B2029034
:10993000BDF80800ADF8000098E700001FF8E00748
:109940002DE9F041046800262648A788256800F024
:10995000C3FF10E0A1420BD008682268904207D1F3
:109960008868A268904203D18888A288904237D044
:109970001C4800F0C3FF0100ECD1002E30D1688CF0
:109980000421C0F3051229E0E86801EBC603C058C2
:10999000830122D5A36820F07F4098421DD1214643
:1099A000104801F034F8204608F04AFEE8683946CD
:1099B00000EBC604206809F0CFFFE86850F83600D5
:1099C00009F029FF00280BD06068216820F07F4251
:1099D0002846BDE8F041FDF74FBD761CB242D3D812
:1099E000BDE8F081447D002070B50468A068A288BD
:1099F00000F47F0631462068FCF7D7FBE060A588BD
:109A00000020A08023462A463146206800F00CF84A
:109A1000A580A1682068F7F734FAA1880068E26899
:109A2000BDE870400AF0A2B82DE9FF5F07469146F5
:109A30000E460024254800F068FF05464FF4702BC1
:109A40004FF0040A3CE0039885423BD029461F486A
:109A500000F058FF80462868B84230D1A868B0426C
:109A600001D05E452BD1A988494503D0A9F57F4196
:109A7000FF3924D1002411E0F8680AEBC4014158F1
:109A80008A010AD55E4503D021F07F41B14204D15D
:109A900050F83400A98809F05FFF641C788CC0F38B
:109AA0000510A042E8D800212846F7F721FD2946F5
:109AB000064800F0ACFF284608F0C2FD01244546E8
:109AC000002DC0D104B02046BDE8F09F447D0020A9
:109AD0002DE9F74F934682B0044600216E22FCF731
:109AE00064FB06B2204600216D22FCF75EFB05B246
:109AF00016B9B5F5807F67D0204600216F22FCF7AC
:109B000054FBADF80000204600217022FCF74DFB0D
:109B1000ADF80200BDF9000004F11401C0F34132B8
:109B200064274FF4FA688A464FF47A79012A14D1EF
:109B300020F4C040404510DC0846F7F746FE0146D9
:109B4000BDF9000020F4C040484501DDC0F57A7041
:109B5000414391FBF7F0ADF80000BDF90200C0F3FE
:109B60004131012914D120F4C040404510DC504659
:109B7000F7F70DFE0146BDF9020020F4C04048454C
:109B800001DDC0F57A70414391FBF7F0ADF80200BA
:109B9000A08ABDF80010BBF1000F0844ADF800002A
:109BA000E08ABDF802100844ADF8020006D0704209
:109BB00006B24FF4803090FBF5F005B26B462A46B2
:109BC0003146039809F076F805B0BDE8F08FF0B59E
:109BD000D0E90646059D4FF480772EB9BC4203D1EB
:109BE00008021860100239E0B0F928C0A1EB0C019E
:109BF000B0F92AC0A2EB0C029EB1BC421AD1446952
:109C000006694C4306FB1244066A06EBA4041C607A
:109C100003694B434169406A01FB023100EBA1003B
:109C20001CE0066A01FB04611960416A806902FB5D
:109C3000001013E0466907694E4307FB126666434E
:109C4000046A04EBA6241C6003694B43416901FBD1
:109C500002318269406A514300EBA1202860F0BDC7
:109C600000000000834D0108694E0108000000005B
:109C7000A5510108820082004A020000000001E0B4
:109C800001E0000000FF0055AAFF001122334455F7
:109C900066778899AABBCCDDEEFF000102030405BC
:109CA000060708090A0B0C0D0E0F101112131415DC
:109CB000161718191A1B1C1D1E1F202122232425CC
:109CC000262728292A2B2C2D2E2F303132333435BC
:109CD000363738393A3B3C3D3E3F404142434445AC
:109CE000464748494A4B4C4D4E4F5051525354559C
:109CF000565758595A5B5C5D5E5F6061626364658C
:109D0000666768696A6B6C6D6E6F7071727374757B
:109D1000767778797A7B7C7D7E7F8081828384856B
:109D2000868788898A8B8C8D8E8F9091929394955B
:109D3000969798999A9B9C9D9E9FA0A1A2A3A4A54B
:109D4000A6A7A8A9AAABACADAEAFB0B1B2B3B4B53B
:109D5000B6B7B8B9BABBBCBDBEBFC0C1C2C3C4C52B
:109D6000C6C7C8C9CACBCCCDCECFD0D1D2D3D4D51B
:109D7000D6D7D8D9DADBDCDDDEDFE0E1E2E3E4E50B
:109D8000E6E7E8E9EAEBECEDEEEFF0F1F2F3F4F5FB
:109D9000F6F7F8F9FAFBFCFDFEFF808080818182F6
:109DA000828384858687898A8C8D8F9193959799F4
:109DB0009B9EA0A2A5A7AAADAFB2B500FF1FFF1F33
:109DC00001E001E09CAF060800000020DC35000047
:109DD0003070020818B80608DC35002054DD000099
:109DE00024C2000870B5044600256FF02F0608E075
:109DF0002068411C2160007805EB850106EB4101DC
:109E000045182068007800F004F80028F0D12846B2
:109E100070BD3038092801D80120704700207047F4
:109E20002DE9F0470F46814690461146384600F02E
:109E30000CF940B100224146384600F0B2F828B192
:109E40000020BDE8F0874FF0FF30FAE700263846E3
:109E500005F0D6FC401E0FFA80FA384605F0AAFC41
:109E6000401E02B2B8F80210B7F90200091A09B28E
:109E700000290FDD3B88012663F30F0460F31F44C4
:109E8000BB88084463F30F0560F31F45C9F8004021
:109E9000C9F80450B8F906007988411A511A09B274
:109EA000002913DDB7F9062090420FDA3A8862F3F1
:109EB0000F04BA8860F31F4462F30F05084460F38F
:109EC0001F4509EBC600761C04604560B8F9020026
:109ED000B7F90210884200DC0846B8F90610B7F955
:109EE0000620914200DB1146B8F80030B7F9002097
:109EF000091A9B1A1BB209B2002B10DD00290EDDD6
:109F000062F30F041A4462F30F05421862F31F450F
:109F100009EBC60260F31F4414605560761CB8F963
:109F200004203B88D71AAAEB07031BB2002B0EDDD7
:109F300062F30F0460F31F441A4462F30F050844F0
:109F400060F31F4509EBC600761C0460456030468F
:109F500077E770B5B1F90040B2F900309C4200DDFE
:109F600023460380B1F90240B2F90250AC4200DC52
:109F70002C464480B1F90450B2F90460B54200DBCC
:109F800035468580B1F90610B2F90620914200DB12
:109F90001146C1800120AB4201DC8C4200DD002073
:109FA00070BDF8B50D460446B0F90000B1F90010D7
:109FB0001646884247DBB4F90210B5F902209142F7
:109FC00041DBB4F90410B5F9042091423BDCB4F94B
:109FD0000610B5F90620914235DC96B3ADF80000C5
:109FE0006088ADF8020032466946284600F099F8CC
:109FF000002827D0A088ADF800006088ADF80200E6
:10A0000032466946284600F08CF800281AD020888D
:10A01000ADF80000E088ADF80200324669462846F7
:10A0200000F07FF800280DD0A088ADF80000E0888F
:10A03000ADF8020032466946284600F072F8002862
:10A0400000D00120F8BD0020F8BDB0F90020B1F922
:10A0500004309A4213DCB0F90420B1F900309A427E
:10A060000DDBB0F90220B1F906309A4207DCB0F9F5
:10A070000600B1F90210884201DB01207047002080
:10A080007047F8B50D460446B0F90400B1F9001068
:10A090001646884243DBB4F90600B5F9021088423F
:10A0A0003DDBB4F90000B5F90410884237DCB4F99F
:10A0B0000210B5F90620914231DC76B3ADF800000C
:10A0C0006088ADF8020032466946284600F029F85B
:10A0D00018BBA088ADF800006088ADF802003246D9
:10A0E0006946284600F01DF8B8B92088ADF8000090
:10A0F000E088ADF8020032466946284600F011F8C3
:10A1000058B9A088ADF80000E088ADF802003246EA
:10A110006946284600F005F808B10020F8BD012086
:10A12000F8BD2DE9FC4105460F46B1F90000B5F92F
:10A130000010144688423BDBB5F90410884237DC36
:10A14000B7F90200B5F90210884231DBB5F9061003
:10A1500088422DDC002C76DD284605F051FB00EB13
:10A16000D0704610284605F025FB00EBD07040105B
:10A17000864200DA3046844200DD04462888ADF885
:10A180000000288800222044ADF804006888ADF85B
:10A190000200688839462044ADF806006846FFF79B
:10A1A000C0FF40B1BDF804002044ADF804003FE01A
:10A1B0000020BDE8FC81E8880022001BADF8020009
:10A1C000E888ADF8060039466846FFF7AAFF28B1CF
:10A1D000BDF804002044ADF8040011E0A888002276
:10A1E000001BADF80000A888ADF8040039466846A9
:10A1F000FFF797FF50B1BDF80000001BADF800005D
:10A20000BDF80200001BADF8020016E06888ADF84A
:10A210000200688800222044ADF8060039466846EE
:10A22000FFF77FFF70B1BDF80000001BADF8000024
:10A23000BDF806002044ADF806003946684608F02F
:10A24000D7FDB6E7FFE70120B3E710B5B1F900305D
:10A25000B2F90040A34200DB23460380B1F902308B
:10A26000B2F90240A34200DB23464380B1F9043037
:10A27000B2F90440A34200DC23468380B1F9061002
:10A28000B2F90620914200DC1146C18010BD0000E9
:10A29000084949680AE04A68824202D00A68824254
:10A2A00003D10A7E42F001020A7649690029F2D1FF
:10A2B00070470000943400207047000004210148DA
:10A2C00000F027BB147D00202021014800F021BBB5
:10A2D0002C7D00202DE9FF410446DDE90A571E00D0
:10A2E0004FF0000002D1B5F5807F2BD00390019094
:10A2F0000290ADF80C100090ADF80410ADF80A20F3
:10A30000ADF80E203B462A463146684608F0D2FC9E
:10A310003B462A46314601A808F0CCFC3B462A467B
:10A32000314602A808F0C6FC3B462A46314603A83F
:10A3300008F0C0FCBDF90030BDF90420934209DAF1
:10A340001D4608E02080491E6080A180521EE280E8
:10A35000BDE8FF811546BDF90800BDF90C10884223
:10A3600001DA064600E00E46B54205DA934201DA0C
:10A37000184604E0104602E0884200DB0846801ED2
:10A380002080BDF90030BDF90400834201DD1D4687
:10A3900000E00546BDF90820BDF90C108A4201DD38
:10A3A000164600E00E46B54203DD834206DD184640
:10A3B00004E08A4201DD104600E00846801CA080CF
:10A3C000BDF90230BDF90620934201DA1D4600E0D6
:10A3D0001546BDF90A10BDF90E00814201DA0E469C
:10A3E00000E00646B54205DA934201DA184604E079
:10A3F000104602E0814200DA0846801E6080BDF906
:10A400000230BDF90620934201DD1D4600E01546ED
:10A41000BDF90A10BDF90E00814201DD0E4600E0D3
:10A420000646B54205DD934201DD184604E01046BC
:10A4300002E0814200DD0846801CE08088E70000E1
:10A440002DE9F04115460E460746114C09F0BAFDBC
:10A4500080462B4632463946204606F07BFF20B127
:10A460000020A062E06950B110E02C21204608F0E5
:10A47000F2F94FF00040A0620020BDE8F0814046B4
:10A4800009F099FDE06108B90120E0612046F4E798
:10A49000507D002010B51421074800F03AFA06F06C
:10A4A0001FFF40B1054901600549416005498160D0
:10A4B0000549C16010BDFEE7387D0020C10C0208CF
:10A4C00035100208011202088D0C020870B50D4605
:10A4D00004461021284608F0BEF9206800780128BB
:10A4E00004D0022807D0042807D008E0A08A2880DA
:10A4F000E08A688003E0E06800E00A206860206885
:10A500004268002A03D02946BDE87040104770BD5C
:10A510002DE9FE430446808A10B9E08A002874D0F1
:10A52000D4F82C805FEA080010D1204602F0D9FA56
:10A530005FEA000869D0204604F034F900220921BE
:10A54000404605F0B3FD607880075ED44FF4807913
:10A5500000274D4646460021304608F0FFFA3844B1
:10A5600007B20021304608F0FFFAC11700EB116076
:10A57000001210FB05F005B23046FBF7B1F80600FB
:10A58000E9D10FB94D450CD0784201B24FF480307B
:10A5900090FBF5F002B26B4604F11400009608F04F
:10A5A00089FBADF80860ADF8046094F8400000F055
:10A5B0000F000328404616D0FBF7C4F90546404675
:10A5C000FBF79AF803460C200090B4F916102A46BF
:10A5D000404602F033F9ADF804004046FBF7DEF8E0
:10A5E000C10713D018E0FBF741F905464046FBF7D9
:10A5F000DDF8024603200090B4F914102B464046C3
:10A6000002F01CF9ADF80800E7E736E0BDF90810E4
:10A61000002901DDADF80860810705D4BDF90810F7
:10A62000002901DAADF80860410705D4BDF904102E
:10A63000002901DDADF80460000705D4BDF9040070
:10A64000002801DAADF8046001AA02A920460AF048
:10A6500032FABDF90420BDF908104046F1F70DFFAC
:10A660006078800709D4208BBDF808100844208347
:10A67000608BBDF8041008446083BDE8FE832DE9BB
:10A68000FC5F0446C06A5FEA000B71D094F840009A
:10A6900000076DD007F0DEF8019000684021457E8C
:10A6A0005846FBF7EDFE4FF0000818B9A4F81E80DD
:10A6B000A4F81C805846FBF737F982465846FBF74A
:10A6C0003AF9064694F840004FF0640900F00F0094
:10A6D0000C2802D003284CD09AE0A4F81C8056B174
:10A6E000B4F91E50002707F0B5F800684946407ECF
:10A6F000C0F1640022E0E08BC5F1640110FB01F1C0
:10A7000091FBF9F0E0835846FAF7F6FF0546584604
:10A71000FBF718F902460C200090B4F91E102B46E6
:10A72000584602F08BF8E083024600231EE07A19B7
:10A7300017B210FB05F292FBF1F215B2002DF6D123
:10A74000ADF80070A4F81E806A46002120460AF089
:10A75000B2F941F6FF72BDF900305142584602F09D
:10A7600057FBBDF800100123084402B200214CE061
:10A770009AE0A4F81E80BAF1000F0AD0B4F91C5078
:10A78000002707F067F800684946407EC0F1640082
:10A7900022E0A08BC5F1640110FB01F191FBF9F0FF
:10A7A000A0835846FBF702F805465846FBF75EF8CB
:10A7B000034603200090B4F91C102A46584602F0C4
:10A7C0003DF8A083014600231EE07A1917B210FB62
:10A7D00005F292FBF1F215B2002DF6D1ADF8007042
:10A7E000A4F81C800022694620460AF064F941F66C
:10A7F000FF72BDF900305142584602F087FABDF8A9
:10A8000000100123084401B200225846FCF7CEFE96
:10A81000A08B002848D1E08B002845D1C6B9584606
:10A82000FBF790F805465846FAF766FF002D06DC60
:10A8300000280DDD002D02DA01232A4604E000285D
:10A8400006DA0123404202B200215846FCF7AEFE70
:10A85000BAF1000F19D15846FAF7A8FF0546584635
:10A86000FBF704F8002D07DC00280EDD002D03DACD
:10A8700001230022294605E0002806DA01230022F0
:10A88000404201B25846FCF791FE0A215846019A0F
:10A8900005F00CFC6078800706D414F8400F20F017
:10A8A0000F00207044F8148CBDE8FC9F70B505467D
:10A8B00000F012F804460CE02146284600F01EF88D
:10A8C00006462146284600F0A2F8204607F0B8FECA
:10A8D0003446002CF0D170BD002800D0406870478D
:10A8E00000B503460022FFF7F7FF03E01846521CAD
:10A8F00000F004F80100F9D1104600BD0068091D00
:10A9000040587047006840587047002800D0806861
:10A91000704700224260C91C21F00301826001607F
:10A92000704770B504460068083007F0FDFD05006B
:10A9300013D001460022204609F0BFFE29462046DA
:10A94000626809F0B1FE616819B12A46204609F033
:10A95000B4FE6560A06800B9A560284670BD2DE909
:10A96000F0410D4606000AD04DB1FFF7B5FFA842F1
:10A9700008D13046FFF7D5FF041E01D01EE00020AD
:10A98000BDE8F0813068083007F0CEFD041EF7D036
:10A990003068224647593046394609F085FE3A4626
:10A9A0002146304609F089FE22462946304609F004
:10A9B00084FE2A462146304609F076FE2046DFE72F
:10A9C00070B504460068083007F0AEFD050013D0EE
:10A9D00001460022204609F067FE29462046A2686B
:10A9E00009F06BFEA16819B12A46204609F05CFE09
:10A9F000A560606800B96560284670BD28B14168EF
:10AA000009B9806808B1002070470120704770B50F
:10AA100004000DD0FFF760FF00228842204608D1D5
:10AA2000FFF76CFF606010B1002201461EE0A260DB
:10AA300070BDFFF76AFF8842206808440AD10168A8
:10AA4000A16029B12046BDE87040002209F02CBE6B
:10AA5000626070BD05682046FFF750FF064602465B
:10AA60002946204609F020FE2A4631462046BDE808
:10AA7000704009F022BEC0F30410072800D9072057
:10AA800070470000A0F57F41FF3905D0002804D0B1
:10AA9000712803D208490AE01F207047074971381E
:10AAA00080B2096829B1064A5268904201D2085C16
:10AAB0007047002070470000905A0208703500204F
:10AAC000843500202DE9F041094C90460E4662681D
:10AAD0001D46074619469047306020B128686268D5
:10AAE000384400219047C8F80000BDE8F08100001C
:10AAF000A03500202DE9F04F87B08A46DDE91058D7
:10AB00001F4693460446002105B129805CB1207898
:10AB1000002809D0BAF1000F05D0002618F0060F62
:10AB200015D0002004E0002007B0BDE8F08F401CE5
:10AB3000215C0A2904D00D2902D00029F7D100E0B8
:10AB4000401C002DF0D04FF0FF312980ECE75FEA88
:10AB5000887001D541F6FF77894608468DF81010B8
:10AB6000059125E00598CDF8189058B3002104AB65
:10AB7000CDE902310DF1180CCDE9008C20443B46A3
:10AB80005A46514609F066FB06997A1A314417B2C3
:10AB90000EB288B105990844059021780A290BD096
:10ABA0000D2909D0205C0A280ED00D280CD005985C
:10ABB000205C08B1002FD5DC059848B105B12E8086
:10ABC0000598B1E70121D2E70598401C0590F3E70D
:10ABD000064A05A92046526890470146002DEFD04D
:10ABE0000022504605F077FB06B2E8E7A0350020CA
:10ABF00000230278232902D0012A0DD00FE02AB1C8
:10AC00000021012A04D0022A04D008E0012101E039
:10AC1000017004E0017001E0202902D001231846F0
:10AC200070470221F6E72DE9F0410B460F468046BA
:10AC300002460021084609F015FD05460026401C85
:10AC400007F072FC040008D066553B464246691C7A
:10AC500009F008FD2046BDE8F081FEE72DE9F04748
:10AC6000984614460D468246DDF8209013E06608AB
:10AC700006FB0857394650464A469047002808DDEB
:10AC800044F30000C0EB540407EB0805A4F10104F1
:10AC900001E005DA3446002CE9D12046BDE8F08712
:10ACA0003846FBE72DE9FC5F0CAD9E4692468B468D
:10ACB00095E81201DDE91132DDE90F7C96074FF0CE
:10ACC000300519D453B1D60708D002F00C0656EA65
:10ACD000080603D05B1E01E00D55641C644504D2D8
:10ACE000202CF9D301E00D55641C5FEAC27903D032
:10ACF0009C4201D2202CF6D3D60624D556050AD480
:10AD00004CB1644501D09C4205D1641E03D0102F84
:10AD100003D1641E04E0102F02D0022F0AD00EE0EF
:10AD2000960603D4202C1ED2782606E0202C1AD2B8
:10AD3000582602E0202C16D262260E55641C202CC8
:10AD400011D20D55641C202C0DD2B8F1000F01D08A
:10AD50002D2506E0550701D52B2502E0150702D564
:10AD600020250D55641CCDE900EB064655468B4663
:10AD700098469146900713D1274606E02A46DDE91A
:10AD800000316D1C2020B0477F1C4745F6D307E0FB
:10AD90002A466D1C641EDDE900311BF80400B04733
:10ADA000002CF5D15FEA897006D409E02A46DDE976
:10ADB00000316D1C2020B047A5EB0A014145F5D3B9
:10ADC0002846BDE8FC9F2DE9F04F8FB099468B4691
:10ADD000DDE91818DDE91C63DDE91A47864692466D
:10ADE000002009B923F010035A0507AD00D5C9B1F9
:10ADF000B1FBF4F204FB1212D2B20A2A01D23032B1
:10AE000009E05FEA836C02D54FF0410C01E04FF09E
:10AE1000610C62440A3AB1FBF4F12A54401C09B1B6
:10AE20002028E5D3CDF80880CDE90563CDE90050B1
:10AE3000CDE903474B46524659467046FFF732FF6D
:10AE40000FB0BDE8F08F2DE9FF4F8FB01CACDDE9EE
:10AE5000239594E8030820AC94E8C004002450EA49
:10AE6000010201D125F010056A050DF11C0802D57B
:10AE700050EA010217D032463B460BF0D3F8D2B26B
:10AE80000A2A01D2303206E0AB0601D5412300E0A8
:10AE900061231A440A3A08F80420641C50EA0102AB
:10AEA00001D0202CE7D3CDE90084CDF808B0CDE95E
:10AEB0000595CDE9036A0FAF97E80F00FFF7F2FEA3
:10AEC00013B0BDE8F08F9A4200D2885470477047A3
:10AED0002DE9FF4F89B082460A980024169D00286C
:10AEE00001D1DFF8F0A367E1252802D02246641CD7
:10AEF000E2E1491C002608460C9101782B291BD061
:10AF000004DC20291BD0232904D11BE02D290ED0DD
:10AF1000302909D00027C8B2FEF77BFFA8B10CA8E2
:10AF2000FEF760FF07461CE046F0010601E046F030
:10AF30000206401C0C90E0E746F00406F9E746F0F4
:10AF40000806F6E746F01006F3E70C9801782A2980
:10AF500007D180CD002F02DA46F002067F42401C66
:10AF60000C900C984FF0000801782E2917D1401C46
:10AF70000C9046F480660078FEF74BFF20B10CA8D9
:10AF8000FEF730FF80460AE00C9908782A2806D19F
:10AF900001CD002800DC0020491C80460C910C9853
:10AFA00001786C290AD004DC68290FD06A2918D1ED
:10AFB00027E0742928D07A2913D125E0401C0C9071
:10AFC000017846F480766C291BD00AE0401C0C9076
:10AFD000017846F08006682903D146F04006401CFF
:10AFE0000C9002460078692822D015DC62281FD018
:10AFF0000DDC252877D050281AD058287FF476AF5A
:10B0000016E046F40076EAE746F48076E7E7632840
:10B010006AD06428F2D10BE073286FD004DC6F286B
:10B0200006D07028EAD103E0752801D07828E5D150
:10B0300078280DD058280BD070280BD0502809D074
:10B040006F2816D0622816D00A2126F0100616E0C6
:10B05000102107E05078102146F48876562804D154
:10B06000521C0C921078582807D01078502804D021
:10B0700005E0082108E0022106E046F020061078ED
:10B08000692803D0642801D026F00C06700501D58C
:10B0900026F001061078692813D0642811D05628AC
:10B0A00054D0B00560D5ED1D0020CDE90410CDF8D9
:10B0B00018800290CDE9077625F00705F5E8020132
:10B0C00021E0B00528D5ED1D25F007050023F5E8A2
:10B0D00002020DF11009002A89E80A01CDE907767C
:10B0E00003DA012102E0E4E070E000210023029194
:10B0F00019461B1A914102DA114604E08EE0002144
:10B10000404261EB0201CDE90001DDE90A1322466C
:10B110005046FFF798FE4BE0F00503D501CD0BE05C
:10B12000404210E0700602D515F8040B04E030062A
:10B13000F4D535F8040B00B2CDE90218CDE9047658
:10B14000C10F0028ECDDCDE900012BE001CD416805
:10B150000968009103680B98021B0A980119504670
:10B16000FFF7B6FE044424E0F00508D5CDE9021847
:10B17000CDE9047602CD0020CDE9001012E0700682
:10B1800002D515F8040B06E0300603D535F8040B9C
:10B1900080B200E001CDCDE902180021CDE9000127
:10B1A000CDE90476DDE90A1322465046FFF70BFE8F
:10B1B00004460C98401C0C900C99087800287FF4E9
:10B1C00093AE0B9884427BD222467AE04FF001087E
:10B1D000B00707D50BE02246DDE90A13641C2020E6
:10B1E000D446E047404608F10108B842F3D3DDE910
:10B1F0000A13224615F8040B641CD446E047B00736
:10B2000006D4D6E72246DDE90A13641C2020D04785
:10B21000414608F10108B942F4D3CAE755F804BB26
:10B22000B8F100005A4601D0014601E04FF0FF316D
:10B23000584600E0401C03780BB1491EFAD2A0EB3F
:10B240000209700505D548464146C14500D3084668
:10B250008146B00707D514E02246DDE90A13641CD5
:10B260002020D446E047494609F10109B942F3D309
:10B2700007E0DDE90A1322460BF1010B641CD446FA
:10B28000E0479BF8000020B17105F2D5B8F1010844
:10B29000EFD2B00706D48CE72246DDE90A13641C1E
:10B2A0002020D047494609F10109B942F4D380E78B
:10B2B00006E02246641C2520DDE90A13D04778E722
:10B2C000421E034600200A99D0470DB02046BDE833
:10B2D000F08F0000CFAE010810B503004FF0000062
:10B2E0000DD04A1E114200D0FEE71944491E914379
:10B2F0000A46B1F5004F02D20C2A01D9084610BD0A
:10B300000C2010BD08444A1E401E9043114200D03C
:10B31000FEE7704770B5044640680D4608B1FFF778
:10B32000F9FF2268002A04D029462046BDE8704073
:10B33000104770BD89B204F055B989B204F0D8B98C
:10B3400070B50D46044600F04DF800B1FEE76868A0
:10B35000616820F00300001D08446060204600F092
:10B3600049F8204670BD4068103120F00300884243
:10B3700001D301207047002070472DE9FC470546A6
:10B3800048680C4620F0030001AA694609F076F9E6
:10B39000DDE9006005EBC61101EB80098046D9F8B4
:10B3A000380060B164B1C4E9020504F10807C46063
:10B3B00038460421FFF7A6FF874202D0FEE7FEE7EA
:10B3C000FEE7C9F838400123286903FA06F108436B
:10B3D000286105EB860003FA08F142690A434261DD
:10B3E000BDE8FC87406830F0030001D000207047C2
:10B3F0000120704710B5044600F08CF8046010BDC1
:10B400002DE9FC474FF0000780460E0001973D46AE
:10B41000009745D00C460DF1040AE946802907D370
:10B4200008460AF08FF9411F01208840401E04445D
:10B430004A465146204609F021F9019C092C2FDA91
:10B4400008EB8400009940694FF0FF3202FA01F1E5
:10B45000454608400CD1641C2869A240104016D013
:10B460000AF068F90446019005EB8000406980B15C
:10B470000AF060F905EBC411009001EB8000856BC8
:10B4800075B1686820F00300B04203D2FEE73D4684
:10B49000F6E7FEE7DDE900322946404609F07CFA8E
:10B4A0002846BDE8FC8710B50446FFF7A3FF4168B6
:10B4B00041F002014160606840F00100606010BD31
:10B4C00010B5044600F026F8416821F00201416001
:10B4D000606820F00100606010BD70B506460D4642
:10B4E000084600F017F8040008D0207910F0010F8A
:10B4F0000ED02846FFF776FF08B1FEE7FEE72146AB
:10B50000304600F03EF821462846FFF719FF054671
:10B51000284670BD10B5426800F1080122F0030210
:10B52000121F8C18FFF75EFF00B1FEE7204610BD2A
:10B5300070B506460C004FF000001FD0FAB120791C
:10B54000154610F0010F1BD011462046FFF70BFFE8
:10B5500078B12946204600F025F805462046FFF739
:10B5600049FF6868294640F0020068603046FFF7EE
:10B5700004FF2046FFF7A4FF04F1080070BDFEE7BA
:10B58000FEE77CB5054648680C4620F003006A4695
:10B5900001A909F073F8DDE900322146284609F0D7
:10B5A000FBF97CBD2DE9F0410D4604460830091F2A
:10B5B0004618606806F1080720F00300401BA0F160
:10B5C000040838460421FFF79DFE874200D0FEE7BD
:10B5D000606808EB050120F00300091D884200D0D7
:10B5E000FEE7307900F0030040EA0800706020F0C8
:10B5F00003000C2800D2FEE7207900F00300284366
:10B6000060603046FFF74FFF3046BDE8F081000034
:10B610002DE9F04F0C4687B005460021F9F760FF91
:10B6200060B32146284600F021F92146284600F063
:10B630006FF80021284607F025FA059000212846DA
:10B6400007F050FA04900021284607F0E1F901289C
:10B6500000D0002080460021284607F091FA0646D7
:10B660000021284607F0F0F942F2D17907464E450D
:10B670000BD1688C000508D4012607E007B02046EE
:10B68000BDE8F04F1C2107F0E6B800262846F9F780
:10B69000A7FFDFF878A0834628460021BAF80420E7
:10B6A000FAF783FDD4F810C0A3682168CDF800C074
:10B6B000CDF80C80CDE90131C2B231465846059B28
:10B6C00002F0B0F920834F4504D1688C400501D4C5
:10B6D000012600E000262846F9F766FF07462846BF
:10B6E0000021BAF80820FAF760FDC2B260690025AF
:10B6F0006368E1688DE82B0031463846049B02F010
:10B7000091F9608307B0BDE8F08F0000E8340020B5
:10B710002DE9F34F81B00C46019801F06BFF804694
:10B720000198F9F75DFF8346404600F02FFB20614A
:10B73000400006F027FF20602069400006F022FF4D
:10B74000002541F69A79A06035E038F91510454E8C
:10B7500049452FD10027DFF810A11CE03946019898
:10B76000F9F7BEFE51460090FAF791FE90B90098A5
:10B7700001F052FF01280DD1009801F043FFA842CB
:10B7800008D10098FAF75DFEB04203DB0098FAF7A3
:10B7900058FE06467F1C0198F9F7B4FEB842DDD882
:10B7A000002E03DBA06820F8156003E0A1680020EC
:10B7B00021F815006D1C2069A842C6D800252F4627
:10B7C000284641F69B764A4615E038F91010B142FA
:10B7D00004DB0D44A5F5F8559B3D0BE0914204D1E7
:10B7E000A16831F81010394403E0A36823F8101061
:10B7F00039440FB2401C21698142E6D800210198EA
:10B8000007F040F92169C1F1010200FB02B0C01B41
:10B8100001B2002900DA002100224FF0FF37104664
:10B8200010E038F91030B3420BDBA3F5F8539B3B23
:10B830001AB211FB02F3B3FBF5F3A76827F8103037
:10B840000746401C23698342EBD8002F07DBA81A68
:10B850004843B0FBF5F0081AA16821F81700BDE8CD
:10B86000FE8F000001E0FFFF010006002DE9F84F08
:10B870000C46834602F03CF8804600F087FA60618F
:10B88000400006F07FFE60606069400006F07AFECE
:10B89000002541F69A79E06035E038F91510474EF9
:10B8A00049452FD10027DFF818A11CE0394658463A
:10B8B000F9F716FE51460090FAF7E9FD90B90098A5
:10B8C00002F028F801280DD1009802F019F8A842DA
:10B8D00008D10098F9F7C9FEB04203DB0098F9F7E8
:10B8E000C4FE06467F1C5846F9F70CFEB842DDD868
:10B8F000002E03DBE06820F8156003E0E16800201B
:10B9000021F815006D1C6069A842C6D800252F4695
:10B91000284641F69B764A4615E038F91010B142A8
:10B9200004DB0D44A5F5F8559B3D0BE0914204D195
:10B93000E16831F81010394403E0E36823F810108F
:10B9400039440FB2401C61698142E6D80021584653
:10B9500007F0C8F881465846F9F726FE6169C1F13B
:10B96000010209FB0200C01B01B2002900DA00211C
:10B9700000224FF0FF37104610E038F91030B34284
:10B980000BDBA3F5F8539B3B1AB211FB02F3B3FB9D
:10B99000F5F3E76827F810300746401C63698342D7
:10B9A000EBD8002F07DBA81A4843B0FBF5F0081AC4
:10B9B000E16821F81700BDE8F88F000001E0FFFF03
:10B9C000010006002DE9FF4F87B0C878189CC0071A
:10B9D0000D46002801D0E84800E0E848059001D075
:10B9E000E74800E0E748824601D1E54800E0E54845
:10B9F00004906188A2884FF0000BA1EB0201584629
:10BA000009B25A46D4F810C010E002EB82034FF09E
:10BA10001007E66807EB8307F75DFF070AD00827E2
:10BA200007EB8303F35AC91A09B2521C9445ECD8A8
:10BA3000002246E00C2707EB8303F35A184400B2B8
:10BA4000F3E709EB89031022E66802EB8302009218
:10BA5000B25CD20733D1A8B191FBF0F70C2202EB14
:10BA6000830E36F80E207A43042707EB830736F956
:10BA700007C0062707EB8307F75F12B2974202DD84
:10BA8000904601E0FEE7B846C44501DD674602E0A6
:10BA9000974200DD1746974205D0009A4FF0010CFF
:10BAA000E34646F802C0E668082202EB8302B7527A
:10BAB000E36833F80E20801AC91B00B209B209F1FD
:10BAC0000102236991464B45BBD8BBF1000F90D1D1
:10BAD0000021079806F096FF012800D00020834639
:10BAE0000020ADF80800ADF80C0003A902A8CDE9CC
:10BAF00000012089B4F9022003B22878169908F0D1
:10BB0000E8FDE97811EA0B0F07D00798F9F768FD0F
:10BB1000BDF808100844ADF8080009990798F9F72E
:10BB2000DFFC0BE098493046FAF7B1FC78B1E878D1
:10BB300009AAC0F38001079801F0C7FE060003D0F0
:10BB4000DDE909018842EDD10BB0BDE8F08F00219D
:10BB5000304606F069FFE8B30027384621690FE058
:10BB6000E26800EB800352F82320B24207D100EBD9
:10BB70008002E168082000EB82000F5E02E0401CBA
:10BB80008142EDD8E878C007708C04D020F4806042
:10BB900040F4006003E020F4006040F480607084B2
:10BBA00006F11400804651468847B84228D03046F6
:10BBB000FAF7F7FEB08AADF80000F08AADF802009F
:10BBC000308BADF80400708BADF806003946404666
:10BBD000059A00E010E090476A462921304604F0BB
:10BBE00065FA3046F9F77CFD3246222104F05EFA10
:10BBF0003046FAF7D6FE03E0708C20F44060708483
:10BC000068784FF0000901280FD0022815D1049957
:10BC100006F114008847B4F90010491C21F0010115
:10BC2000081A00EBD070401005E0049906F11400EA
:10BC300088472188081A0FFA80F9E87810EA0B0F74
:10BC400008D006F1140051468847BDF80810081ABC
:10BC5000ADF80800304600216B22FAF7A6FA0FFA79
:10BC600080F8304600216C22FAF79FFA07B230467E
:10BC7000FAF7E7FB00903046F9F7F7FC0146C8F306
:10BC80004130012810D128F4C040B0F5FA6F0BDC28
:10BC9000B0F57A7F01DDC0F57A70009A50436422D6
:10BCA00090FBF2F00FFA80F8C7F3413001280ED173
:10BCB00027F4C040B0F5FA6F09DCB0F57A7F01DDFA
:10BCC000C0F57A704843642190FBF1F007B2B18A65
:10BCD0001498411A01EB080002B2F18A1598401A33
:10BCE000384401B2E878C007002802D0BDF9080046
:10BCF00000E04846104407B201D0484601E0BDF9D3
:10BD0000080008440FFA80F857EA080019D03046B6
:10BD1000FAF747FEB08A3844B082308B384430831B
:10BD2000F18A01EB0800F082718B01EB080070834F
:10BD30003046FAF736FE0023424639463046FAF7D7
:10BD4000D7FEE87810EA0B0F0CD106F1140051462B
:10BD5000884717990844BDF80C100844BDF808102E
:10BD6000084406E0BDF80C1017980844BDF8081008
:10BD7000081AADF80800DAE665F801085BF8010872
:10BD8000F5F70108A9F701080100060001460020A7
:10BD900041F6FF7200E0401C31F910309342FAD1B5
:10BDA000704708B50846114603F08CFE0090BDF8B8
:10BDB000000008BD2DE9F04F93B0834604F033F93D
:10BDC0000646584604F06DF90446122E7ED0152E14
:10BDD00001D0182E7BD1FAF734FB06902046F9F7F4
:10BDE00044FC0590204600213222FAF7DEF9054690
:10BDF000204600211222FAF7D8F928440FFA80F8D9
:10BE0000204600211322FAF7D0F928440FFA80FACD
:10BE1000204600211022FAF7C8F9284407B220462C
:10BE200000211122FAF7C1F92844618E0FFA80F936
:10BE300001EB0800ADF83C00A08E3844ADF83E00A0
:10BE400094F8390000F0030001287DD00FA9E08E9E
:10BE5000CDE90001DDE90521B4F9303003A8FEF792
:10BE600039FABDF80C10A08A0844ADF80C00BDF8F2
:10BE70000E10E08A0844ADF80E00BDF81010A08A3C
:10BE80000844ADF81000BDF81210E08A0844ADF87F
:10BE9000120004F114010D4610A80D9103F075FC79
:10BEA00003A9284603F071FC5946D24806F07BFDF1
:10BEB000012860D110A90D9803F067FC152E5AD106
:10BEC000E08D002857D0A08D002801E056E052E018
:10BED00051D0E08E00284ED0584604F0AAF806460D
:10BEE00001A80D9903F051FC204605F0B1FB054671
:10BEF00094F8390000F0030001287CD0BDF8100050
:10BF0000BDF80C10401ABDF804100844ADF8080044
:10BF1000BDF81200BDF80E10401ABDF80610084416
:10BF2000BDF80410ADF80A0001EB0800ADF80400FC
:10BF3000BDF80600BDF808103844ADF80600A1EBC6
:10BF40000A00ADF8080000E07DE0BDF80A10A1EBA2
:10BF50000900ADF80A0094F8381001F00300012838
:10BF60006FD089076DD002286CD000231946304667
:10BF70000D9AF5F7A3FF13B0BDE8F08F584604F013
:10BF80008EF8054600780228F5D094F838004FF076
:10BF90000106C14389074ED000F0030102294AD0AF
:10BFA000C0F38400042801D0012844D12046002198
:10BFB0004622FAF7FAF8C0B2FF283CD1208ED0BB57
:10BFC000584604F06CF80746E08EB0F5807F34D018
:10BFD0002046F9F74AFB80462046FAF732FA014636
:10BFE00004F13202E08ECDE900020023424602A8AD
:10BFF000FEF770F900E02BE0BDF80800A18A0022EE
:10C000000844ADF80800BDF80A00E18A0844ADF81C
:10C010000A00BDF80C00A18A0844ADF80C00BDF878
:10C020000E00E18A0844ADF80E0002A93846FDF77B
:10C03000B8FF00289FD12E709DE7002204F1140163
:10C04000F4E730E0C5E003A92046F9F7E5FA20E778
:10C05000B4F92C0029B2401ABDF80410401C00EBC2
:10C06000D070A1EB6001ADF80410BDF80810BDF868
:10C070000620A1EB6000ADF80800B4F92E002914E9
:10C08000401A401C00EBD070A2EB6000ADF8060037
:10C09000B4F92E00401ABDF80A10401C00EBD07015
:10C0A000A1EB60003CE707A8F5F73CFF07AA0021D9
:10C0B0002046FAF776FAE08EADF81E00208EADF835
:10C0C0001C00608EADF82000A08EADF8220094F820
:10C0D0003800BDF80C10C0098DF8300001EB0800E5
:10C0E000ADF83400BDF80E00BDF810103844ADF8BE
:10C0F0003600A1EB0A00ADF83800BDF812100DAA09
:10C10000A1EB0900ADF83A00B16810468846FDF78A
:10C1100020FF002890D00DA8B060B4F92800B4F931
:10C120002C1090FBF1F201FB1207B4F92A00B4F9CC
:10C130002E1090FBF1F201FB1200BDF9061008442D
:10C1400000B2ADF81600884203DDE18D401AADF86B
:10C150001600E18D80B20844401E2FE0BDF90410A6
:10C16000C81900B2ADF81400884203DDA18D401A51
:10C17000ADF81400A18D80B20844401E0DE005AA60
:10C1800007A93046636AF5F799FEBDF81400284404
:10C19000ADF81400BDF818002844ADF81800BDF93A
:10C1A0001400BDF908108842E9DBBDF81610281408
:10C1B0000144ADF81610BDF81A100844ADF81A0085
:10C1C000BDF91600BDF90A108842C7DBC6F8088021
:10C1D000D1E605A8F6F756F905AA00212046FAF798
:10C1E00033FA00200090636A05A930460D9AF5F7EE
:10C1F000B3FEC0E6585B02082DE9F0438FB0044659
:10C2000003F04FFF0546F9F76BFA064601A8F6F76B
:10C2100039F901AA00213046FAF716FA284605F046
:10C2200043FE28B19DF8210040F001008DF8210067
:10C23000204603F0FEFE816804460F4606F1140214
:10C240000DA8FDF786FE002850D00DA8A0600BA910
:10C25000304601F069FBA88AADF82400E88AADF801
:10C260002600288BADF82800BDF82E00ADF82A0076
:10C2700009AA1046A168FDF76CFE4FF000080DF109
:10C28000240978B1A6682846C4F8089005F011FE84
:10C29000034605F1140201A92046CDF80080F5F708
:10C2A0005BFEA660A88AADF82400BDF83200ADF8A8
:10C2B0002600288BADF82800688BADF82A0009AA63
:10C2C0001046A168FDF745FE78B1A6682846C4F877
:10C2D000089005F0EEFD034605F1140201A9204681
:10C2E000CDF80080F5F738FEA660A7600FB0BDE876
:10C2F000F0832DE9F04790B0054603F0D2FE0446E6
:10C30000284603F096FE06460BA92046F9F71EF9CB
:10C3100094F848000025C10600D50125800601D506
:10C3200045F002050021204606F030FCA0F51C5126
:10C33000D13904D1608C000501D445F0040503A86F
:10C34000F6F7A0F8B4F84400ADF82200B4F84600BF
:10C35000ADF824008DF8295003AA00212046FAF7F1
:10C3600073F99DF828004FF0010808B98DF828806E
:10C37000E06B0490206C059004994FF6FF708142A9
:10C380001ED0059981421BD04FF4802927465522A3
:10C3900049462046F9F709FF024649463846F0F774
:10C3A00090F80090BDF80000ADF81A002046202259
:10C3B0004946F9F7FAFE0090BDF80000ADF81C0000
:10C3C00094F8480041F6FF7A00F00700022801D0F7
:10C3D00003281AD19DF82800022801D0032814D17F
:10C3E000BDF91E10CDE9001A0295BDF92030039A5F
:10C3F0000DA8616A07F0D0FF0BA803F007FABDF99A
:10C400003410884201DA8DF8288094F8480004F14D
:10C41000300700F00700032805D00BA803F0D0F97F
:10C42000B0F5806F00DA00270BA90EA8B268FDF7FF
:10C4300090FD00287DD094F8480040070BD120469D
:10C44000F9F780FA404202B200210BA803F0F1F99B
:10C45000608BADF8320094F848000DF1380900F017
:10C460000700022813D0032811D000970BAA03A9B4
:10C470003046636AF5F770FDB068C6F808908046EC
:10C4800094F8480000F0070003280FD058E0D6F8D1
:10C490000880C6F8089000970BAA03A93046636A83
:10C4A000F5F75AFD4046C6F80880E6E7BDF91E10CC
:10C4B000CDE9001A0295BDF92030039A0DA8616AF2
:10C4C00007F06AFF0BA803F0A1F9BDF93410884208
:10C4D00019DA20221146039803F0FDFEB4F8441047
:10C4E000BDF8342000EB400011440844ADF82200B0
:10C4F000B4F84600ADF8240000970BAA03A9304613
:10C50000636AF5F729FD0BA803F05AF90146BDF956
:10C510003600814214DAB4F84410ADF822100399C1
:10C52000B4F84620098910440844ADF82400009767
:10C5300000E007E00BAA03A93046636AF5F70CFD9B
:10C54000C6F8088010B0BDE8F0872DE9F04393B03D
:10C55000074603F068FD0546384603F0A2FD044691
:10C560004FF48026152D7ED0182D7DD1384603F04E
:10C5700060FD054603A8F5F785FF03AA314620466E
:10C58000FAF762F80EA9204601F0CEF90EAA10A81B
:10C59000A968FDF7DEFC002866D0204601F092F97C
:10C5A000814605F081FC28B19DF8290040F001008A
:10C5B0008DF829002046F9F744FF0646484605F065
:10C5C00078FC0146BDF91E00CDE900060222029268
:10C5D000BDF920300DA8039A07F0DEFE2046F9F7DA
:10C5E00044F8B4F9161000EBD076B9F9160001EB57
:10C5F0006601471A4846F9F738F8B90391FBF0F796
:10C600000021204606F095FA0399B0F90800B1F927
:10C610000810081A00EBD070BDF836104010091A47
:10C6200009B2ADF83610E28A794302EB660202EBFA
:10C63000A1310E1A0021204606F0F0F9804620466E
:10C6400000211222F9F7B1FD0746204600211322EE
:10C65000F9F7ABFDA28A07EB08011144ADF82C10E5
:10C66000ADF82E6001E023E01FE0218B081AA0EB5B
:10C670000800ADF83000BDF836003044ADF83200A7
:10C680009DF8290040F002008DF8290010A8AC6840
:10C69000A860484605F00DFC0346002000900BAA58
:10C6A00003A92846F5F758FCAC6013B0BDE8F08349
:10C6B000384603F0BEFC05460EA9204601F034F9C9
:10C6C0006846F6F7BBFC6A4631462046FAF70CF896
:10C6D0000EAA69462846F6F79DFCE6E72DE9F043E9
:10C6E000A1B0054603F0DDFC0446284603F0A1FC9A
:10C6F00081460021204606F0D7F907460021204652
:10C7000006F0E4F906460021204606F0FDF905464C
:10C710000021204606F0AAF9A38AE28AADF87A2021
:10C72000218BADF87C10B4F81AC0891BADF87C10D1
:10C730003B44ACEB0000ADF878305119ADF87E0009
:10C74000ADF87A106846F6F779FC6A464FF4003186
:10C750002046F9F7C9FF1EAA69464846F6F75AFC73
:10C760002046F8F782FF0646208BA18A401A401C1B
:10C77000801B05B2606A411C06D06843C11700EBFC
:10C780001160001207B208E02046F9F73BFCC0F345
:10C79000000008B12F4600E00027204600211622A5
:10C7A000F9F703FDC0B2012801D1E81B07B2A08A46
:10C7B0004FF440353844ADF870003044ADF87400A3
:10C7C000E08AADF87200608BADF87600294620460D
:10C7D00006F06AF907462946204606F077F98046B2
:10C7E0002946204606F090F906462946204606F0DE
:10C7F0003DF9BDF87010BDF87420C91BADF870107C
:10C8000002EB0801ADF87410BDF87210891BADF889
:10C810007210BDF876100844ADF876000EA8F6F751
:10C820000DFC0EAA29462046F9F75EFF1CAA0EA9A8
:10C830004846F6F7EFFB21B0BDE8F0832DE9FF4F46
:10C8400081B00C4680462021DDF838A0F9F718FEAB
:10C85000002878D0BAF1030F404621D0F9F76BF8E1
:10C86000814605F007F80546002708F114000090FE
:10C870003E46BAF1030F3946404614D006F038F967
:10C8800082460021404606F0E5F883464846B9F165
:10C89000010F59D002285FD0B9F1030F63D138E0FE
:10C8A000F9F742F8DCE706F0F3F88346002140464A
:10C8B00006F000F982464846B9F1010F19D0022866
:10C8C0001FD0B9F1030F4ED1009802F08DFFA0EBFD
:10C8D0000B01A1EB0A00B8F8141000EBD0720BEBBF
:10C8E0006200084407B205F1140002F07DFFA98A36
:10C8F00023E0B8F81410B5F9146001EB0B0007B28F
:10C9000031E0B8F81810B5F91860A1EB0A0007B2C9
:10C9100029E0009802F042FFA0EB0A01A1EB0B0016
:10C92000B8F8161000EBD0720AEB6200084407B2A8
:10C9300005F1140002F032FFE98A00EBD07001EB40
:10C94000600006B20FE030E0B8F81610B5F91660D6
:10C9500001EB0A0007B206E0B8F81A10B5F91A6040
:10C96000A1EB0B0007B2A01E049900B2002910DA57
:10C97000B9F1000F15D0BE4221DC12E0002C01DD20
:10C98000A41C24B2E01704EB9070801005B0BDE841
:10C99000F08F0399002912DAB9F1000F01D0BE42DD
:10C9A0000DDB002CEADA0446E8E70498E04202D501
:10C9B0000498404204B20398001B00D5039C204613
:10C9C000E4E770B5044604F045FF48B100688268AA
:10C9D0000AB1217A9047207E810743D4C0077CD1D9
:10C9E00001260021606805F0F4FF00251AE00168C7
:10C9F00099B1017ACA0910D0802904D0227A21F095
:10CA00008001914209D14168E16001682046884770
:10CA1000207E810726D4C0075FD16D1C294660683F
:10CA200005F0D7FF08B1002EE1D12146002005F026
:10CA3000BAFF051E03D00021606805F0CAFF00267A
:10CA400019E0016891B1017A0A060FD411B1227A76
:10CA500091420BD14168E160016820468847207E01
:10CA6000810701D5012070BDC00736D1761C314643
:10CA7000606805F0AEFF10B1012DE2D02FE0012D6E
:10CA80002DD16068416851B3217E490727D4217AAE
:10CA9000232919D0242917D0A903F9F7F1FCF0B103
:10CAA000207A11381C280FD2DFE800F01919191963
:10CAB000191919191919190E0E190E0E1919191912
:10CAC0000E0E0E0E19190E1960684068606020463F
:10CAD000FFF777FF0546012801D0002070BD2846EA
:10CAE00070BD2DE9F04F89B00546002002900390FB
:10CAF00004F0B0FE00680026B146047E686A00902B
:10CB0000288BA98A08442883688BE98A08446883AB
:10CB10000098E5E04FF000084FF48077CDF81C80D6
:10CB200000980EE0002106F019F840440FFA80F852
:10CB30000021504606F018F847433F125046F8F7D8
:10CB4000CFFD5FEA000A5046ECD1A8690190B8F128
:10CB5000000F02D1B7F5807F0AD0C8F1000001B202
:10CB60004FF4803090FBF7F207AB01A806F0A2F873
:10CB7000BDF90410002900DC4942BDF90600002877
:10CB800000DC4042814201DD012601E04FF0010955
:10CB900010210098F9F774FC00287ED0B046CB46EF
:10CBA000CA4647460098F8F7F9FDC10700D1884604
:10CBB000810700D40027410701D44FF0000B000784
:10CBC00001D44FF0000A0098F8F7BCFE06900098D8
:10CBD000F8F792FD05900098F8F7E8FD04900098AA
:10CBE000F8F744FE0699002902DC0599002912DDB8
:10CBF000BBF1000F03D0BDF90610A14207DABAF16C
:10CC0000000F08D0BDF906106242914203DC009982
:10CC100002910C2103910499002901DC002810DD08
:10CC2000B8F1000F03D0BDF90410A14205DA47B1F5
:10CC3000BDF904106242914203DC00990291032184
:10CC400003910699002901DC4FF0000B059900299A
:10CC500001DC4FF0000A0499002901DC4FF00008C4
:10CC6000002800DC0027B8F1000F03D0BDF9040054
:10CC7000A04216DA27B1BDF904006142884210DDF6
:10CC8000BBF1000F03D0BDF90600A04209DABAF1EA
:10CC9000000F11D0BDF9060000E00DE061428842AE
:10CCA0000ADC0EB1032000E00C2095F8401060F380
:10CCB000030185F8401016E04FF480710098F9F7F1
:10CCC000DFFB36EA00000ED14FF400710098F9F74F
:10CCD000D7FB39EA000006D10098F8F701FD009073
:10CCE00000287FF417AF029858B195F840000399D7
:10CCF00061F3030085F840000298E8620020288371
:10CD00006883029809B0BDE8F08F00002DE9FF5F4D
:10CD10000646F8F709FEB0F1000A72D041F6FF743A
:10CD20000021304605F0B4FE80460021304605F073
:10CD3000C1FE81463046F8F7E5FB8346002758E000
:10CD4000B0683249006850F827502846F9F79FFB31
:10CD5000F0BB4FF480512846F9F792FBC0B3504620
:10CD6000BAF1010F05D0022809D0BAF1030F3FD163
:10CD70001AE0B18AB5F9145001EB080004E0318BD8
:10CD8000B5F91850A1EB09000399019A294409B299
:10CD900000B291422CDB029A914229DC081A00B2BF
:10CDA00000281CDD01461BE005F1140002F01CFD0B
:10CDB000A98A00EBD07001EB600005B206F1140007
:10CDC00002F012FDA0EB0801A1EB0900B18A00E01E
:10CDD0000EE000EBD07208EB62000844D4E7414259
:10CDE000002C01DD224600E06242914200DA044656
:10CDF0007F1C5F45A4D3A4F5F850FF3804D06042EF
:10CE000000B204B0BDE8F09F0020F9E70100040083
:10CE10002DE9FF5F0646F8F78EFDB0F1000A72D0EB
:10CE200041F6FF740021304605F062FE8046002185
:10CE3000304605F00FFE81463046F8F763FB834627
:10CE4000002758E0B0683249006850F8275028465B
:10CE5000F9F71DFBF0BB4FF480512846F9F710FBA2
:10CE6000C0B35046BAF1010F05D0022809D0BAF17B
:10CE7000030F3FD11AE0F18AB5F9165001EB080013
:10CE800004E0718BB5F91A50A1EB09000399019ADE
:10CE9000294409B200B291422CDB029A914229DC6A
:10CEA000081A00B200281CDD01461BE005F1140041
:10CEB00002F074FCE98A00EBD07001EB600005B26F
:10CEC00006F1140002F06AFCA0EB0801A1EB0900D6
:10CED000F18A00E00EE000EBD07208EB620008443B
:10CEE000D4E74142002C01DD224600E0624291423B
:10CEF00000DA04467F1C5F45A4D3A4F5F850FF3840
:10CF000004D0604200B204B0BDE8F09F0020F9E711
:10CF1000010004002DE9FF4F83B00F46DDE910A4A6
:10CF200093460021039805F025FE0546002103984D
:10CF300005F084FDF9788A070BD5CB0742F2D17250
:10CF400002D0954202D007E0904207D121F00200C2
:10CF5000F870F878C00701D0744800E07448019078
:10CF6000F878C0070CD0724859468146002060808E
:10CF7000A08020612080A060E060CDF800B0A2E039
:10CF80006A48F1E70099594506D04FF40001304650
:10CF9000F9F776FA00287DD166493046F9F777FA35
:10CFA000002878D10021304605F03EFD5FEA0008F8
:10CFB0005CD02069401C2061A28802EB0A01A1809C
:10CFC000217DC90762D000EB8000800005F0DAFA0D
:10CFD00005001BD0E16851B12069401E00EB8000C4
:10CFE0008200284605F068FBE06805F017FB206921
:10CFF0004FF0000100EB800005EB800040F8146C5E
:10D00000F878C007304602D0022201E0FEE7052290
:10D01000F9F7CBF8216900B201EB810105EB810141
:10D0200021F8100CF8784FF00001C007304601D00D
:10D03000032200E00622F9F7B8F8216900B201EBFB
:10D04000810105EB810121F80E0C2069002100EB24
:10D05000800005EB800040F8088C206900EB800020
:10D0600005EB800040F8041CE5600FE001993046B4
:10D070008847F978890705D5B4F904100A18069984
:10D080008A4226DCA28850441044A080304649469B
:10D09000884701E01DE00BE00146B4F90000814241
:10D0A00002DD3046494688472080A068401CA060C9
:10D0B000F878400702D54FF0FF3000E001200099DA
:10D0C0004118009105D40398F8F70AFA061E7FF478
:10D0D00059AFB4F90400002802DDA0EB0A00A080DB
:10D0E000206908B1069801E0B4F904006080CEB16F
:10D0F0000098584516D103996A468968096851F81D
:10D100002050F878C0F38001039800F0DEFB4DB1A9
:10D1100028464946884720800199284688476080EC
:10D120000120A060009807B0BDE8F08F43640108BB
:10D130006B560108010006002DE9F04FB34D93B086
:10D14000044600216A88F9F730F89DF81710421C50
:10D1500062F30001820862F34101C00860F38201BA
:10D160008DF8171020460021AA88F9F71EF88DF8CF
:10D17000140020460021EA88F9F717F88DF8150009
:10D18000204600212A89F9F710F88DF816000021B1
:10D19000204605F037FC012800D0002083469DF88A
:10D1A00017004FF00001C00720460CD005F094FC9A
:10D1B00006469DF817004FF00001C007204605D035
:10D1C00005F05AFC04E005F057FCF1E705F084FC9B
:10D1D00081469DF81700C007204602D0F8F700FAF4
:10D1E00001E0F8F7E1F90C90204600213222F8F72F
:10D1F000DCFF0546204600211022F8F7D6FFE18A21
:10D20000284447182046F8F7ABFB381AADF834002D
:10D21000204600211222F8F7C8FFA18A28444518A9
:10D220002046F8F796FB281AADF83C009DF8170049
:10D230009DF81680C00701D00DAD00E00FAD0021B4
:10D24000204605F097FC11900021204605F0F6FBE2
:10D2500010909DF81700C10709D01099A1F51C5234
:10D26000D13A02D1618C490509D5C10709D111997B
:10D27000A1F51C52D13A04D1618C090501D44FF0BB
:10D280000008BBF1000F0CD0C0070AD1B8F1000FA5
:10D2900003D0B8F1010F02D003E0012000E000202C
:10D2A00080460027ADF83870BA46B8F1000F3AD082
:10D2B0009DF81700400703D5A0684268521E13E08E
:10D2C000002211E000200B9006A8CDE9009005A9EE
:10D2D00020460C9BFFF71EFEBDF81810BA1911442A
:10D2E0000FB20AF1010A0246A0684068904201DDCF
:10D2F000002AE7DABAF1000F01D0B81B07B29DF897
:10D300001700C007204602D0F8F74EF901E0F8F701
:10D3100067F90EA9CDE9005101460FFA8AF33A46A2
:10D32000404607F0D6F99DF81710480703D5A068C6
:10D330004068401E00E000208046BBF1000F04D092
:10D34000C80702D12888384428800DF1180AA0683F
:10D350004168414546DDB8F1000F43DB01200B90E9
:10D36000CDE9009A424605A920460C9BFFF7D2FD65
:10D370000746BBF1000F08D09DF81700C00704D185
:10D380002888BDF81810401A2880BDF934300C9A4E
:10D3900002A8019380E80406BDF93C0000903B46DA
:10D3A000424605A92046FEF70DFBB846099805F050
:10D3B00035F900200990BBF1000F03D09DF817004C
:10D3C000C00709D02888BDF818100844BDF83810E7
:10D3D000314408442880BAE7BDF838102888314421
:10D3E000401AF7E7119942F2D170814202D01099A8
:10D3F000814202D12046F9F7D3FD00222B2120469D
:10D4000002F054FE13B0BDE8F08F0000DC340020C1
:10D410002DE9F74F0546007F93464FF0000AC007FD
:10D4200060D14FF00108EC680026C1467CB9287F26
:10D43000C0F3C000401E304254D1B9F1000F51D0AA
:10D440000199284688474FF000080446C1460EB9A6
:10D45000261E47D0B8F1000F06D0214628465A466E
:10D4600090470446B0423DD04FF00108002CDDD07B
:10D470002068F8F7C7FD0006D8D427681FE001210F
:10D480003846F8F7FDFFB0B12FB101213846F8F763
:10D49000F7FF0028CAD1E868A04223D0B0B12846DF
:10D4A00000F054F90246E8680F21006802F0FEFD22
:10D4B000012817D106E03846F8F712F90746002F81
:10D4C000DDD1E8E7E8680068F9F76BFA2846EC6018
:10D4D00000F03CF90246E8680E21006802F0E6FD23
:10D4E000012802D05046BDE8FE8FE8680068F9F7D1
:10D4F00058FA296909B1284688470120F3E770B531
:10D50000426B818C12F0060F06D0C2F34102022A50
:10D5100004D0012A05D022E0008D00E0C08C084430
:10D520001CE0B0F92C40468DA2B2B24202D202F504
:10D53000B47214B2B0F92830C58C9AB2AA4202D2A1
:10D5400002F5B47003B2301900EBD0704010854280
:10D5500001DA681802E0834203DD501881B208B294
:10D5600070BD0844FAE72DE9F05F8946934682468C
:10D57000002105F093FA05460021504605F0A0FA77
:10D5800080460021504605F0B9FA04460021504675
:10D5900005F066FA06465046F8F753FF411BA1EB2B
:10D5A00008075046F8F761F8001B801B8742504679
:10D5B00005DAF8F746FF411BA1EB080003E0F8F796
:10D5C00054F8001B801B00EBD070401001B2BAF879
:10D5D00014004A191044A9F80000BAF816000A19F4
:10D5E0001044A9F80200BBF1000F01D0ABF8001005
:10D5F000BDE8F09F024A00215288F8F7D6BD00002E
:10D60000E8340020034A10B500215289F8F7CDFD17
:10D61000C0B210BDE8340020034A10B50021928941
:10D62000F8F7C3FDC0B210BDE83400202DE9FC4777
:10D630000F0023D005696C692CB12068B84202D173
:10D640006068BDE8FC87698A00204FF0040CC1F3D4
:10D6500008060CE0A96800EB800351F823200CEBCE
:10D660008303C95ABA1A91420AD2401C80B2864238
:10D67000F0D81CB127606969002048600020E0E70D
:10D6800000EB80041220A96800EB84000026085CEF
:10D690004FF0060902280CD04FF00C0A70B1DFF8E9
:10D6A000A8C008234FF0100803280FD0012826D067
:10D6B00043E009EB8400085A86183EE00AEB840038
:10D6C00009EB84030858C95A805C35E008EB8400F4
:10D6D000ADF80420CDF800C00A5A03EB84080223F9
:10D6E00051F8081001A8FDF7B9FA30B3A96851F84C
:10D6F0000820801A09EB84024010895A1CE008EBCC
:10D700008400ADF80420CDF800C00A5A03EB840869
:10D71000022351F8081001A8FDF7A0FA68B1A96822
:10D7200009EB840351F80820801A42100AEB8400A8
:10D730000858C95A30F812000E18686910B107600D
:10D740006869466030467CE7535702082DE9F0418E
:10D7500000260746354630460FE004F0BCF8616D00
:10D76000B94209D1022802D0042803D003E02046A0
:10D77000BDE8F08126462546204604F071F80400F5
:10D78000EBD10EB13046F3E70DB12846F0E7BDE826
:10D79000F041002004F064B87CB5036900690025FD
:10D7A0005B8AC4689B04A0682AD4830F16D0012327
:10D7B000B3EB907F30D101EB02402668019017480F
:10D7C0000090A068042320F04042314601A8FDF7F4
:10D7D00045FA08B3801B801061681CE001EB022150
:10D7E0002668ADF804100E4920F040420091022353
:10D7F000314601A8FDF732FA70B1801B4010EBE70B
:10D800006368805C595C39B130B1637B2268491E22
:10D8100011FB0321401E0D5628467CBD9DEC0108DE
:10D82000B1EC01082DE9FF4F81B00E461D461746A9
:10D830004FF40031019805F0DFF800EBD070441090
:10D840003F1B0198FFF75BFE81465A3000B206F09D
:10D85000D7FC10FB07F04FEAE038484606F0D0FC52
:10D8600010FB07F0C7134FF440394946019805F003
:10D8700015F983464946019805F022F9009049467A
:10D88000019805F03BF982464946019805F0E8F811
:10D89000328820444244A2EB0B01091B29803288C4
:10D8A0000099424421441144A9807188CA19A2EB0D
:10D8B0000A01091B6980718839440844E88005B071
:10D8C000BDE8F08F0021F7F70BBE136821B15B1E96
:10D8D00013600BD4806805E05B1C136080684168AE
:10D8E0008B4203DA006850F823007047002070472D
:10D8F000024A0021D288F8F758BC0000E834002022
:10D90000034A10B50021128AF8F74FFCC0B210BDCF
:10D91000E8340020034A10B50021528AF8F745FC8C
:10D92000C0B210BDE83400202DE9FC410C4606468B
:10D93000002105F0FEF805464FF48021304605F041
:10D94000F8F8B5F90870B0F908500021304605F034
:10D95000FFF80146E81900EBD07001EB600005B25A
:10D960003046F7F782FEF18A00EBD07001EB6000E1
:10D9700005EBD571A0EB610060802844E08069462A
:10D980003046F7F749FEBDF800002080BDF80400DE
:10D99000A080BDE8FC812DE9FF410746FFF792FF1B
:10D9A000040020D04FF480252946384605F0C1F800
:10D9B0000646384658222946F8F7F7FB05B22046B6
:10D9C00004F077FA0146002041F6FF72CDE900022B
:10D9D00002902B46324603A806F0DEFCBDF90C008F
:10D9E00004B0BDE8F0810020FAE7000038B50C482B
:10D9F0000D46144690F820004FF00201C0074FF08A
:10DA0000120002D005F014F901E005F029F92246D0
:10DA1000294602F0E7F80090BDF8000038BD00008C
:10DA2000CC7C00202DE9F0474FF0000CDDE90964C3
:10DA3000089DDDF82CA0E1466F1EF9B9052A03D038
:10DA4000062A01D0042A03D10023012D00D101228E
:10DA5000002106E036F811809C44C4440FFA8CFC87
:10DA6000491CA942F6D3ACEB030109B2072A2AD21A
:10DA7000DFE802F004070B2921160D00A4F800903E
:10DA800021E0411A01EBD17112E0411A11E0411A73
:10DA900009B23AB291FBF2F1A4F800900BB212E095
:10DAA000411A09B22AB291FBF2F10BB203EBD37126
:10DAB0004910218007E0411A0AB2691C09B292FBA1
:10DAC000F1F10BB2238000210AE034F8112036F87E
:10DAD00011C0624404EB410C1A44ACF80220491C0A
:10DAE000B942F2D304EB450106EB450231F8021CC2
:10DAF00032F8022C11442288891A0BB2BAF1000FB5
:10DB00000CD0002108E034F8112036F81170821A88
:10DB1000D21B24F81120491CA942F4D31846BDE8B1
:10DB2000F08770B58AB00546FFF764FD04462846C5
:10DB3000FFF7DEFE002C5CD000285AD0694628464C
:10DB4000FDF766FD0C2107A804F085FE284600219C
:10DB50003222F8F72AFB0446284600211222F8F761
:10DB600024FB0619284600211022F8F71EFB044466
:10DB70002846F7F7EEFEA98A3144081AADF82400CA
:10DB80002846F7F7EDFEE98A2144081AADF8260089
:10DB9000002407E0006807AA694650F8240000F056
:10DBA00013FF641CA8684168A142F3D8009804F0F0
:10DBB00035FD019804F032FD029804F02FFD039822
:10DBC00004F02CFD0021284604F0DAFF0446002171
:10DBD000284604F039FF42F2D1718C4201D08842CC
:10DBE00002D12846F9F7DCF900222B21284602F061
:10DBF0005DFA0AB070BD2DE9F0410446806D0D4616
